:020000040800F2
:100000008C010020BD020008D1020008D3020008C4
:10001000D5020008D7020008D9020008000000003D
:10002000000000000000000000000000DB020008EB
:10003000DD02000800000000DF020008E102000805
:10004000E3020008E5020008E7020008E9020008F0
:10005000EB020008ED020008EF020008F1020008C0
:10006000F3020008F5020008F7020008E79C0B08FD
:10007000FB020008FD020008C1990B0801030008FB
:10008000030300080503000807030008090300082C
:100090000B0300080D0300080F03000811030008FC
:1000A00029980B0869980B08DB980B0819030008BE
:1000B000A1950B087D970B08B9970B082103000841
:1000C000230300082503000827030008290300086C
:1000D0002B0300082D030008DDA70B0831030008DF
:1000E0003303000835030008370300081B990B0889
:1000F00039990B0867990B083F030008599D0B08B5
:100100004303000845030008F5970B08490300085E
:100110008DA80B084D030008A7990B08BB950B0889
:10012000530300085503000857030008E7A80B080D
:100130005B0300085D0300085F030008610300081B
:1001400063030008650300086703000869030008EB
:100150006B030008459B0B086F03000837A80B08CA
:10016000730300087503000877030008790300088B
:100170007B0300087D0300087F030008810300085B
:10018000830300088503000887030008890300082B
:100190008B0300088D0300088F0300082D9D0B08BA
:0C01A00093030008950300089703000873
:1001AC002A49072291438D4629482A492A4A00F0B8
:1001BC003AF82A482A492B4A00F035F82A482B49A4
:1001CC002B4A00F030F82B482B492C4A00F02BF826
:1001DC002B482C492C4A00F026F82C482C492D4A47
:1001EC0000F021F82C482D49002200F027F82C486B
:1001FC002C49091A082903DB002202600430016033
:10020C001D481E49884205D00268043003B490474B
:10021C0003BCF7E700208646EC4600200021BBE03B
:10022C00214A9047FEE7884207D0521A05D003783E
:10023C0001300B700131013AF9D17047884202D07C
:10024C0002700130FAE77047184870478C010020A3
:10025C0004B80B080000002000000020A4030008D4
:10026C00A4030008E4B70B0804B80B080000002036
:10027C0000000020E4B70B08E4B70B08E4B70B0848
:10028C00E4B70B08E4B70B08E4B70B08E4B70B08AA
:10029C00E4B70B0804B80B08000000200C00002089
:1002AC000C0000208C000020A4030008FFFFFFFFBF
:1002BC003648854600F005F8354836490160FFF7A9
:1002CC006FBF7047FEE7FEE7FEE7FEE7FEE7FEE7DF
:1002DC00FEE7FEE7FEE7FEE7FEE7FEE7FEE7FEE7EA
:1002EC00FEE7FEE7FEE7FEE7FEE7FEE7FEE7FEE7DA
:1002FC00FEE7FEE7FEE7FEE7FEE7FEE7FEE7FEE7CA
:10030C00FEE7FEE7FEE7FEE7FEE7FEE7FEE7FEE7B9
:10031C00FEE7FEE7FEE7FEE7FEE7FEE7FEE7FEE7A9
:10032C00FEE7FEE7FEE7FEE7FEE7FEE7FEE7FEE799
:10033C00FEE7FEE7FEE7FEE7FEE7FEE7FEE7FEE789
:10034C00FEE7FEE7FEE7FEE7FEE7FEE7FEE7FEE779
:10035C00FEE7FEE7FEE7FEE7FEE7FEE7FEE7FEE769
:10036C00FEE7FEE7FEE7FEE7FEE7FEE7FEE7FEE759
:10037C00FEE7FEE7FEE7FEE7FEE7FEE7FEE7FEE749
:10038C00FEE7FEE7FEE7FEE7FEE7FEE700000320E0
:08039C0008ED00E0000000087C
:1003A40003F02CBE0000000000000000000000006C
:1003B4000000000000000000000000000000000039
:1003C4000000000000000000000000000000000029
:1003D4000000000000000000000000000000000019
:1003E4000000000000000000000000000000000009
:103FF4000000000000000000000000000BF0FEBF05
:1040040000000000000000000000000000000000AC
:10401400000000000000000000000000000000009C
:10402400000000000000000000000000000000008C
:10403400000000000000000000000000000000007C
:020000040801F1
:100000004FF0005040F26E36A0F8CC64A0F8CC65FA
:10001000A0F8CC66A0F8CC67A0F8CC68A0F8CC69B2
:10002000A0F8CC6AA0F8CC6B40F2200680F8B06251
:1000300040F24E0680F8B16240F2650680F8B26286
:1000400040F2770680F8B36240F2200680F8B4628E
:1000500040F2530680F8B56240F2610680F8B6625D
:1000600040F26D0680F8B76240F2700680F8B86220
:1000700040F26C0680F8B96240F2650680F8BA6218
:1000800040F2200680F8BB6240F2200680F8BC6295
:1000900040F2200680F8BD6240F2200680F8BE6281
:1000A00040F2200680F8BF6240F2500680F8206DD2
:1000B00080F8066F467440F25A06A0F8BA604FF016
:1000C000180680F8BB634FF0030680F8C6606FF037
:1000D0000006C0F8E464C0F8E465C0F8E466C0F85F
:1000E000E467C0F8E468C0F8E469C0F8E46AC0F8FE
:1000F000E46B8665C0F88062C0F8846280F82D6188
:100100004FF0010680F832616FF0000645F20041C1
:10011000C1F2000101F5007241F8046B9142FBD17C
:100120006FF0000645F20061C1F2000101F50072B6
:1001300041F8046B9142FBD14FF04E0680F86063AA
:100140004FF0450680F861634FF0570680F8626310
:100150004FF05F0680F863634FF0440680F86463F5
:100160004FF0490680F865634FF0520680F86663E9
:100170004FF05F0680F8676349F20070C1F200003B
:1001800040F2800100F8011B40F2830100F8011BDE
:1001900040F2860100F8011B40F2890100F8011BC2
:1001A00040F28D0100F8011B40F2900100F8011BA4
:1001B00040F2930100F8011B40F2960100F8011B88
:1001C00040F2990100F8011B40F29C0100F8011B6C
:1001D00040F29F0100F8011B40F2A20100F8011B50
:1001E00040F2A50100F8011B40F2A80100F8011B34
:1001F00040F2AB0100F8011B40F2AE0100F8011B18
:1002000040F2B10100F8011B40F2B40100F8011BFB
:1002100040F2B70100F8011B40F2BA0100F8011BDF
:1002200040F2BC0100F8011B40F2BF0100F8011BC5
:1002300040F2C20100F8011B40F2C40100F8011BAA
:1002400040F2C70100F8011B40F2CA0100F8011B8F
:1002500040F2CC0100F8011B40F2CF0100F8011B75
:1002600040F2D10100F8011B40F2D30100F8011B5C
:1002700040F2D60100F8011B40F2D80100F8011B42
:1002800040F2DA0100F8011B40F2DD0100F8011B29
:1002900040F2DF0100F8011B40F2E10100F8011B10
:1002A00040F2E30100F8011B40F2E50100F8011BF8
:1002B00040F2E70100F8011B40F2E80100F8011BE1
:1002C00040F2EA0100F8011B40F2EC0100F8011BCA
:1002D00040F2ED0100F8011B40F2EF0100F8011BB4
:1002E00040F2F10100F8011B40F2F20100F8011B9D
:1002F00040F2F30100F8011B40F2F50100F8011B88
:1003000040F2F60100F8011B40F2F70100F8011B72
:1003100040F2F80100F8011B40F2F90100F8011B5E
:1003200040F2FA0100F8011B40F2FB0100F8011B4A
:1003300040F2FC0100F8011B40F2FC0100F8011B37
:1003400040F2FD0100F8011B40F2FD0100F8011B25
:1003500040F2FE0100F8011B40F2FE0100F8011B13
:1003600040F2FE0100F8011B40F2FE0100F8011B03
:1003700040F2FE0100F8011B40F2FF0100F8011BF2
:1003800040F2FF0100F8011B40F2FF0100F8011BE1
:1003900040F2FE0100F8011B40F2FE0100F8011BD3
:1003A00040F2FE0100F8011B40F2FE0100F8011BC3
:1003B00040F2FE0100F8011B40F2FD0100F8011BB4
:1003C00040F2FD0100F8011B40F2FC0100F8011BA6
:1003D00040F2FB0100F8011B40F2FA0100F8011B9A
:1003E00040F2F90100F8011B40F2F80100F8011B8E
:1003F00040F2F70100F8011B40F2F60100F8011B82
:1004000040F2F50100F8011B40F2F40100F8011B75
:1004100040F2F30100F8011B40F2F10100F8011B6A
:1004200040F2F00100F8011B40F2EE0100F8011B60
:1004300040F2ED0100F8011B40F2EB0100F8011B56
:1004400040F2E90100F8011B40F2E70100F8011B4E
:1004500040F2E60100F8011B40F2E40100F8011B44
:1004600040F2E20100F8011B40F2E00100F8011B3C
:1004700040F2DE0100F8011B40F2DB0100F8011B35
:1004800040F2D90100F8011B40F2D70100F8011B2E
:1004900040F2D50100F8011B40F2D20100F8011B27
:1004A00040F2D00100F8011B40F2CD0100F8011B21
:1004B00040F2CB0100F8011B40F2C80100F8011B1B
:1004C00040F2C60100F8011B40F2C30100F8011B15
:1004D00040F2C00100F8011B40F2BE0100F8011B10
:1004E00040F2BB0100F8011B40F2B80100F8011B0B
:1004F00040F2B50100F8011B40F2B30100F8011B06
:1005000040F2B00100F8011B40F2AD0100F8011B00
:1005100040F2AA0100F8011B40F2A70100F8011BFC
:1005200040F2A40100F8011B40F2A10100F8011BF8
:1005300040F29E0100F8011B40F29B0100F8011BF4
:1005400040F2970100F8011B40F2940100F8011BF2
:1005500040F2910100F8011B40F28E0100F8011BEE
:1005600040F28B0100F8011B40F2880100F8011BEA
:1005700040F2850100F8011B40F2820100F8011BE6
:1005800049F28070C1F2000040F200014FEAC1015F
:1005900020F8021B40F21C014FEAC10141F00601A4
:1005A00020F8021B40F238014FEAC10120F8021B7B
:1005B00040F251014FEAC10141F0040120F8021B51
:1005C00040F269014FEAC10141F0060120F8021B27
:1005D00040F280014FEAC10141F0040120F8021B02
:1005E00040F296014FEAC10120F8021B40F2AA0135
:1005F0004FEAC10141F0020120F8021B40F2BD01A7
:100600004FEAC10141F0040120F8021B40F2CF0182
:100610004FEAC10141F0040120F8021B40F2E00161
:100620004FEAC10141F0040120F8021B40F2F00141
:100630004FEAC10141F0060120F8021B40F200110F
:100640004FEAC10120F8021B49F60000C1F2000088
:1006500040F2000240F201034FEA422242EA030262
:100660004FEAC22240F8042B40F2000240F2640339
:100670004FEA422242EA03024FEAC22240F8042B28
:1006800040F2000240F2C8034FEA422242EA03026B
:100690004FEAC22240F8042B40F2000240F22C1331
:1006A0004FEA422242EA03024FEAC22240F8042BF8
:1006B00040F2000240F25E134FEA422242EA030295
:1006C0004FEAC22240F8042B40F2000240F290139D
:1006D0004FEA422242EA03024FEAC22240F8042BC8
:1006E00040F2000240F2C2134FEA422242EA030201
:1006F0004FEAC22240F8042B40F2010240F200030C
:100700004FEA422242EA03024FEAC22240F8042B97
:1007100040F2010240F232034FEA422242EA03026F
:100720004FEAC22240F8042B40F2010240F2640377
:100730004FEA422242EA03024FEAC22240F8042B67
:1007400040F2010240F296034FEA422242EA0302DB
:100750004FEAC22240F8042B40F2010240F2C803E3
:100760004FEA422242EA03024FEAC22240F8042B37
:1007700040F2010240F20D134FEA422242EA030224
:100780004FEAC22240F8042B40F2010240F23B1330
:100790004FEA422242EA03024FEAC22240F8042B07
:1007A00040F2010240F26C134FEA422242EA030295
:1007B0004FEAC22240F8042B40F2010240F2A0139B
:1007C0004FEA422242EA03024FEAC22240F8042BD7
:1007D00040F2010240F2D8134FEA422242EA0302F9
:1007E0004FEAC22240F8042B40F2020240F2120308
:1007F0004FEA422242EA03024FEAC22240F8042BA7
:1008000040F2020240F250034FEA422242EA03025F
:100810004FEAC22240F8042B40F2020240F2920357
:100820004FEA422242EA03024FEAC22240F8042B76
:1008300040F2020240F2DA034FEA422242EA0302A5
:100840004FEAC22240F8042B40F2020240F2211388
:100850004FEA422242EA03024FEAC22240F8042B46
:1008600040F2020240F26F134FEA422242EA0302D0
:100870004FEAC22240F8042B40F2020240F2C113B8
:100880004FEA422242EA03024FEAC22240F8042B16
:1008900040F2030240F219034FEA422242EA030205
:1008A0004FEAC22240F8042B40F2030240F27603E2
:1008B0004FEA422242EA03024FEAC22240F8042BE6
:1008C00040F2030240F2D9034FEA422242EA030215
:1008D0004FEAC22240F8042B40F2030240F24113D7
:1008E0004FEA422242EA03024FEAC22240F8042BB6
:1008F00040F2030240F2AF134FEA422242EA0302FF
:100900004FEAC22240F8042B40F2040240F22403D2
:100910004FEA422242EA03024FEAC22240F8042B85
:1009200040F2040240F2A0034FEA422242EA0302EC
:100930004FEAC22240F8042B40F2040240F2241392
:100940004FEA422242EA03024FEAC22240F8042B55
:1009500040F2040240F2AE134FEA422242EA03029E
:100960004FEAC22240F8042B40F2050240F2410354
:100970004FEA422242EA03024FEAC22240F8042B25
:1009800040F2050240F2DE034FEA422242EA03024D
:100990004FEAC22240F8042B40F2050240F28213D3
:1009A0004FEA422242EA03024FEAC22240F8042BF5
:1009B00040F2060240F234034FEA422242EA0302C6
:1009C0004FEAC22240F8042B40F2060240F2F00344
:1009D0004FEA422242EA03024FEAC22240F8042BC5
:1009E00040F2060240F2B2134FEA422242EA030208
:1009F0004FEAC22240F8042B40F2070240F284037F
:100A00004FEA422242EA03024FEAC22240F8042B94
:100A100040F2070240F264134FEA422242EA030224
:100A20004FEAC22240F8042B40F2080240F2500381
:100A30004FEA422242EA03024FEAC22240F8042B64
:100A400040F2080240F246134FEA422242EA030211
:100A50004FEAC22240F8042B40F2090240F24C0354
:100A60004FEA422242EA03024FEAC22240F8042B34
:100A700040F2090240F25E134FEA422242EA0302C8
:100A80004FEAC22240F8042B40F20A0240F28C03E3
:100A90004FEA422242EA03024FEAC22240F8042B04
:100AA00040F20A0240F2C2134FEA422242EA030233
:100AB0004FEAC22240F8042B40F20B0240F212131C
:100AC0004FEA422242EA03024FEAC22240F8042BD4
:100AD00040F20C0240F268034FEA422242EA03026B
:100AE0004FEAC22240F8042B40F20C0240F2E0131D
:100AF0004FEA422242EA03024FEAC22240F8042BA4
:100B000040F20D0240F268134FEA422242EA030229
:100B10004FEAC22240F8042B40F20E0240F20E13BC
:100B20004FEA422242EA03024FEAC22240F8042B73
:100B300040F20F0240F2C8034FEA422242EA0302A7
:100B40004FEAC22240F8042B40F2100240F2A00308
:100B50004FEA422242EA03024FEAC22240F8042B43
:100B600040F2110240F28E034FEA422242EA0302AF
:100B70004FEAC22240F8042B40F2120240F29603E0
:100B80004FEA422242EA03024FEAC22240F8042B13
:100B900040F2130240F2CE034FEA422242EA03023D
:100BA0004FEAC22240F8042B40F2140240F2241310
:100BB0004FEA422242EA03024FEAC22240F8042BE3
:100BC00040F2150240F28C134FEA422242EA03023D
:100BD0004FEAC22240F8042B40F2170240F20A0307
:100BE0004FEA422242EA03024FEAC22240F8042BB3
:100BF00040F2180240F2E0034FEA422242EA0302C6
:100C00004FEAC22240F8042B40F2190240F2D813F6
:100C10004FEA422242EA03024FEAC22240F8042B82
:100C200040F21B0240F2E2034FEA422242EA030290
:100C30004FEAC22240F8042B40F21D0240F21E038C
:100C40004FEA422242EA03024FEAC22240F8042B52
:100C500040F21E0240F2A6134FEA422242EA030289
:100C60004FEAC22240F8042B40F2200240F24A131D
:100C70004FEA422242EA03024FEAC22240F8042B22
:100C800040F2220240F22C134FEA422242EA0302CF
:100C90004FEAC22240F8042B40F2240240F26813CB
:100CA0004FEA422242EA03024FEAC22240F8042BF2
:100CB00040F2270240F200034FEA422242EA0302D6
:100CC0004FEAC22240F8042B40F2290240F200030E
:100CD0004FEA422242EA03024FEAC22240F8042BC2
:100CE00040F22C0240F200034FEA422242EA0302A1
:100CF0004FEAC22240F8042B40F22E0240F28C034D
:100D00004FEA422242EA03024FEAC22240F8042B91
:100D100040F2310240F200034FEA422242EA03026B
:100D20004FEAC22240F8042B40F2340240F20003A2
:100D30004FEA422242EA03024FEAC22240F8042B61
:100D400040F2370240F200034FEA422242EA030235
:100D50004FEAC22240F8042B40F23A0240F200036C
:100D60004FEA422242EA03024FEAC22240F8042B31
:100D700040F23E0240F200034FEA422242EA0302FE
:100D80004FEAC22240F8042B40F2420240F2000334
:100D90004FEA422242EA03024FEAC22240F8042B01
:100DA00040F2460240F200034FEA422242EA0302C6
:100DB0004FEAC22240F8042B40F24A0240F20003FC
:100DC0004FEA422242EA03024FEAC22240F8042BD1
:100DD00040F24E0240F200034FEA422242EA03028E
:100DE0004FEAC22240F8042B40F2530240F20003C3
:100DF0004FEA422242EA03024FEAC22240F8042BA1
:100E000040F2580240F200034FEA422242EA030253
:100E10004FEAC22240F8042B40F25E0240F2000387
:100E20004FEA422242EA03024FEAC22240F8042B70
:100E300040F2620240F200034FEA422242EA030219
:100E40004FEAC22240F8042B40F2680240F200034D
:100E50004FEA422242EA03024FEAC22240F8042B40
:100E600040F2710240F200034FEA422242EA0302DA
:100E70004FEAC22240F8042B40F2760240F200030F
:100E80004FEA422242EA03024FEAC22240F8042B10
:100E900040F27E0240F200034FEA422242EA03029D
:100EA0004FEAC22240F8042B40F2870240F20003CE
:100EB0004FEA422242EA03024FEAC22240F8042BE0
:100EC00040F28C0240F200034FEA422242EA03025F
:100ED0004FEAC22240F8042B40F2960240F200038F
:100EE0004FEA422242EA03024FEAC22240F8042BB0
:100EF00040F2A00240F200034FEA422242EA03021B
:100F00004FEAC22240F8042B40F2A70240F200034D
:100F10004FEA422242EA03024FEAC22240F8042B7F
:100F200040F2B00240F200034FEA422242EA0302DA
:100F30004FEAC22240F8042B40F2C00240F2000304
:100F40004FEA422242EA03024FEAC22240F8042B4F
:100F500040F2C80240F200034FEA422242EA030292
:100F60004FEAC22240F8042B40F2D20240F20003C2
:100F70004FEA422242EA03024FEAC22240F8042B1F
:100F800040F2DC0240F200034FEA422242EA03024E
:100F90004FEAC22240F8042B40F2EA0240F200037A
:100FA0004FEA422242EA03024FEAC22240F8042BEF
:100FB00040F2FA0240F200034FEA422242EA030200
:100FC0004FEAC22240F8042B40F2041240F2000320
:100FD0004FEA422242EA03024FEAC22240F8042BBF
:100FE00040F2181240F200034FEA422242EA0302A2
:100FF0004FEAC22240F8042B40F22C1240F20003C8
:101000004FEA422242EA03024FEAC22240F8042B8E
:1010100040F24A1240F200034FEA422242EA03023F
:101020004FEAC22240F8042B40F2681240F200035B
:101030004FEA422242EA03024FEAC22240F8042B5E
:1010400040F2681240F200034FEA422242EA0302F1
:101050004FEAC22240F8042B40F2901240F2000303
:101060004FEA422242EA03024FEAC22240F8042B2E
:1010700040F2901240F200034FEA422242EA030299
:101080004FEAC22240F8042B40F2901240F20003D3
:101090004FEA422242EA03024FEAC22240F8042BFE
:1010A00040F2901240F200034FEA422242EA030269
:1010B0004FEAC22240F8042B40F2901240F20003A3
:1010C0004FEA422242EA03024FEAC22240F8042BCE
:1010D00040F2901240F200034FEA422242EA030239
:1010E0004FEAC22240F8042B40F2901240F2000373
:1010F0004FEA422242EA03024FEAC22240F8042B9E
:1011000040F2901240F200034FEA422242EA030208
:101110004FEAC22240F8042B40F2901240F2000342
:101120004FEA422242EA03024FEAC22240F8042B6D
:1011300040F2901240F200034FEA422242EA0302D8
:101140004FEAC22240F8042B40F2901240F2000312
:101150004FEA422242EA03024FEAC22240F8042B3D
:1011600040F2901240F200034FEA422242EA0302A8
:101170004FEAC22240F8042B40F2901240F20003E2
:101180004FEA422242EA03024FEAC22240F8042B0D
:1011900040F2901240F200034FEA422242EA030278
:1011A0004FEAC22240F8042B40F2901240F20003B2
:1011B0004FEA422242EA03024FEAC22240F8042BDD
:1011C00040F2901240F200034FEA422242EA030248
:1011D0004FEAC22240F8042B40F2901240F2000382
:1011E0004FEA422242EA03024FEAC22240F8042BAD
:1011F00040F2901240F200034FEA422242EA030218
:101200004FEAC22240F8042B40F2901240F2000351
:101210004FEA422242EA03024FEAC22240F8042B7C
:1012200040F2901240F200034FEA422242EA0302E7
:101230004FEAC22240F8042B40F2901240F2000321
:101240004FEA422242EA03024FEAC22240F8042B4C
:1012500046F20040C4F2020045F29061C0F2010182
:1012600081654FF00001C0F60001816040F2090184
:1012700042F24C01C4F2010149F20001C2F2000144
:1012800046F20040C4F20200816D41F0010142F2D9
:101290000000C4F2000040F20101C0F20001C16090
:1012A00040F20001C0F20001816242F26C01C162B1
:1012B00040F28501C0F2000140F20101C0F20001DC
:1012C00040F60040C4F2000040F20101C0F200010B
:1012D000C16040F28F01816243F2DD21C16240F2C0
:1012E0008501C0F20001016040F20101C0F200017D
:1012F000416140F20000C4F2000040F20001C0F27F
:101300000001C16040F20001C0F20001816240F2C0
:10131000DC6140F26E316FF00001C16240F2850184
:10132000C0F20001016040F20101C0F20001416120
:1013300040F60000C4F2000040F20101C0F20001DA
:10134000C16040F20101C0F20001816240F2DC6143
:1013500040F26E31C16240F28501C0F200010160CD
:1013600040F20101C0F20001416140F20040C4F2CC
:10137000000040F20101C0F20001C16040F2010131
:10138000C0F20001816240F26E31C16240F285011B
:10139000C0F20001016040F20101C0F200014161B0
:1013A00040F20000C4F2010040F20101C0F200016D
:1013B000C16040F20101C0F20001816240F26E3171
:1013C000C16240F28501C0F20001016040F20101FA
:1013D000C0F20001416144F20000C4F2010040F299
:1013E0000101C0F20001C16040F20101C0F2000140
:1013F000816240F26E31C16240F28501C0F20001AB
:10140000016040F20101C0F20001416144F200407C
:10141000C4F2010040F20101C0F20001C16040F2DB
:101420000101C0F20001816240F26E31C16240F2FE
:101430008501C0F20001016040F20101C0F200012B
:10144000416144F60000C4F2010040F20101C0F223
:101450000001C16040F20101C0F20001816240F26E
:101460006E31C16240F28501C0F20001016040F2BC
:101470000101C0F20001416141F20040C4F20000EC
:1014800040F20101C0F20001C16040F20001C0F26F
:101490000001816244F2A011C16240F28501C0F2F4
:1014A0000001016040F20101C0F2000141614EF211
:1014B0000010CEF20000016844F60002C6F200728D
:1014C00041EA0201016041684BF6E002C0F6D40235
:1014D00041EA020141604EF20810CEF200000168BC
:1014E00041F0A00141F4000101604FF006014FF00E
:1014F00046064EF66027013FFDD1013EF9D1013984
:10150000F5D141F20002C4F2020246F62021C5F2F2
:101510005551116040F20043C4F202034FF000073E
:10152000CFF60077976140F290074FEA072747F41C
:101530000007976140F20405C0F201059D6100BFFC
:1015400040F20105C0F204059D614FF00007CFF69F
:101550000077976140F20205C0F201059D6100BF6E
:1015600040F20105C0F202059D6146F62021C0F25D
:101570000001116040F2000BC0F6000B40F6000CB9
:10158000C3F818B000BF00BF00BF00BFB2F8109092
:10159000C3F818C04FEA192909F0FF094FF00050AD
:1015A00080F80490C3F818B000BF00BF00BF00BFB0
:1015B000B2F81090C3F818C04FEA192909F0FF09D2
:1015C0004FF0005080F80590C3F818B000BF00BF7E
:1015D00000BF00BFB2F81090C3F818C04FEA192935
:1015E00009F0FF094FF0005080F80690C3F818B0DA
:1015F00000BF00BF00BF00BFB2F81090C3F818C012
:101600004FEA192909F0FF094FF0005080F80790C0
:10161000C3F818B000BF00BF00BF00BFB2F8109001
:10162000C3F818C04FEA192909F0FF094FF000501C
:1016300080F8089040F28005956190F80490B9F127
:10164000010F6FD190F80590B9F1D30F6AD190F8DE
:101650000690B9F1D10F65D190F80790B9F1950FC7
:1016600060D190F80890B9F1580F5BD1817A41F0C0
:101670000101817249F6002BC1F2000B49F680216D
:10168000C1F200014FF6FF72CFF6FF724BF8042B48
:101690008B45FBD14FF0000149F60023C1F2000356
:1016A0004FF000064FF000504FF00102C2721F29A8
:1016B00034D091F074FC4FF00002C0F60002A26139
:1016C00000BF00BF00BF00BFB5F810A04FEA1A2A44
:1016D00040F60002A26140F28002AA610AF0FF0A0D
:1016E000BAF1FF0F04D001F1010143F8046B09E0E6
:1016F00016F4006202D146F40066D8E76FF4006287
:1017000006EA02066FF4006206EA020606F50036F3
:101710004FF480424FEA02423240C8D04FF00002FC
:10172000C272017341F20002C4F2020246F62021A5
:10173000C5F25551116040F20043C4F2020340F675
:101740000004C4F202044FF00007CFF6007797615F
:1017500040F290074FEA0727976140F20005C0F278
:101760002005A56140F20405C0F201059D6100BF9E
:1017700040F20105C0F204059D614FF00007CFF66D
:101780000077976140F20205C0F201059D6100BF3C
:1017900040F20105C0F202059D6146F62021C0F22B
:1017A0000001116040F2000BC0F6000B40F6000C87
:1017B000C3F818B000BF00BF00BF00BFB2F8109060
:1017C000C3F818C04FEA192909F0FF094FF000507B
:1017D00080F8AC93C3F818B000BF00BF00BF00BFD3
:1017E000B2F81090C3F818C04FEA192909F0FF09A0
:1017F0004FF0005080F8AD93C3F818B000BF00BFA1
:1018000000BF00BFB2F81090C3F818C04FEA192902
:1018100009F0FF094FF0005080F8AE93C3F818B0FC
:1018200000BF00BF00BF00BFB2F81090C3F818C0DF
:101830004FEA192909F0FF094FF0005080F8AF93E3
:10184000C3F818B000BF00BF00BF00BFB2F81090CF
:10185000C3F818C04FEA192909F0FF094FF00050EA
:1018600080F8B09340F22005A56190F8AC93B9F1EF
:10187000010F71D190F8AD93B9F1D30F6CD190F8FD
:10188000AE93B9F1D10F67D190F8AF93B9F1950F3D
:1018900062D190F8B093B9F1580F5DD1817A41F0DF
:1018A0000201817249F6802BC1F2000B49F600312A
:1018B000C1F200014FF6FF72CFF6FF724BF8042B16
:1018C0008B45FBD14FF0000149F68023C1F20003A4
:1018D0004FF000064FF000504FF00102C2721F2976
:1018E00035D091F042FC4FF00002C0F60002A26138
:1018F00000BF00BF00BF00BFB5F810A04FEA1A2A12
:1019000040F60002A26140F22002C9F818200AF055
:10191000FF0ABAF1FF0F04D001F1010143F8046B93
:1019200009E016F4006202D146F40066D7E76FF4CE
:10193000006206EA02066FF4006206EA020606F595
:1019400000364FF480424FEA02423240C7D04FF097
:101950000002C27280F8B1134FF0230892F052FFD8
:101960004FF0540892F04EFF4FF0410892F04AFFBA
:1019700090F8206D40F265018E4201D340F264067A
:10198000142E38BF14264FF0230892F03BFF4FF07F
:10199000590892F037FF4FF0480892F033FF93F068
:1019A00049F84FF02C0892F02DFF4FF0230892F0E9
:1019B00029FF4FF0460892F025FF4FF0500892F0B3
:1019C00021FF4FF0310892F01DFF4FF0390892F0DF
:1019D00019FF4FF02C0892F015FF4FF0320892F0EB
:1019E00011FF4FF0330892F00DFF4FF0300892F0E6
:1019F00009FF4FF02C0892F005FF4FF0320892F0EB
:101A000001FF4FF0330892F0FDFE4FF0300892F0E6
:101A1000F9FE4FF02C0892F0F5FE4FF0320892F0EC
:101A2000F1FE4FF0330892F0EDFE4FF0300892F0E7
:101A3000E9FE4FF02C0892F0E5FE4FF0230892F0FB
:101A4000E1FE4FF0460892F0DDFE4FF0500892F0B4
:101A5000D9FE4FF0320892F0D5FE4FF0300892F0E8
:101A6000D1FE4FF02C0892F0CDFE4FF05A0692F0C6
:101A7000E1FF4FF02C0892F0C5FE4FF0D00692F037
:101A8000D9FF4FF02C0892F0BDFE4FF0BE0692F049
:101A9000D1FF4FF02C0892F0B5FE4FF0230892F0E2
:101AA000B1FE4FF0460892F0ADFE4FF0500892F0B4
:101AB000A9FE4FF0320892F0A5FE4FF0310892F0E7
:101AC000A1FE4FF02C0892F09DFE4FF0FB0692F025
:101AD000B1FF4FF02C0892F095FE4FF0CE0692F039
:101AE000A9FF4FF02C0892F08DFE4FF0B10692F056
:101AF000A1FF4FF02C0892F085FE4FF0230892F0E2
:101B000081FE4FF0460892F07DFE4FF0500892F0B3
:101B100079FE4FF0320892F075FE4FF0320892F0E5
:101B200071FE4FF02C0892F06DFE4FF0FB0692F024
:101B300081FF4FF02C0892F065FE4FF0AE0692F058
:101B400079FF4FF02C0892F05DFE4FF0910692F075
:101B500071FF4FF02C0892F055FE4FF0230892F0E1
:101B600051FE4FF0460892F04DFE4FF0500892F0B3
:101B700049FE4FF0320892F045FE4FF0330892F0E4
:101B800041FE4FF02C0892F03DFE4FF0E90692F036
:101B900051FF4FF02C0892F035FE4FF0E60692F020
:101BA00049FF4FF02C0892F02DFE4FF08B0692F07B
:101BB00041FF4FF02C0892F025FE91F056FD8FF07A
:101BC0002FFA4FF000504EF60022C2F20002D0F879
:101BD00064144FEA114122F8021BD0F864154FEA51
:101BE000114122F8021BD0F864164FEA114122F885
:101BF000021BD0F864174FEA114122F8021BD0F8FB
:101C000064184FEA114122F8021BD0F864194FEA18
:101C1000114122F8021BD0F8641A4FEA114122F850
:101C2000021BD0F8641B4FEA114122F8021B4FF04F
:101C30000001A0F8F41241F20013C2F2000333F8DD
:101C400001C040F2FF130CEA030C4FF000034FEA0F
:101C500041234CEA030C22F802CB01F1020140F6C9
:101C60000013994228BF0021A0F8F41290F85410F4
:101C700047F22803C1F20003082928BF083301F006
:101C8000070C4FEA0C2C6344D3F800C04FEA1C5CED
:101C900040F6FF730CEA030C4FEA01334CEA030CE5
:101CA00022F802CB01F1010140F21003994228BF52
:101CB000002180F8541090F8551047F20003C1F24B
:101CC0000003082928BF0833102928BF083301F072
:101CD000070C4FEA0C2C6344D3F800C04FEA5C5C5D
:101CE00040F2FF730CEA030C4FEAC1234CEA030CE9
:101CF00022F802CB01F1010140F21803994228BFFA
:101D0000002180F85510B0F8561040F60053C2F28A
:101D1000000313F801C00CF0FF0C4FEA01234CEA5A
:101D2000030C22F802CB01F1010140F20023994299
:101D300028BF0021A0F856104FF0010180F868106C
:101D40004FF0230892F05EFD4FF0410892F05AFDEB
:101D50004FF0450892F056FD4FF0300892F052FDDA
:101D60004FF02C0892F04EFD4FF0300892F04AFDF3
:101D70004FF0000892F046FD4FF0230892F042FD2C
:101D80004FF0460892F03EFD4FF0450892F03AFDC4
:101D90004FF0300892F036FD4FF02C0892F032FDF3
:101DA0004FF0300892F02EFD4FF02C0892F02AFDF3
:101DB0004FF0300892F026FD4FF02C0892F022FDF3
:101DC0004FF0300892F01EFD4FF02C0892F01AFDF3
:101DD0004FF0300892F016FD4FF02C0892F012FDF3
:101DE0004FF0300892F00EFD4FF0000892F00AFD1F
:101DF0004FF0230892F006FD4FF0410892F002FDEB
:101E00004FF0540892F0FEFC4FF0000692F012FEE4
:101E10004FF02C0892F0F6FC4FF0000692F00AFE0C
:101E20004FF02C0892F0EEFC4FF0280692F002FEE4
:101E30004FF02C0892F0E6FC40F20F1692F0FAFDFB
:101E40004FF02C0892F0DEFC4FF00A0692F0F2FD03
:101E50004FF02C0892F0D6FC4FF0500692F0EAFDBD
:101E60004FF02C0892F0CEFC4FF0430892F0CAFCE1
:101E70004FF0200892F0C6FC4FF0000892F0C2FC30
:101E80004FF0230892F0BEFC4FF0410892F0BAFCEC
:101E90004FF0540892F0B6FC4FF0290692F0CAFDBC
:101EA0004FF02C0892F0AEFC4FF0000692F0C2FD0D
:101EB0004FF02C0892F0A6FC4FF0500692F0BAFDBD
:101EC0004FF02C0892F09EFC40F20F1692F0B2FDFB
:101ED0004FF02C0892F096FC4FF00B0692F0AAFD02
:101EE0004FF02C0892F08EFC4FF0510692F0A2FDBC
:101EF0004FF02C0892F086FC4FF0430892F082FCE1
:101F00004FF0200892F07EFC4FF0000892F07AFC2F
:101F10004FF0230892F076FC4FF0410892F072FCEB
:101F20004FF0540892F06EFC4FF0510692F082FD93
:101F30004FF02C0892F066FC4FF0000692F07AFD0C
:101F40004FF02C0892F05EFC4FF0780692F072FD94
:101F50004FF02C0892F056FC40F20F1692F06AFDFA
:101F60004FF02C0892F04EFC4FF00C0692F062FD00
:101F70004FF02C0892F046FC4FF0520692F05AFDBA
:101F80004FF02C0892F03EFC4FF0430892F03AFCE0
:101F90004FF0200892F036FC4FF0000892F032FC2F
:101FA0004FF0230892F02EFC4FF0410892F02AFCEB
:101FB0004FF0540892F026FC4FF0790692F03AFD6B
:101FC0004FF02C0892F01EFC4FF0000692F032FD0C
:101FD0004FF02C0892F016FC4FF0A00692F02AFD6C
:101FE0004FF02C0892F00EFC40F20F1692F022FDFA
:101FF0004FF02C0892F006FC4FF00D0692F01AFDFF
:102000004FF02C0892F0FEFB4FF0530692F012FDB9
:102010004FF02C0892F0F6FB4FF0430892F0F2FBE1
:102020004FF0200892F0EEFB4FF0000892F0EAFB30
:102030004FF0230892F0E6FB4FF0410892F0E2FBEC
:102040004FF0540892F0DEFB4FF0A10692F0F2FC44
:102050004FF02C0892F0D6FB4FF0000692F0EAFC0D
:102060004FF02C0892F0CEFB4FF0C80692F0E2FC45
:102070004FF02C0892F0C6FB40F20F1692F0DAFCFB
:102080004FF02C0892F0BEFB4FF00E0692F0D2FCFF
:102090004FF02C0892F0B6FB4FF0540692F0CAFCB9
:1020A0004FF02C0892F0AEFB4FF0430892F0AAFBE1
:1020B0004FF0200892F0A6FB4FF0000892F0A2FB30
:1020C0004FF0230892F09EFB4FF0410892F09AFBEC
:1020D0004FF0540892F096FB4FF0C90692F0AAFC1C
:1020E0004FF02C0892F08EFB4FF0000692F0A2FC0D
:1020F0004FF02C0892F086FB4FF0F00692F09AFC1D
:102100004FF02C0892F07EFB40F20F1692F092FCFA
:102110004FF02C0892F076FB4FF00F0692F08AFCFD
:102120004FF02C0892F06EFB4FF0550692F082FCB7
:102130004FF02C0892F066FB4FF0430892F062FBE0
:102140004FF0200892F05EFB4FF0000892F05AFB2F
:102150004FF0230892F056FB4FF0410892F052FBEB
:102160004FF0540892F04EFB4FF0F10692F062FCF3
:102170004FF02C0892F046FB4FF0000692F05AFC0C
:102180004FF02C0892F03EFB4FF48C7692F052FC0C
:102190004FF02C0892F036FB40F20F1692F04AFCFA
:1021A0004FF02C0892F02EFB4FF0100692F042FCFC
:1021B0004FF02C0892F026FB4FF0560692F03AFCB6
:1021C0004FF02C0892F01EFB4FF0430892F01AFBE0
:1021D0004FF0200892F016FB4FF0000892F012FB2F
:1021E0004FF0230892F00EFB4FF0410892F00AFBEB
:1021F0004FF0540892F006FB40F2191692F01AFCC8
:102200004FF02C0892F0FEFA4FF0000692F012FC0C
:102210004FF02C0892F0F6FA4FF4A07692F00AFCF8
:102220004FF02C0892F0EEFA40F20F1692F002FCFA
:102230004FF02C0892F0E6FA4FF0110692F0FAFBFC
:102240004FF02C0892F0DEFA4FF0570692F0F2FBB6
:102250004FF02C0892F0D6FA4FF0430892F0D2FAE1
:102260004FF0200892F0CEFA4FF0000892F0CAFA30
:102270004FF0230892F0C6FA4FF0410892F0C2FAEC
:102280004FF0540892F0BEFA40F2411692F0D2FBA1
:102290004FF02C0892F0B6FA4FF0000692F0CAFB0D
:1022A0004FF02C0892F0AEFA4FF4B47692F0C2FBE5
:1022B0004FF02C0892F0A6FA40F20F1692F0BAFBFB
:1022C0004FF02C0892F09EFA4FF0120692F0B2FBFB
:1022D0004FF02C0892F096FA4FF0580692F0AAFBB5
:1022E0004FF02C0892F08EFA4FF0430892F08AFAE1
:1022F0004FF0200892F086FA4FF0000892F082FA30
:102300004FF0230892F07EFA4FF0410892F07AFAEB
:102310004FF0540892F076FA40F2691692F08AFB78
:102320004FF02C0892F06EFA4FF0000692F082FB0C
:102330004FF02C0892F066FA4FF4C87692F07AFBD0
:102340004FF02C0892F05EFA40F20F1692F072FBFA
:102350004FF02C0892F056FA4FF0130692F06AFBF9
:102360004FF02C0892F04EFA4FF0590692F062FBB3
:102370004FF02C0892F046FA4FF0430892F042FAE0
:102380004FF0200892F03EFA4FF0000892F03AFA2F
:102390004FF0230892F036FA4FF0410892F032FAEB
:1023A0004FF0540892F02EFA40F2911692F042FB50
:1023B0004FF02C0892F026FA4FF0000692F03AFB0C
:1023C0004FF02C0892F01EFA4FF4DC7692F032FBBC
:1023D0004FF02C0892F016FA40F20F1692F02AFBFA
:1023E0004FF02C0892F00EFA4FF0140692F022FBF8
:1023F0004FF02C0892F006FA4FF05A0692F01AFBB2
:102400004FF02C0892F0FEF94FF0430892F0FAF9E1
:102410004FF0200892F0F6F94FF0000892F0F2F930
:102420004FF0230892F0EEF94FF0410892F0EAF9EC
:102430004FF0540892F0E6F940F2B91692F0FAFA29
:102440004FF02C0892F0DEF94FF0000692F0F2FA0D
:102450004FF02C0892F0D6F94FF4F07692F0EAFAA9
:102460004FF02C0892F0CEF940F20F1692F0E2FAFB
:102470004FF02C0892F0C6F94FF0150692F0DAFAF8
:102480004FF02C0892F0BEF94FF05B0692F0D2FAB2
:102490004FF02C0892F0B6F94FF0430892F0B2F9E1
:1024A0004FF0200892F0AEF94FF0000892F0AAF930
:1024B0000DF0A6BD000000000000000000000000BC
:1024C000000000000000000000000000000000000C
:1024D00000000000000000000000000000000000FC
:1024E00000000000000000000000000000000000EC
:1024F00000000000000000000000000000000000DC
:020000040802F0
:100000004FF00050B0F86E206FF0020102EA0102DA
:10001000A0F86E2083F029FB4FF00050B0F86E106E
:1000200021F00101A0F86E104FF0000180F8D1110D
:1000300090F8311111F002020CBF21F0010121F002
:10004000020180F831114FF00001A0F8B4102BF03C
:1000500058BC4FF00050B0F86E2012F00202CFD121
:10006000B0F86E2012F004011AD012F0020117D17C
:1000700022F00402A0F86E2041F20001C2F2000159
:1000800090F8C430A3F108034FEA0323034490F827
:10009000C4A0AAF1080A4FEA0A2A51448CF087FA50
:1000A0004FF0005046F20049C4F20209D9F82C1072
:1000B000A1F10101B0F86BA0514509F09C83AAF1B0
:1000C000010140F2FF7201EA0201A0F86B106FEA31
:1000D0000A0A0AEA020A49F6000BC2F2000B1BF8F0
:1000E0000A40B0F8A42245F20003C1F200039C5478
:1000F00002F1010202F0FF02A0F8A4224FF07F01FA
:100100009954B0F83A130C2910D1D0F850130029A3
:100110000CD04FF04E02A2EB010245F60003C1F2F3
:1001200000039C540139C0F85013B9E7B0F83A13F2
:100130000E2910D1D0F8501300290CD0D0F8C020CF
:10014000A2EB010243F20003C2F202039C54013904
:10015000C0F85013A4E7B0F83A13282910D1D0F80A
:10016000501300290CD04FF04E02A2EB010245F6CD
:100170000003C1F200039C540139C0F850138FE70B
:10018000B0F83A132A2910D1D0F8501300290CD016
:10019000D0F8C020A2EB010243F20003C2F2020336
:1001A0009C540139C0F850137AE7B0F83A132F295C
:1001B00012D1D0F8501300290ED04FF00802A2EB54
:1001C000010202F1240245F60003C1F200039C542F
:1001D0000139C0F8501363E7B0F83A13312912D14E
:1001E000D0F8501300290ED04FF00802A2EB010204
:1001F00002F1240245F60003C1F200039C540139C8
:10020000C0F850134CE7B0F83A13392923D1D0F88D
:10021000501300291FD04FF40062A2EB0102D0F866
:100220005C63A6F500663244B2F5805F08D241F205
:100230000003C2F200039C540139C0F850132FE7A9
:10024000A2F5805240F20003C2F201039C5401392E
:10025000C0F8501324E7B0F83A133C2923D1D0F862
:10026000501300291FD04FF40062A2EB0102D0F816
:100270005C63A6F500663244B2F5805F08D241F2B5
:100280000003C2F200039C540139C0F8501307E781
:10029000A2F5805240F20003C2F201039C540139DE
:1002A000C0F85013FCE6B0F83A134B2910D1D0F83F
:1002B000501300290CD0D0F8C020A2EB010247F265
:1002C0000003C2F200039C540139C0F85013E7E662
:1002D000B0F83A134D2910D1D0F8501300290CD0A2
:1002E000D0F8C020A2EB010247F60003C2F20003DF
:1002F0009C540139C0F85013D2E60D2C49F06A82A3
:10030000B0F83C23002A3FF4CBAEB0F83A130029F2
:1003100030D145F20023C1F200034FF00005595DD2
:1003200056291CD105F10105AA4218D3595D65294A
:1003300015D105F10105AA4211D3595D72290ED1DB
:100340004FF00002A0F83C234FF00101A0F83A134F
:10035000D0F8401341F00101C0F840135CE64FF0C3
:100360000002A0F83C23D0F8401321F00101C0F8AE
:10037000401351E6012940F0B68045F20023C1F256
:1003800000034FF00005595D442940F0A78005F1B6
:100390000105AA42C0F0A280595D652940F09E8007
:1003A00005F10105AA42C0F09980595D762940F017
:1003B000958005F10105AA42C0F09080595D692938
:1003C00040F08C8005F10105AA42C0F08780595D9C
:1003D000632940F0838005F10105AA427ED3595D6F
:1003E00065297BD105F10105AA4277D3595D202902
:1003F00074D105F10105AA4270D3595D44296DD12C
:1004000005F10105AA4269D3595D652966D105F157
:100410000105AA4262D3595D74295FD105F1010536
:10042000AA425BD3595D652958D105F10105AA425D
:1004300054D3595D632951D105F10105AA424DD329
:10044000595D74294AD105F10105AA4246D3595D87
:10045000652943D105F10105AA423FD3595D6429BD
:100460003CD14FF00002A0F83C23D0F8401341F0FB
:100470000201C0F8401390F8551311F0010104D1A6
:100480004FF01001A0F83A130AE64FF00201A0F86D
:100490003A1390F8391341F0010180F839134FF005
:1004A000440886F0C1FA4FF0490886F0BDFA4FF0D3
:1004B000520886F0B9FA4FF00D0886F0B5FA4FF001
:1004C0000001C0F84413D0F848134FF00C02B1FB00
:1004D000F2F101FB02F1C0F84C13E1E54FF000022C
:1004E000A0F83C23DCE5022940F0488145F20023D6
:1004F000C1F20003151F57D3595D442920D105F1DE
:100500000105595D3A291BD105F10105595D5C29A9
:1005100016D105F10105595D3E2911D141F2004680
:10052000C4F20106376817F00F0808D037687768FB
:1005300090F86D7007F1010780F86D70A5E789E00C
:10054000151F31D3595D2E295BD105F10105595D88
:1005500057293CD105F10105595D412924D105F107
:100560000105595D56291FD1D0F8441301F101014D
:10057000C0F84413D0F84C13002908D0A1F10101B0
:10058000C0F84C134FF00002A0F83C2388E545F278
:100590000046C1F2000606F1C0073178FF2908D0F5
:1005A00006F11006BE42F8D14FF00002A0F83C233D
:1005B00076E54FF00005595D06F8011B05F10105D0
:1005C0009542F8D14FF00002A0F83C2368E5462997
:1005D0000AD105F10105595D5A29E5D105F1010559
:1005E000595D5029E0D1BFE74829DDD105F101056A
:1005F000595D4529D8D105F10105595D5829D3D157
:10060000B2E72029D0D105F10105595D44290FD168
:1006100005F10105595D4929C6D105F10105595D6D
:100620005229C1D1A5F103054FF02E0159559BE781
:100630006429B9D105F10105595D6929B4D105F1E4
:100640000105595D7229AFD1A5F103054FF02E01C7
:10065000595589E790F8391321F0010180F83913D1
:1006600045F20042C1F200021178FF299CD04FF000
:100670000301A0F83A134FF00001A0F83E1345F231
:100680000042C1F2000202F1C004B0F83E334FEA6A
:1006900003131A44A24200F052821178FF2900F09D
:1006A0004E824FF0010912F809102E2902D009F1EB
:1006B0000109F8E709F1010912F8091057290CD1CD
:1006C00009F1010912F80910412950D109F1010974
:1006D00012F8091056294AD11CE046290CD109F11B
:1006E000010912F809105A2941D109F1010912F83A
:1006F000091050293BD10DE0482938D109F10109F1
:1007000012F80910452932D109F1010912F809102E
:1007100058292CD109F1060980F85F904FF0440860
:1007200086F082F94FF0490886F07EF94FF05208C2
:1007300086F07AF94FF0200886F076F912F8018BEE
:10074000B8F1FF0F04D086F06FF912F00F01F5D168
:100750004FF00D0886F068F9B0F83E1301F1010181
:10076000A0F83E134FF00002A0F83C2398E4B0F844
:100770003E1301F10101A0F83E1380E7032940F088
:10078000068241F20046C4F20106376817F00F08EE
:100790000ED03768776890F86D7007F1010780F820
:1007A0006D70D0F83E63A6F10106C0F83E63D7E055
:1007B00045F20023C1F20003B2F10905C9F00A8035
:1007C000595D2E2949F0068005F10105595D57292B
:1007D00040F0BF8105F10105595D412940F0458197
:1007E00005F10105595D562940F03F8145F200466B
:1007F000C1F2000606F1C00790F85F90A2EB090570
:100800003178FF2900F0318113F80580884540F0E8
:10081000278105F101057178FF2900F0928013F816
:100820000580884540F01C8105F10105B178FF295C
:1008300000F0878013F80580884540F0118105F1AC
:100840000105F178FF297CD013F80580884540F038
:10085000078105F101053179FF2972D013F8058070
:10086000884540F0FD8005F101057179FF2968D0C8
:1008700013F80580884540F0F38005F10105B17952
:10088000FF295ED013F80580884540F0E98005F126
:100890000105F179FF2954D013F80580884540F00F
:1008A000DF8005F10105317AFF294AD013F8058070
:1008B000884540F0D58005F10105717AFF2940D0C7
:1008C00013F80580884540F0CB8005F10105B17A29
:1008D000FF2936D013F80580884540F0C18005F126
:1008E0000105F17AFF292CD013F80580884540F0E6
:1008F000B78005F10105317BFF2922D013F805806F
:10090000884540F0AD8005F10105717BFF2918D0C5
:1009100013F80580884540F0A38005F10105B17BFF
:10092000FF290ED013F80580884540F0998005F125
:100930000105F17BFF2904D013F80580884540F0BC
:100940008F8006F50076A2F104054FF0A90106F8A4
:10095000041B595D06F8011B05F101059542F8D10C
:1009600045F20042C1F2000202F1C004B0F83E3389
:100970004FEA03131A44A24200F0E1801178FF29E4
:1009800000F0DD804FF0010912F809102E2902D085
:1009900009F10109F8E709F1010912F809105729CD
:1009A0000CD109F1010912F80910412951D109F1BD
:1009B000010912F8091056294BD11CE046290CD127
:1009C00009F1010912F809105A2942D109F1010966
:1009D00012F8091050293CD10DE0482939D109F10C
:1009E000010912F80910452933D109F1010912F85A
:1009F000091058292DD109F1060980F85F904FF0B0
:100A0000440886F011F84FF0490886F00DF84FF0D1
:100A1000520886F009F84FF0200886F005F812F821
:100A2000018BB8F1FF0F04D085F0FEFF12F00F012B
:100A3000F5D14FF00D0885F0F7FFB0F83E1301F146
:100A40000101A0F83E134FF00002A0F83C23FFF78D
:100A500027BBB0F83E1301F10101A0F83E137FE778
:100A600006F11006BE427FF4C7AE45F20025C1F282
:100A7000000515F8011B432933D115F8011B6F2917
:100A80002FD115F8011B6D292BD115F8011B6D29EC
:100A900027D115F8011B612923D115F8011B6E29F7
:100AA0001FD115F8011B64291BD115F8011B202942
:100AB00017D115F8011B462913D115F8011B61291F
:100AC0000FD115F8011B69290BD115F8011B6C29F1
:100AD00007D115F8011B652903D115F8011B6429FD
:100AE000B7D045F20025C1F2000515F8011B4629D3
:100AF0001FD115F8011B69291BD115F8011B6C29A1
:100B000017D115F8011B652913D115F8011B2029F0
:100B10000FD115F8011B4F290BD115F8011B7029B6
:100B200007D115F8011B652903D115F8011B6E29A2
:100B30008FD04FF00002A0F83C23FFF7B1BA4FF07E
:100B40000401A0F83A134FF00002A0F83C23FFF78D
:100B500063BA46290BD105F10105595D5A2984D1A3
:100B600005F10105595D50297FF47FAF3EE6482924
:100B70007FF47BAF05F10105595D45297FF475AF21
:100B800005F10105595D58297FF46FAF2EE6042960
:100B900060D145F20023C1F200034FF00005595D1A
:100BA0004E2951D105F10105AA424DD3595D6F2956
:100BB0004AD105F10105AA4246D3595D202943D106
:100BC00005F10105AA423FD3595D44293CD105F105
:100BD0000105AA4238D3595D692935D105F10105CE
:100BE000AA4231D3595D73292ED105F10105AA42DC
:100BF0002AD3595D6B2927D14FF00002A0F83C237E
:100C00004FF00101A0F83A13D0F8401321F002018F
:100C1000C0F840136FF0000645F20041C1F2000138
:100C200001F5007241F8046B9142FBD16FF00006B0
:100C300045F20061C1F2000101F5007241F8046B58
:100C40009142FBD1FFF7E8B94FF00002A0F83C2336
:100C5000FFF726BA0B294FD145F20023C1F200035A
:100C6000151F47D3595D442944D105F10105595D4C
:100C70003A293FD105F10105595D5C293AD105F1C9
:100C80000105595D3E2935D14FF0520885F0CCFE63
:100C90004FF0440885F0C8FE4FF0460885F0C4FECA
:100CA0004FF0200885F0C0FE4FF04E02C0F85023F0
:100CB0004FEA126885F0B8FE4FEA124808F0FF08C4
:100CC00085F0B2FE4FEA122808F0FF0885F0ACFE6E
:100CD00002F0FF0885F0A8FE4FF00D0885F0A4FE95
:100CE0004FF00C01A0F83A134FF00002A0F83C239B
:100CF000FFF7D6B902F02EBE0C2940F0D58641F29E
:100D00000046C4F20106376817F00F0835D037687F
:100D1000776890F86D7007F1010780F86D704FF0FB
:100D2000530885F081FE4FF0450885F07DFE4FF0B9
:100D30004B0885F079FE4FF0200885F075FE4FF0E6
:100D4000000885F071FE4FF0000885F06DFE4FF051
:100D5000000885F069FE4FF0000885F065FE4FF051
:100D60000D0885F061FE4FF00B01A0F83A134FF02B
:100D70000002A0F83C23FFF793B945F20023C1F22B
:100D80000003151FC0F0E681595D442940F0E2815F
:100D900005F10105595D3A2940F0DC8105F10105B5
:100DA000595D5C2940F0D68105F10105595D3E2968
:100DB00040F0D08145F6000AC1F2000A1AF8011B82
:100DC000522940F0C9811AF8011B492940F0C48119
:100DD0001AF8011B462940F0BF811AF8051B462965
:100DE00040F0BA811AF8011B572940F0B5811AF872
:100DF000011B412940F0B0811AF8011B562940F02F
:100E0000AB811AF8011B452940F0A6811AF8011B95
:100E1000662940F0F6821AF8011B6D2940F0F18234
:100E20001AF8011B742940F0EC821AF8011B2029E2
:100E300040F0E7825AF8041B102940F0E2823AF8A9
:100E4000021B012940F0DD824FF000023AF80C1B32
:100E5000022908BF012280F886233AF8021B1029D4
:100E600040F0CF824FF0000180F8D01180F8C61F0B
:100E70004FF02401C0F86C1345F6000AC1F2000AD5
:100E80000AF1240A9AF80010472940F09B809AF84A
:100E900001104D2940F096809AF80210412940F047
:100EA00091809AF803104E2940F08C804FF0010198
:100EB00080F8D0119AF8081080F8B0129AF809104A
:100EC00080F8B1129AF80A1080F8B2129AF80B1052
:100ED00080F8B3129AF80C1080F8B4129AF80D103A
:100EE00080F8B5129AF80E1080F8B6129AF80F1022
:100EF00080F8B7129AF8101080F8B8129AF811100A
:100F000080F8B9129AF8121080F8BA129AF81310F1
:100F100080F8BB129AF8141080F8BC129AF81510D9
:100F200080F8BD129AF8161080F8BE129AF81710C1
:100F300080F8BF124FF03C01C0F86C1345F6000A70
:100F4000C1F2000ADAF83C10CAF82410DAF84010AE
:100F5000CAF8281045F6000AC1F2000A0AF13C0A54
:100F60009AF8001047292DD19AF80110542929D157
:100F70009AF80210452925D19AF803104D2921D15C
:100F80004FF0010180F8C61F9AF808909AF80910EE
:100F900009F0FF0901F0FF014FEA012149EA0109C7
:100FA000A0F8C49F4FF04601C0F86C1345F6000A44
:100FB000C1F2000ADAF84610CAF82410DAF84A102A
:100FC000CAF8281045F6000AC1F2000A0AF1240AFC
:100FD0009AF8001064290BD19AF80110612907D101
:100FE0009AF80210742903D19AF8031061293AD0B3
:100FF000DAF8041001F10801D0F86C938944C0F8C4
:101000006C934FF0530885F00FFD4FF0450885F0C5
:101010000BFD4FF04B0885F007FD4FF0200885F0E1
:1010200003FD4FEA196885F0FFFC4FEA194808F004
:10103000FF0885F0F9FC4FEA192808F0FF0885F051
:10104000F3FC09F0FF0885F0EFFC4FF00D0885F088
:10105000EBFC4FF02E01A0F83A134FF00002A0F87D
:101060003C23FFF71DB890F8FF12002940F0FA82E8
:1010700090F8B21311F001010ED1426E4FF480418D
:101080004FEA01418A4280F00284B0F86060B6F510
:10109000006F80F0FC830EE0D0F8B4234FF4804161
:1010A0004FEA01418A4280F0F283B0F8B863B6F5A6
:1010B000805F80F0EC83C0F8EC2245F60005C1F2B9
:1010C0000005AB6A13444FF480414FEA01418B4263
:1010D00028BF0B46C0F858334FF0530885F0A4FCE6
:1010E0004FF0450885F0A0FC4FF04B0885F09CFCC4
:1010F0004FF0200885F098FCD0F86C6306F10806E4
:101100004FEA166885F090FC4FEA164808F0FF0891
:1011100085F08AFC4FEA162808F0FF0885F084FC69
:1011200006F0FF0885F080FC4FF00D0885F07CFC90
:101130004FF00D01A0F83A134FF00002A0F83C2345
:101140004FF40061C0F868134FF0000180F8BD1043
:10115000FEF762BF02F0FEBB4FF0230883F052FBA4
:101160004FF0460883F04EFB4FF05A0883F04AFBDD
:101170004FF0330883F046FB4FF02C0883F042FB1E
:101180004FF0320883F03EFB4FF0330883F03AFB18
:101190004FF02C0883F036FB4FF0230883F032FB2E
:1011A0004FF05A0883F02EFB4FF0460883F02AFBDD
:1011B0004FF0310883F026FB4FF0300883F022FB1C
:1011C0004FF02C0883F01EFB4FF0230883F01AFB2E
:1011D0004FF05A0883F016FB4FF04C0883F012FBD7
:1011E0004FF0310883F00EFB4FF0320883F00AFB1A
:1011F0004FF0300883F006FB4FF02C0883F002FB21
:101200004FF0310883F0FEFA4FF0300883F0FAFA1D
:101210004FF0300883F0F6FA4FF02C0883F0F2FA22
:101220004FF0490883F0EEFA4FF06E0883F0EAFAC7
:101230004FF0630883F0E6FA4FF06F0883F0E2FAAC
:101240004FF0720883F0DEFA4FF0720883F0DAFA9A
:101250004FF0650883F0D6FA4FF0630883F0D2FAB6
:101260004FF0740883F0CEFA4FF0000883F0CAFA0A
:101270004FF0230883F0C6FA4FF05A0883F0C2FA01
:101280004FF04C0883F0BEFA4FF0310883F0BAFA01
:101290004FF0320883F0B6FA4FF0300883F0B2FA1C
:1012A0004FF02C0883F0AEFA4FF0310883F0AAFA21
:1012B0004FF0330883F0A6FA4FF0300883F0A2FA1B
:1012C0004FF02C0883F09EFA4FF0460883F09AFA0C
:1012D0004FF0690883F096FA4FF06C0883F092FAA9
:1012E0004FF0650883F08EFA4FF0000883F08AFA19
:1012F0004FF0230883F086FA4FF05A0883F082FA01
:101300004FF04C0883F07EFA4FF0310883F07AFA00
:101310004FF0320883F076FA4FF0300883F072FA1B
:101320004FF02C0883F06EFA4FF0310883F06AFA20
:101330004FF0360883F066FA4FF0300883F062FA17
:101340004FF02C0883F05EFA4FF0460883F05AFA0B
:101350004FF06F0883F056FA4FF0720883F052FA9C
:101360004FF06D0883F04EFA4FF0610883F04AFAAF
:101370004FF0740883F046FA4FF0210883F042FAE8
:101380004FF0000883F03EFAD0F848134FF00C02FB
:10139000B1FBF2F303FB02F3A1EB030145F20049B9
:1013A000C1F200094FEA011189444FF0430885F06A
:1013B0003BFB4FF04C0885F037FB4FF0460885F0BB
:1013C00033FB4FF0200885F02FFB19F8018BB8F1A3
:1013D000FF0F04D085F028FB19F00F01F5D14FF075
:1013E0000D0885F021FB4FF00F01A0F83A134FF0E4
:1013F0000002A0F83C234FF00101C0F86813FEF78B
:1014000028BE4FF0230883F0FDF94FF0460883F023
:10141000F9F94FF05A0883F0F5F94FF0330883F0EB
:10142000F1F94FF02C0883F0EDF94FF0320883F01A
:10143000E9F94FF0330883F0E5F94FF02C0883F019
:10144000E1F94FF0230883F0DDF94FF05A0883F0FB
:10145000D9F94FF0460883F0D5F94FF0310883F001
:10146000D1F94FF0300883F0CDF94FF02C0883F01C
:10147000C9F94FF0230883F0C5F94FF05A0883F0FB
:10148000C1F94FF04C0883F0BDF94FF0310883F0FB
:10149000B9F94FF0320883F0B5F94FF0300883F016
:1014A000B1F94FF02C0883F0ADF94FF0310883F01B
:1014B000A9F94FF0300883F0A5F94FF0300883F018
:1014C000A1F94FF02C0883F09DF94FF04E0883F0FE
:1014D00099F94FF06F0883F095F94FF0740883F095
:1014E00091F94FF0000883F08DF94FF0230883F055
:1014F00089F94FF05A0883F085F94FF04C0883F0D2
:1015000081F94FF0310883F07DF94FF0320883F014
:1015100079F94FF0300883F075F94FF02C0883F01B
:1015200071F94FF0310883F06DF94FF0330883F013
:1015300069F94FF0300883F065F94FF02C0883F01B
:1015400061F94FF0550883F05DF94FF06E0883F0B4
:1015500059F94FF0630883F055F94FF06F0883F0A5
:1015600051F94FF06D0883F04DF94FF0700883F09A
:1015700049F94FF0720883F045F94FF0650883F0A0
:1015800041F94FF0730883F03DF94FF0730883F091
:1015900039F94FF0650883F035F94FF0640883F0AE
:1015A00031F94FF0000883F02DF94FF0230883F054
:1015B00029F94FF05A0883F025F94FF04C0883F0D1
:1015C00021F94FF0310883F01DF94FF0320883F014
:1015D00019F94FF0300883F015F94FF02C0883F01B
:1015E00011F94FF0310883F00DF94FF0360883F010
:1015F00009F94FF0300883F005F94FF02C0883F01B
:1016000001F94FF0310883F0FDF84FF0360883F010
:10161000F9F84FF0200883F0F5F84FF0620883F0F6
:10162000F1F84FF0690883F0EDF84FF0740883F09B
:10163000E9F84FF0200883F0E5F84FF0500883F008
:10164000E1F84FF0430883F0DDF84FF04D0883F0E8
:10165000D9F84FF0210883F0D5F84FF0000883F057
:10166000D1F891E64FF0230883F0CCF84FF046080C
:1016700083F0C8F84FF05A0883F0C4F84FF03308ED
:1016800083F0C0F84FF02C0883F0BCF84FF032081C
:1016900083F0B8F84FF0330883F0B4F84FF02C081B
:1016A00083F0B0F84FF0230883F0ACF84FF05A08FD
:1016B00083F0A8F84FF0460883F0A4F84FF0310803
:1016C00083F0A0F84FF0300883F09CF84FF02C081E
:1016D00083F098F84FF0230883F094F84FF05A08FD
:1016E00083F090F84FF04C0883F08CF84FF03108FD
:1016F00083F088F84FF0320883F084F84FF0300818
:1017000083F080F84FF02C0883F07CF84FF031081C
:1017100083F078F84FF0300883F074F84FF0300819
:1017200083F070F84FF02C0883F06CF84FF05308FA
:1017300083F068F84FF0740883F064F84FF06F0896
:1017400083F060F84FF0700883F05CF84FF0000809
:1017500083F058F84FF0230883F054F84FF05A08FC
:1017600083F050F84FF04C0883F04CF84FF03108FC
:1017700083F048F84FF0320883F044F84FF0300817
:1017800083F040F84FF02C0883F03CF84FF031081C
:1017900083F038F84FF0330883F034F84FF0300816
:1017A00083F030F84FF02C0883F02CF84FF05208FB
:1017B00083F028F84FF0650883F024F84FF06308B1
:1017C00083F020F84FF06F0883F01CF84FF0720898
:1017D00083F018F84FF0640883F014F84FF06908AC
:1017E00083F010F84FF06E0883F00CF84FF06708A4
:1017F00083F008F84FF0000883F004F84FF0230856
:1018000083F000F84FF05A0882F0FCFF4FF04C08CC
:1018100082F0F8FF4FF0310882F0F4FF4FF0320809
:1018200082F0F0FF4FF0300882F0ECFF4FF02C0810
:1018300082F0E8FF4FF0310882F0E4FF4FF0360805
:1018400082F0E0FF4FF0300882F0DCFF4FF02C0810
:1018500082F0D8FF4FF0460882F0D4FF4FF06908BD
:1018600082F0D0FF4FF0720882F0CCFF4FF0730887
:1018700082F0C8FF4FF0740882F0C4FF4FF02108D7
:1018800082F0C0FF4FF0000882F0BCFF7CE54FF013
:10189000230882F0B7FF4FF0460882F0B3FF4FF005
:1018A0005A0882F0AFFF4FF0330882F0ABFF4FF0E1
:1018B0002C0882F0A7FF4FF0320882F0A3FF4FF010
:1018C000330882F09FFF4FF02C0882F09BFF4FF00F
:1018D000230882F097FF4FF05A0882F093FF4FF0F1
:1018E000460882F08FFF4FF0310882F08BFF4FF0F7
:1018F000330882F087FF4FF02C0882F083FF4FF00F
:10190000230882F07FFF4FF05A0882F07BFF4FF0F0
:101910004C0882F077FF4FF0310882F073FF4FF0F0
:10192000320882F06FFF4FF0300882F06BFF4FF00B
:101930002C0882F067FF4FF0310882F063FF4FF010
:10194000300882F05FFF4FF0300882F05BFF4FF00D
:101950002C0882F057FF4FF0530882F053FF4FF0EE
:10196000610882F04FFF4FF06D0882F04BFF4FF09F
:10197000700882F047FF4FF06C0882F043FF4FF091
:10198000650882F03FFF4FF0000882F03BFF4FF008
:10199000230882F037FF4FF05A0882F033FF4FF0F0
:1019A0004C0882F02FFF4FF0310882F02BFF4FF0F0
:1019B000320882F027FF4FF0300882F023FF4FF00B
:1019C0002C0882F01FFF4FF0310882F01BFF4FF010
:1019D000330882F017FF4FF0300882F013FF4FF00A
:1019E0002C0882F00FFF4FF0420882F00BFF4FF0FF
:1019F000610882F007FF4FF06E0882F003FF4FF09E
:101A00006B0882F0FFFE4FF0200882F0FBFE4FF0E3
:101A1000410882F0F7FE4FF0000882F0F3FE4FF02D
:101A2000230882F0EFFE4FF05A0882F0EBFE4FF0F1
:101A30004C0882F0E7FE4FF0310882F0E3FE4FF0F1
:101A4000320882F0DFFE4FF0300882F0DBFE4FF00C
:101A50002C0882F0D7FE4FF0310882F0D3FE4FF011
:101A6000360882F0CFFE4FF0300882F0CBFE4FF008
:101A70002C0882F0C7FE4FF0460882F0C3FE4FF0FC
:101A8000750882F0BFFE4FF06C0882F0BBFE4FF08D
:101A90006C0882F0B7FE4FF0210882F0B3FE4FF0E1
:101AA000000882F0AFFE6FE40D2964D145F20023F7
:101AB000C1F20003151F5CD3595D442959D105F1CA
:101AC0000105595D3A2954D105F10105595D5C299B
:101AD0004FD105F10105595D3E294AD1D0F8EC22DC
:101AE000D0F85833A3EB0203B3F5304F05D2002BE7
:101AF00002D0C0F8503304E013E14FF43043C0F893
:101B00005033C0F85C334FF0520884F08DFF4FF033
:101B1000440884F089FF4FF0460884F085FF4FF0B9
:101B2000200884F081FFD0F85023C0F8C0204FEA8D
:101B3000126884F079FF4FEA124808F0FF0884F039
:101B400073FF4FEA122808F0FF0884F06DFF02F0DF
:101B5000FF0884F069FF4FF00D0884F065FF4FF037
:101B60000E01A0F83A134FF00002A0F83C23FEF754
:101B700097BA01F0EFBE0E2941F0F28041F2004623
:101B8000C4F20106376817F00F080ED0376877687F
:101B900090F86D7007F1010780F86D7090F8B2232E
:101BA00012F0010240F0EB847FE090F8B22312F0D3
:101BB000010240F0648443F2000BC2F2020BD0F841
:101BC0005823446EA2EB04024FEA9212D0F8EC6262
:101BD000A6EB0406B6FBF2F280F8BD20D0F8EC626A
:101BE0004FF6FF72C0F2010212EA060401D181F041
:101BF000D1FE44F200024FEA0242964280F0918008
:101C000081F0E4FAD0F85C934FF40067B9F5006F07
:101C100038BF4F46C0F8F07FA9EB0709C0F85C93C6
:101C20000BEB07094FF00007C0F201074FF0010866
:101C30001BF801AB85F815A0A76100BF00BFC4F871
:101C40001880CB45F4D140F20407C0F2010740F2FE
:101C500010026A75A76140F20107C0F2040700BFD5
:101C600000BF00BF00BFA76100BF00BF228A12F4FF
:101C70008062FBD146F62022C0F200022A6000BF3B
:101C800000BF228A12F48062FBD04FF08007AF6160
:101C9000D0F8F04F2644C0F8EC62D0F85C43002C3A
:101CA0008DD1D0F85843A6423BD24FF0530884F070
:101CB000BBFE4FF0450884F0B7FE4FF04B0884F0B0
:101CC000B3FE4FF0200884F0AFFED0F8EC62456E12
:101CD000A6EB0506D0F86C5305F108052E444FEA33
:101CE000166884F0A1FE4FEA164808F0FF0884F059
:101CF0009BFE4FEA162808F0FF0884F095FE06F0D8
:101D0000FF0884F091FE4FF00D0884F08DFE4FF037
:101D10000D01A0F83A134FF00002A0F83C23FEF7A3
:101D2000BFB9466E4FF00101C17281F033FE06F17A
:101D3000010681F04BFA40F2A9024FF00007C0F211
:101D400001076A75A76100BF00BF00BF4FF0010720
:101D5000A761D0F8586306F500364FEA164202F044
:101D6000FE024FF00007C0F201076A75A76100BFCD
:101D700000BF00BF4FF00107A7614FEA166202F0F3
:101D80001F024FF00007C0F201076A75A76100BF8C
:101D900000BF00BF4FF00107A761D0F848134FF014
:101DA0000C02B1FBF2F303FB02F3A1EB030145F2DA
:101DB0000049C1F200094FEA011189444FF00001C6
:101DC00080F8571319F8012B90F8D01111F0010188
:101DD00018BF90F8B0224FF00007C0F201076A75F3
:101DE000A76100BF00BF00BF4FF00107A76119F84E
:101DF000012B2E2A03D14FF0010180F8571390F8E0
:101E00005713012908BF202290F8D01111F00101C9
:101E100018BF90F8B1224FF00007C0F201076A75B1
:101E2000A76100BF00BF00BF4FF00107A76119F80D
:101E3000012B2E2A03D14FF0010180F8571390F89F
:101E40005713012908BF202290F8D01111F0010189
:101E500018BF90F8B2224FF00007C0F201076A7570
:101E6000A76100BF00BF00BF4FF00107A76119F8CD
:101E7000012B2E2A03D14FF0010180F8571390F85F
:101E80005713012908BF202290F8D01111F0010149
:101E900018BF90F8B3224FF00007C0F201076A752F
:101EA000A76100BF00BF00BF4FF00107A76119F88D
:101EB000012B2E2A03D14FF0010180F8571390F81F
:101EC0005713012908BF202290F8D01111F0010109
:101ED00018BF90F8B4224FF00007C0F201076A75EE
:101EE000A76100BF00BF00BF4FF00107A76119F84D
:101EF000012B2E2A03D14FF0010180F8571390F8DF
:101F00005713012908BF202290F8D01111F00101C8
:101F100018BF90F8B5224FF00007C0F201076A75AC
:101F2000A76100BF00BF00BF4FF00107A76119F80C
:101F3000012B2E2A03D14FF0010180F8571390F89E
:101F40005713012908BF202290F8D01111F0010188
:101F500018BF90F8B6224FF00007C0F201076A756B
:101F6000A76100BF00BF00BF4FF00107A76119F8CC
:101F7000012B2E2A03D14FF0010180F8571390F85E
:101F80005713012908BF202290F8D01111F0010148
:101F900018BF90F8B7224FF00007C0F201076A752A
:101FA000A76100BF00BF00BF4FF00107A7614FF05E
:101FB000200290F8D01111F0010118BF90F8B8225A
:101FC0004FF00007C0F201076A75A76100BF00BFAC
:101FD00000BF4FF00107A7614FF0200290F8D01129
:101FE00011F0010118BF90F8B9224FF00007C0F2BC
:101FF00001076A75A76100BF00BF00BF4FF001076E
:10200000A7614FF0200290F8D01111F0010118BF24
:1020100090F8BA224FF00007C0F201076A75A76175
:1020200000BF00BF00BF4FF00107A7614FF02002C3
:1020300090F8D01111F0010118BF90F8BB224FF0B9
:102040000007C0F201076A75A76100BF00BF00BFAB
:102050004FF00107A7614FF0200290F8D01111F066
:10206000010118BF90F8BC224FF00007C0F2010731
:102070006A75A76100BF00BF00BF4FF00107A761ED
:102080004FF0200290F8D01111F0010118BF90F824
:10209000BD224FF00007C0F201076A75A76100BFBB
:1020A00000BF00BF4FF00107A7614FF0200290F87A
:1020B000D01111F0010118BF90F8BE224FF00007B7
:1020C000C0F201076A75A76100BF00BF00BF4FF0F3
:1020D0000107A7614FF0200290F8D01111F0010123
:1020E00018BF90F8BF224FF00007C0F201076A75D1
:1020F000A76100BF00BF00BF4FF00107A761D0F884
:1021000058130A464FF00007C0F201076A75A7612D
:1021100000BF00BF00BF4FF00107A7614FEA1122C7
:102120004FF00007C0F201076A75A76100BF00BF4A
:1021300000BF4FF00107A7614FEA11424FF00007BF
:10214000C0F201076A75A76100BF00BF00BF4FF072
:102150000107A7614FEA11624FF00007C0F20107C3
:102160006A75A76100BF00BF00BF4FF00107A761FC
:1021700090F8861311F0010114BFA922FF224FF03D
:102180000007C0F201076A75A76100BF00BF00BF6A
:102190004FF00107A76190F8C61F11F0010100F090
:1021A00040814FF0FF014FF00007C0F20107697551
:1021B000A76100BF00BF00BF4FF00107A76100BFCC
:1021C00000BF6FF000014FF00007C0F20107697512
:1021D000A76100BF00BF00BF4FF00107A76100BFAC
:1021E00000BF4FEA11224FF00007C0F201076A75E5
:1021F000A76100BF00BF00BF4FF00107A76100BF8C
:1022000000BF6FF000014FF00007C0F201076975D1
:10221000A76100BF00BF00BF4FF00107A76100BF6B
:1022200000BF4FEA11224FF00007C0F201076A75A4
:10223000A76100BF00BF00BF4FF00107A76100BF4B
:1022400000BF6FF000014FF00007C0F20107697591
:10225000A76100BF00BF00BF4FF00107A76100BF2B
:1022600000BF4FEA11224FF00007C0F201076A7564
:10227000A76100BF00BF00BF4FF00107A76100BF0B
:1022800000BF6FF000014FF00007C0F20107697551
:10229000A76100BF00BF00BF4FF00107A76100BFEB
:1022A00000BF4FEA11224FF00007C0F201076A7524
:1022B000A76100BF00BF00BF4FF00107A76100BFCB
:1022C00000BF6FF000014FF00007C0F20107697511
:1022D000A76100BF00BF00BF4FF00107A76100BFAB
:1022E00000BF4FEA11224FF00007C0F201076A75E4
:1022F000A76100BF00BF00BF4FF00107A76100BF8B
:1023000000BF4FEA11424FF00007C0F201076A75A3
:10231000A76100BF00BF00BF4FF00107A76100BF6A
:1023200000BF4FEA11624FF00007C0F201076A7563
:10233000A76100BF00BF00BF4FF00107A76100BF4A
:1023400000BF6FF000014FF00007C0F20107697590
:10235000A76100BF00BF00BF4FF00107A76100BF2A
:1023600000BF4FEA11224FF00007C0F201076A7563
:10237000A76100BF00BF00BF4FF00107A76100BF0A
:1023800000BF4FEA11424FF00007C0F201076A7523
:10239000A76100BF00BF00BF4FF00107A76100BFEA
:1023A00000BF4FEA11624FF00007C0F201076A75E3
:1023B000A76100BF00BF00BF4FF00107A76100BFCA
:1023C00000BF4FF0A9014FF00007C0F20107697587
:1023D000A76100BF00BF00BF4FF00107A76100BFAA
:1023E00000BFB0F8C42F4FF00007C0F201076A75B4
:1023F000A76100BF00BF00BF4FF00107A76100BF8A
:1024000000BF4FEA12214FF00007C0F201076975C3
:10241000A76100BF00BF00BF4FF00107A76100BF69
:1024200000BF40F20407C0F2010740F210026A75D3
:10243000A76140F20107C0F20407A76100BF00BF17
:10244000228A12F48062FBD146F62022C0F20002FA
:102450002A60228A12F48062FBD04FF00001C17220
:102460004FF08007AF61B0F86E1041F00201A0F8A4
:102470006E104FF00002A0F83C23FEF785BF43F238
:10248000000BC2F2020BD0F85823D0F8B443A2EBF1
:1024900004024FEA9212D0F8EC62A6EB0406B6FBF7
:1024A000F2F280F8BD20D0F8EC624FF6FF72C0F275
:1024B000010212EA060401D181F07FFA44F200021F
:1024C0004FEA0242964280F0978080F040FFD0F8B9
:1024D0005C934FF40067B9F5006F38BF4F46C0F802
:1024E000F07FA9EB0709C0F85C930BEB07094FF0ED
:1024F0000007C0F201074FF001081BF801AB85F897
:1025000015A0A76100BF00BFC4F81880CB45F4D167
:1025100040F20407C0F2010740F210026A75A76199
:1025200040F20107C0F2040700BF00BF00BF00BFB8
:10253000A76100BF00BF228A12F48062FBD146F679
:102540002022C0F200022A6000BF00BF228A12F4DB
:102550008062FBD040F60009C4F202094FF0200768
:10256000C9F81870D0F8F04F2644C0F8EC62D0F8E3
:102570005C43002C87D1D0F85843A6423CD24FF0A0
:10258000530884F051FA4FF0450884F04DFA4FF0AB
:102590004B0884F049FA4FF0200884F045FAD0F84F
:1025A000EC62D0F8B453A6EB0506D0F86C5305F1F5
:1025B00008052E444FEA166884F036FA4FEA1648AA
:1025C00008F0FF0884F030FA4FEA162808F0FF08F8
:1025D00084F02AFA06F0FF0884F026FA4FF00D087E
:1025E00084F022FA4FF00D01A0F83A134FF00002E8
:1025F000A0F83C23FDF754BDD0F8B4634FF00101BF
:10260000C17281F0DAF906F1010680F0A0FE40F215
:10261000A9024FF00007C0F201076A75A76100BF69
:1026200000BF00BF4FF00107A761D0F8586306F55F
:1026300000364FEA164202F0FE024FF00007C0F2E9
:1026400001076A75A76100BF00BF00BF4FF0010717
:10265000A7614FEA166202F01F024FF00007C0F2B6
:1026600001076A75A76100BF00BF00BF4FF00107F7
:10267000A761D0F848134FF00C02B1FBF2F303FB53
:1026800002F3A1EB030145F20049C1F200094FEA50
:10269000011189444FF0000180F8571319F8012BFC
:1026A00090F8D01111F0010118BF90F8B0224FF04E
:1026B0000007C0F201076A75A76100BF00BF00BF35
:1026C0004FF00107A76119F8012B2E2A03D14FF013
:1026D000010180F8571390F85713012908BF2022F1
:1026E00090F8D01111F0010118BF90F8B1224FF00D
:1026F0000007C0F201076A75A76100BF00BF00BFF5
:102700004FF00107A76119F8012B2E2A03D14FF0D2
:10271000010180F8571390F85713012908BF2022B0
:1027200090F8D01111F0010118BF90F8B2224FF0CB
:102730000007C0F201076A75A76100BF00BF00BFB4
:102740004FF00107A76119F8012B2E2A03D14FF092
:10275000010180F8571390F85713012908BF202270
:1027600090F8D01111F0010118BF90F8B3224FF08A
:102770000007C0F201076A75A76100BF00BF00BF74
:102780004FF00107A76119F8012B2E2A03D14FF052
:10279000010180F8571390F85713012908BF202230
:1027A00090F8D01111F0010118BF90F8B4224FF049
:1027B0000007C0F201076A75A76100BF00BF00BF34
:1027C0004FF00107A76119F8012B2E2A03D14FF012
:1027D000010180F8571390F85713012908BF2022F0
:1027E00090F8D01111F0010118BF90F8B5224FF008
:1027F0000007C0F201076A75A76100BF00BF00BFF4
:102800004FF00107A76119F8012B2E2A03D14FF0D1
:10281000010180F8571390F85713012908BF2022AF
:1028200090F8D01111F0010118BF90F8B6224FF0C6
:102830000007C0F201076A75A76100BF00BF00BFB3
:102840004FF00107A76119F8012B2E2A03D14FF091
:10285000010180F8571390F85713012908BF20226F
:1028600090F8D01111F0010118BF90F8B7224FF085
:102870000007C0F201076A75A76100BF00BF00BF73
:102880004FF00107A7614FF0200290F8D01111F02E
:10289000010118BF90F8B8224FF00007C0F20107FD
:1028A0006A75A76100BF00BF00BF4FF00107A761B5
:1028B0004FF0200290F8D01111F0010118BF90F8EC
:1028C000B9224FF00007C0F201076A75A76100BF87
:1028D00000BF00BF4FF00107A7614FF0200290F842
:1028E000D01111F0010118BF90F8BA224FF0000783
:1028F000C0F201076A75A76100BF00BF00BF4FF0BB
:102900000107A7614FF0200290F8D01111F00101EA
:1029100018BF90F8BB224FF00007C0F201076A759C
:10292000A76100BF00BF00BF4FF00107A7614FF0D4
:10293000200290F8D01111F0010118BF90F8BC22CC
:102940004FF00007C0F201076A75A76100BF00BF22
:1029500000BF4FF00107A7614FF0200290F8D0119F
:1029600011F0010118BF90F8BD224FF00007C0F22E
:1029700001076A75A76100BF00BF00BF4FF00107E4
:10298000A7614FF0200290F8D01111F0010118BF9B
:1029900090F8BE224FF00007C0F201076A75A761E8
:1029A00000BF00BF00BF4FF00107A7614FF020023A
:1029B00090F8D01111F0010118BF90F8BF224FF02C
:1029C0000007C0F201076A75A76100BF00BF00BF22
:1029D0004FF00107A761D0F858130A464FF00007DF
:1029E000C0F201076A75A76100BF00BF00BF4FF0CA
:1029F0000107A7614FEA11224FF00007C0F201075B
:102A00006A75A76100BF00BF00BF4FF00107A76153
:102A10004FEA11424FF00007C0F201076A75A76143
:102A200000BF00BF00BF4FF00107A7614FEA11626E
:102A30004FF00007C0F201076A75A76100BF00BF31
:102A400000BF4FF00107A76190F8861311F0010154
:102A500014BFA922FF224FF00007C0F201076A75D8
:102A6000A76100BF00BF00BF4FF00107A76190F84A
:102A7000C61F11F0010100F040814FF0FF014FF03F
:102A80000007C0F201076975A76100BF00BF00BF62
:102A90004FF00107A76100BF00BF6FF000014FF0CA
:102AA0000007C0F201076975A76100BF00BF00BF42
:102AB0004FF00107A76100BF00BF4FEA11224FF09E
:102AC0000007C0F201076A75A76100BF00BF00BF21
:102AD0004FF00107A76100BF00BF6FF000014FF08A
:102AE0000007C0F201076975A76100BF00BF00BF02
:102AF0004FF00107A76100BF00BF4FEA11224FF05E
:102B00000007C0F201076A75A76100BF00BF00BFE0
:102B10004FF00107A76100BF00BF6FF000014FF049
:102B20000007C0F201076975A76100BF00BF00BFC1
:102B30004FF00107A76100BF00BF4FEA11224FF01D
:102B40000007C0F201076A75A76100BF00BF00BFA0
:102B50004FF00107A76100BF00BF6FF000014FF009
:102B60000007C0F201076975A76100BF00BF00BF81
:102B70004FF00107A76100BF00BF4FEA11224FF0DD
:102B80000007C0F201076A75A76100BF00BF00BF60
:102B90004FF00107A76100BF00BF6FF000014FF0C9
:102BA0000007C0F201076975A76100BF00BF00BF41
:102BB0004FF00107A76100BF00BF4FEA11224FF09D
:102BC0000007C0F201076A75A76100BF00BF00BF20
:102BD0004FF00107A76100BF00BF4FEA11424FF05D
:102BE0000007C0F201076A75A76100BF00BF00BF00
:102BF0004FF00107A76100BF00BF4FEA11624FF01D
:102C00000007C0F201076A75A76100BF00BF00BFDF
:102C10004FF00107A76100BF00BF6FF000014FF048
:102C20000007C0F201076975A76100BF00BF00BFC0
:102C30004FF00107A76100BF00BF4FEA11224FF01C
:102C40000007C0F201076A75A76100BF00BF00BF9F
:102C50004FF00107A76100BF00BF4FEA11424FF0DC
:102C60000007C0F201076A75A76100BF00BF00BF7F
:102C70004FF00107A76100BF00BF4FEA11624FF09C
:102C80000007C0F201076A75A76100BF00BF00BF5F
:102C90004FF00107A76100BF00BF4FF0A9014FF03F
:102CA0000007C0F201076975A76100BF00BF00BF40
:102CB0004FF00107A76100BF00BFB0F8C42F4FF06D
:102CC0000007C0F201076A75A76100BF00BF00BF1F
:102CD0004FF00107A76100BF00BF4FEA12214FF07C
:102CE0000007C0F201076975A76100BF00BF00BF00
:102CF0004FF00107A76100BF00BF40F20407C0F218
:102D0000010740F210026A75A76140F20107C0F2A4
:102D10000407A76100BF00BF228A12F48062FBD1C2
:102D200046F62022C0F200022A60228A12F4806253
:102D3000FBD04FF00001C17240F60009C4F2020955
:102D40004FF02007C9F81870B0F86E1041F002017A
:102D5000A0F86E104FF00002A0F83C23FEF714BB61
:102D60000F2929D145F20023C1F20003151F21D3F9
:102D7000595D44291ED105F10105595D3A2919D142
:102D800005F10105595D5C2914D105F10105595D75
:102D90003E290FD190F8391321F0010180F8391341
:102DA0004FF00401A0F83A134FF00002A0F83C23C2
:102DB000FDF776B900F0CEBD102947D145F20023CA
:102DC000C1F20003151F3BD3595D442938D105F1E9
:102DD0000105595D3A2933D105F10105595D5C2999
:102DE0002ED105F10105595D3E2929D14FF0530837
:102DF00083F01AFE4FF0420883F016FE4FF04408AD
:102E000083F012FE4FF0200883F00EFE4FF0010811
:102E100083F00AFE4FF0000883F006FE4FF0000832
:102E200083F002FE4FF00D0883F0FEFD4FF011011C
:102E3000A0F83A134FF00002A0F83C23FDF7ECB8DD
:102E40004FF00002A0F83C23FDF72AB9112954D114
:102E500045F20023C1F20003151F48D3595D4429F0
:102E600045D105F10105595D3A2940D105F101052A
:102E7000595D5C293BD105F10105595D3E2936D1EB
:102E8000C18B0029FCD141F2004CC4F2010CDCF8EA
:102E90000C1040F20C02C0F2000221EA0201CCF850
:102EA0000C104FF01702CCF80820DCF8141040F298
:102EB0000032C0F2000241EA0201CCF81410DCF842
:102EC0000C1040F20C02C0F2000241EA0201CCF800
:102ED0000C104FF0010180F855134FF01201A0F8CB
:102EE0003A134FF00002A0F83C23FDF7D9B84FF099
:102EF0000002A0F83C23FDF7D3B8122947D145F2D0
:102F00000023C1F20003151F3BD3595D442938D17A
:102F100005F10105595D3A2933D105F10105595DE6
:102F20005C292ED105F10105595D3E2929D14FF0CB
:102F30000201A0F83A1390F8391341F0010180F82A
:102F400039134FF0440883F06FFD4FF0490883F0C8
:102F50006BFD4FF0520883F067FD4FF00D0883F0D2
:102F600063FD4FF00001C0F84413D0F848134FF050
:102F70000C02B1FBF2F101FB02F1C0F84C13FDF7BA
:102F80008FB84FF00002A0F83C23FDF789B8132951
:102F900040F01C8345F20023C1F20003151FC0F06E
:102FA0001483595D442940F0108305F10105595DF2
:102FB0003A2940F00A8305F10105595D5C2940F08A
:102FC000048305F10105595D3E2940F0FE824FF072
:102FD000570883F029FD4FF0520883F025FD4FF08C
:102FE000460883F021FD4FF0200883F01DFDD0F846
:102FF000D013D0F8D423A2EB0102C0F85C2302F175
:103000004E024FEA126883F00FFD4FEA124808F0B3
:10301000FF0883F009FD4FEA122808F0FF0883F04B
:1030200003FD904608F0FF0883F0FEFC4FF00D080A
:1030300083F0FAFC4FF0520883F0F6FC4FF0490899
:1030400083F0F2FC4FF0460883F0EEFC4FF04608A8
:1030500083F0EAFCD0F85C2302F14602904608F0C7
:10306000FF0883F0E1FC4FEA122808F0FF0883F024
:10307000DBFC4FEA124808F0FF0883F0D5FC4FEA6A
:10308000126883F0D1FC4FF0570883F0CDFC4FF06D
:10309000410883F0C9FC4FF0560883F0C5FC4FF09F
:1030A000450883F0C1FC4FF0660883F0BDFC4FF08B
:1030B0006D0883F0B9FC4FF0740883F0B5FC4FF055
:1030C000200883F0B1FC4FF01002904608F0FF0892
:1030D00083F0AAFC4FEA122808F0FF0883F0A4FC52
:1030E0004FEA124808F0FF0883F09EFC4FEA12688E
:1030F00083F09AFC4FF00102904608F0FF0883F03D
:1031000093FC4FEA122808F0FF0883F08DFC4FF083
:10311000010290F88833A92B08BF5200904608F0AE
:10312000FF0883F081FC4FEA122808F0FF0883F0C3
:103130007BFC4AF64442904608F0FF0883F074FC9A
:103140004FEA122808F0FF0883F06EFC4FEA12489D
:1031500008F0FF0883F068FC4FEA126883F064FC13
:103160004AF644424FEA420290F88833A92B08BF3E
:103170005200904608F0FF0883F056FC4FEA1228F0
:1031800008F0FF0883F050FC4FEA124808F0FF08EF
:1031900083F04AFC4FEA126883F046FC4FF00202CB
:1031A00090F88833A92B08BF5200904608F0FF081A
:1031B00083F03AFC4FEA122808F0FF0883F034FC51
:1031C0004FF01002904608F0FF0883F02DFC4FEA04
:1031D000122808F0FF0883F027FC4FF0470883F01F
:1031E00023FC4FF04D0883F01FFC4FF0410883F0A3
:1031F0001BFC4FF04E0883F017FC4FF01002904676
:1032000008F0FF0883F010FC4FEA122808F0FF08CE
:1032100083F00AFC4FEA124808F0FF0883F004FC30
:103220004FEA126883F000FC90F8028383F0FCFB05
:1032300090F8038383F0F8FB90F8048383F0F4FBA9
:1032400090F8058383F0F0FB90F8068383F0ECFBA5
:1032500090F8078383F0E8FB90F8088383F0E4FBA1
:1032600090F8098383F0E0FB90F80A8383F0DCFB9D
:1032700090F80B8383F0D8FB90F80C8383F0D4FB99
:1032800090F80D8383F0D0FB90F80E8383F0CCFB95
:1032900090F80F8383F0C8FB90F8108383F0C4FB91
:1032A00090F8118383F0C0FB4FF0470883F0BCFB1C
:1032B0004FF0540883F0B8FB4FF0450883F0B4FB9F
:1032C0004FF04D0883F0B0FB4FF00202904608F03B
:1032D000FF0883F0A9FB4FEA122808F0FF0883F0EB
:1032E000A3FB4FEA124808F0FF0883F09DFB4FEA6A
:1032F000126883F099FBB0F8F421904608F0FF08BB
:1033000083F092FB4FEA122808F0FF0883F08CFB51
:103310004FF0640883F088FB4FF0610883F084FB72
:103320004FF0740883F080FB4FF0610883F07CFB62
:10333000D0F85C23904608F0FF0883F075FB4FEA55
:10334000122808F0FF0883F06FFB4FEA124808F0DC
:10335000FF0883F069FB4FEA126883F065FBD0F841
:10336000D063C28B002AFCD190F8B31311F0010195
:1033700040F0978034464FF6FF72C0F2010226EA11
:10338000020604EA02044FF0000380F003FBC0F8D9
:10339000E03346EA0406C28B002AFCD190F8B3134E
:1033A00011F0010140F08E804FF6FF72C0F2010271
:1033B00012EA060405D1D0F8E03380F0EBFAC0F849
:1033C000E0337FF0ECFD41F2000BC2F2020B4FF450
:1033D000806240F2FF7707EA0607174440F60208CA
:1033E000474503D3A7F50067A2EB0702C0F85C23AB
:1033F0000BEB02094FF00007C0F600074FF400681E
:10340000A76100BF00BF00BF00BF95F811A0C4F8BE
:1034100018800BF801ABCB45F2D14FF08007AF61BC
:1034200041F20003C2F20203D0F85C2303EB02096D
:10343000D0F8D473A7EB0607974205D2002F10D01F
:1034400003EB0709C0F85C7313F8018B83F0ECFA07
:103450004B45F9D1D0F85C733E44D0F8D473BE42EA
:1034600099D3D0F8E023002A0DD0C38B002BFCD1D8
:103470004FF480644FF0000883F0D6FA013CFBD192
:10348000B2F58062F1D14FF00D0883F0CDFA4FF024
:103490001401A0F83A134FF00002A0F83C23FCF707
:1034A000FFBD34464FF6FF72C0F2010226EA020663
:1034B00004EA02044FF0000380F07FFAC0F8E03322
:1034C00046EA04064FF6FF72C0F2010212EA060451
:1034D00005D1D0F8E03380F070FAC0F8E0337FF027
:1034E00044FE41F2000BC2F2020B4FF4806240F244
:1034F000FF7707EA0607174440F60208474503D35B
:10350000A7F50067A2EB0702C0F85C230BEB0209EA
:103510004FF00007C0F600074FF40068A76100BF36
:1035200000BF00BF00BF95F811A0C4F818800BF8C9
:1035300001ABCB45F2D140F60009C4F202094FF0CD
:103540002007C9F8187041F20003C2F20203D0F854
:103550005C2303EB0209D0F8D473A7EB060797426C
:1035600005D2002F11D003EB0709C0F85C7313F8E4
:10357000018B83F059FA4B45F9D1D0F85C733E4486
:10358000D0F8D473BE42FFF406AFD0F8E023002A8F
:103590000DD0C38B002BFCD14FF480644FF000089A
:1035A00083F042FA013CFBD1B2F58062F1D14FF0D9
:1035B0000D0883F039FA4FF01401A0F83A134FF0D8
:1035C0000002A0F83C23FCF76BBDC3E1142943D1F2
:1035D00045F20023C1F20003151F3CD3595D442975
:1035E00039D105F10105595D3A2934D105F10105BB
:1035F000595D5C292FD105F10105595D3E292AD17C
:103600004FF00002A0F83C2390F8A31211F0010142
:1036100005D14FF0010180F8A312FCF741BD4FF036
:10362000000180F8A3124FF0430883F0FDF94FF03A
:103630004C0883F0F9F94FF0460883F0F5F94FF0A4
:10364000200883F0F1F97CF053FD4FF01501A0F84C
:103650003A13FCF725BD7DE115295CD145F2002325
:10366000C1F20003151F55D3595D442952D105F10C
:103670000105595D3A294DD105F10105595D5C29D6
:1036800048D105F10105595D3E2943D14FF00002B3
:10369000A0F83C234FF00201A0F83A134FF0440881
:1036A00083F0C2F94FF0490883F0BEF94FF0520899
:1036B00083F0BAF94FF00D0883F0B6F94FF000012E
:1036C000C0F84413D0F848134FF00C02B1FBF2F1EC
:1036D00001FB02F1C0F84C136FF0000645F2004107
:1036E000C1F2000101F5007241F8046B9142FBD177
:1036F0006FF0000645F20061C1F2000101F50072B1
:1037000041F8046B9142FBD14FF00801C0F86813F7
:10371000FCF7C6BC1EE1162962D145F20023C1F2B6
:103720000003151F5BD3595D442958D105F10105EC
:10373000595D3A2953D105F10105595D5C294ED1F6
:1037400005F10105595D3E2949D14FF00002A0F86D
:103750003C2390F8391341F0010180F839134FF000
:103760000201A0F83A134FF0440883F05DF94FF0DE
:10377000490883F059F94FF0520883F055F94FF09A
:103780000D0883F051F94FF00001C0F844134FF0D9
:103790000001C0F84813D0F848134FF00C02B1FBF9
:1037A000F2F101FB02F1C0F84C136FF0000645F294
:1037B0000041C1F2000101F5007241F8046B914231
:1037C000FBD16FF0000645F20061C1F2000101F586
:1037D000007241F8046B9142FBD1FCF761BCB9E087
:1037E000172958D145F20023C1F20003151F51D308
:1037F000595D44294ED105F10105595D3A2949D158
:1038000005F10105595D5C2944D105F10105595DBA
:103810003E293FD14FF00002A0F83C234FF00201B7
:10382000A0F83A134FF0440883F0FEF84FF049082F
:1038300083F0FAF84FF0520883F0F6F84FF00D08D5
:1038400083F0F2F84FF00001C0F84413D0F84813A9
:103850004FF00C02B1FBF2F101FB02F1C0F84C1386
:103860006FF0000645F20041C1F2000101F500725F
:1038700041F8046B9142FBD16FF0000645F2006104
:10388000C1F2000101F5007241F8046B9142FBD1D5
:10389000FCF706BC5EE0182940F0E08045F200230A
:1038A000C1F20003151F55D3595D442952D105F1CA
:1038B0000105595D3A294DD105F10105595D5C2994
:1038C00048D105F10105595D3E2943D14FF0000271
:1038D000A0F83C234FF00201A0F83A134FF044083F
:1038E00083F0A2F84FF0490883F09EF84FF0520899
:1038F00083F09AF84FF00D0883F096F84FF000012E
:10390000C0F84413D0F848134FF00C02B1FBF2F1A9
:1039100001FB02F1C0F84C136FF0000645F20041C4
:10392000C1F2000101F5007241F8046B9142FBD134
:103930006FF0000645F20061C1F2000101F500726E
:1039400041F8046B9142FBD14FF00101C0F86813BC
:10395000FCF7A6BB45F20023C1F2000303EB02050E
:103960004FF0230880F04EFF4FF0460880F04AFFEA
:103970004FF05A0880F046FF4FF0330880F042FFC6
:103980004FF02C0880F03EFF4FF0320880F03AFFF5
:103990004FF0330880F036FF4FF02C0880F032FFF4
:1039A0004FF0230880F02EFF4FF05A0880F02AFFD6
:1039B0004FF0460880F026FF4FF0310880F022FFDC
:1039C0004FF0330880F01EFF4FF02C0880F01AFFF4
:1039D0004FF0230880F016FF4FF05A0880F012FFD6
:1039E0004FF04C0880F00EFF4FF0300880F00AFFD7
:1039F0004FF0310880F006FF4FF0300880F002FFF2
:103A00004FF02C0880F0FEFE4FF0310880F0FAFEF7
:103A10004FF0300880F0F6FE4FF0300880F0F2FEF4
:103A20004FF02C0880F0EEFE13F8018B80F0EAFED8
:103A3000AB42F9D14FF0000880F0E4FE4FF00002F5
:103A4000A0F83C234FF00401A0F83A1390F8391382
:103A500021F0010180F83913FCF722BB192940F04D
:103A60009C8045F20023C1F20003151F21D3595D4C
:103A700044291ED105F10105595D3A2919D105F1F5
:103A80000105595D5C2914D105F10105595D3E29F7
:103A90000FD14FF00002A0F83C234FF04001C0F8D6
:103AA000681390F8391321F0010180F83913FCF7FD
:103AB000B3BA45F20025C1F2000515F8011B4329F0
:103AC0007FF448AF15F8011B6F297FF443AF15F859
:103AD000011B6D297FF43EAF15F8011B6D297FF4A2
:103AE00039AF15F8011B61297FF434AF15F8011BBC
:103AF0006E297FF42FAF15F8011B64297FF42AAFDC
:103B000015F8011B20297FF425AF15F8011B462964
:103B10007FF420AF15F8011B61297FF41BAF15F866
:103B2000011B69297FF416AF15F8011B6C297FF47E
:103B300011AF15F8011B65297FF40CAF15F8011BB7
:103B400064297FF407AF4FF00002A0F83C234FF048
:103B50004F0882F069FF4FF0500882F065FF4FF088
:103B6000570882F061FF4FF0200882F05DFF7CF083
:103B7000BFFA4FF01301A0F83A1390F8391341F04F
:103B8000010180F839134FF40071C0F868134FF049
:103B9000000180F8BD10FCF73FBA1A292CD145F27C
:103BA0000023C1F20003151FFFF4D4AE595D442970
:103BB0007FF4D0AE05F10105595D3A297FF4CAAE14
:103BC00005F10105595D5C297FF4C4AE05F10105DD
:103BD000595D3E297FF4BEAE4FF00002A0F83C23B1
:103BE0004FF00401A0F83A1390F8391321F00101C5
:103BF00080F83913FCF754BA1B2938D145F2002359
:103C0000C1F20003151FFFF4A5AE595D44297FF4EE
:103C1000A1AE05F10105595D3A297FF49BAE05F18E
:103C20000105595D5C297FF495AE05F10105595DEB
:103C30003E297FF48FAE4FF00002A0F83C234FF0F6
:103C4000440882F0F1FE4FF04C0882F0EDFE4FF098
:103C5000460882F0E9FE4FF0200882F0E5FE7CF095
:103C600047FA4FF01C01A0F83A13FCF719BA1C29C7
:103C700021D145F20023C1F20003151FFFF46AAE03
:103C8000595D44297FF466AE05F10105595D3A2975
:103C90007FF460AE05F10105595D5C297FF45AAEF1
:103CA00005F10105595D3E297FF454AE4FF0000245
:103CB000A0F83C234BE71D2940F0A38045F20023E8
:103CC000C1F20003151F2CD3595D442929D105F1F8
:103CD0000105595D3A2924D105F10105595D5C2999
:103CE0001FD105F10105595D3E291AD14FF000029F
:103CF000A0F83C2390F8331111F0010205D011F027
:103D0000020225F03D8024F052BA4FF48071C0F8D1
:103D1000681390F8391321F0010180F83913FCF78A
:103D20007BB945F20025C1F2000515F8011B4329B6
:103D30007FF410AE15F8011B6F297FF40BAE15F858
:103D4000011B6D297FF406AE15F8011B6D297FF468
:103D500001AE15F8011B61297FF4FCAD15F8011BBC
:103D60006E297FF4F7AD15F8011B64297FF4F2ADDD
:103D700015F8011B20297FF4EDAD15F8011B46292C
:103D80007FF4E8AD15F8011B61297FF4E3AD15F868
:103D9000011B69297FF4DEAD15F8011B6C297FF446
:103DA000D9AD15F8011B65297FF4D4AD15F8011BB9
:103DB00064297FF4CFAD4FF00002A0F83C234FF010
:103DC0004F0882F031FE4FF0500882F02DFE4FF088
:103DD000570882F029FE4FF0200882F025FE7CF083
:103DE00087F94FF01E01A0F83A1390F8391341F00B
:103DF000010180F839134FF40071C0F86813FCF723
:103E00000BB91E2940F01B8345F20023C1F20003C9
:103E1000151FFFF49FAD595D44297FF49BAD05F15B
:103E20000105595D3A297FF495AD05F10105595D0C
:103E30005C297FF48FAD05F10105595D3E297FF4C2
:103E400089AD4FF0570882F0EFFD4FF0520882F035
:103E5000EBFD4FF0460882F0E7FD4FF0200882F0BE
:103E6000E3FDD0F8D013D0F8D423A2EB0102C0F8C0
:103E70005C2302F14E024FEA126882F0D5FD4FEA50
:103E8000124808F0FF0882F0CFFD4FEA122808F030
:103E9000FF0882F0C9FD904608F0FF0882F0C4FDDB
:103EA0004FF00D0882F0C0FD4FF0520882F0BCFDCB
:103EB0004FF0490882F0B8FD4FF0460882F0B4FD9B
:103EC0004FF0460882F0B0FDD0F85C2302F14602C4
:103ED000904608F0FF0882F0A7FD4FEA122808F08C
:103EE000FF0882F0A1FD4FEA124808F0FF0882F0B7
:103EF0009BFD4FEA126882F097FD4FF0570882F061
:103F000093FD4FF0410882F08FFD4FF0560882F08C
:103F10008BFD4FF0450882F087FD4FF0660882F078
:103F200083FD4FF06D0882F07FFD4FF0740882F042
:103F30007BFD4FF0200882F077FD4FF01002904695
:103F400008F0FF0882F070FD4FEA122808F0FF0821
:103F500082F06AFD4FEA124808F0FF0882F064FD23
:103F60004FEA126882F060FD4FF00102904608F0BF
:103F7000FF0882F059FD4FEA122808F0FF0882F08E
:103F800053FD4FF0010290F88833A92B08BF52006F
:103F9000904608F0FF0882F047FD4FEA122808F02B
:103FA000FF0882F041FD4AF64442904608F0FF08BF
:103FB00082F03AFD4FEA122808F0FF0882F034FD43
:103FC0004FEA124808F0FF0882F02EFD4FEA12680F
:103FD00082F02AFD4AF644424FEA420290F88833C2
:103FE000A92B08BF5200904608F0FF0882F01CFD84
:103FF0004FEA122808F0FF0882F016FD4FEA124837
:1040000008F0FF0882F010FD4FEA126882F00CFD04
:104010004FF0020290F88833A92B08BF5200904657
:1040200008F0FF0882F000FD4FEA122808F0FF08B0
:1040300082F0FAFC4FF01002904608F0FF0882F080
:10404000F3FC4FEA122808F0FF0882F0EDFC4FF075
:10405000470882F0E9FC4FF04D0882F0E5FC4FF094
:10406000410882F0E1FC4FF04E0882F0DDFC4FF099
:104070001002904608F0FF0882F0D6FC4FEA1228A2
:1040800008F0FF0882F0D0FC4FEA124808F0FF0861
:1040900082F0CAFC4FEA126882F0C6FC90F80283F4
:1040A00082F0C2FC90F8038382F0BEFC90F8048397
:1040B00082F0BAFC90F8058382F0B6FC90F8068393
:1040C00082F0B2FC90F8078382F0AEFC90F808838F
:1040D00082F0AAFC90F8098382F0A6FC90F80A838B
:1040E00082F0A2FC90F80B8382F09EFC90F80C8387
:1040F00082F09AFC90F80D8382F096FC90F80E8383
:1041000082F092FC90F80F8382F08EFC90F810837E
:1041100082F08AFC90F8118382F086FC4FF0470809
:1041200082F082FC4FF0540882F07EFC4FF045088C
:1041300082F07AFC4FF04D0882F076FC4FF00202DC
:10414000904608F0FF0882F06FFC4FEA122808F052
:10415000FF0882F069FC4FEA124808F0FF0882F07D
:1041600063FC4FEA126882F05FFCB0F8F4219046DD
:1041700008F0FF0882F058FC4FEA122808F0FF0808
:1041800082F052FC4FF0640882F04EFC4FF0610860
:1041900082F04AFC4FF0740882F046FC4FF0610850
:1041A00082F042FCD0F85C23904608F0FF0882F0D1
:1041B0003BFC4FEA122808F0FF0882F035FC4FEA7A
:1041C000124808F0FF0882F02FFC4FEA126882F0D4
:1041D0002BFCD0F8D063C28B002AFCD190F8B3132B
:1041E00011F0010140F0978034464FF6FF72C0F2A3
:1041F000010226EA020604EA02044FF000037FF0FF
:10420000C9FBC0F8E03346EA0406C28B002AFCD1A1
:1042100090F8B31311F0010140F08E804FF6FF7259
:10422000C0F2010212EA060405D1D0F8E0337FF0B3
:10423000B1FBC0F8E0337EF0B2FE41F2000BC2F2F7
:10424000020B4FF4806240F2FF7707EA060717443B
:1042500040F60208474503D3A7F50067A2EB070223
:10426000C0F85C230BEB02094FF00007C0F6000713
:104270004FF40068A76100BF00BF00BF00BF95F802
:1042800011A0C4F818800BF801ABCB45F2D14FF068
:104290008007AF6141F20003C2F20203D0F85C2351
:1042A00003EB0209D0F8D473A7EB0607974205D2B7
:1042B000002F10D003EB0709C0F85C7313F8018BD3
:1042C00082F0B2FB4B45F9D1D0F85C733E44D0F894
:1042D000D473BE4299D3D0F8E023002A0DD0C38B0B
:1042E000002BFCD14FF480644FF0000882F09CFB5F
:1042F000013CFBD1B2F58062F1D14FF00D0882F0A4
:1043000093FB4FF01F01A0F83A134FF00002A0F802
:104310003C23FBF7C5BE34464FF6FF72C0F20102E4
:1043200026EA020604EA02044FF000037FF045FB90
:10433000C0F8E03346EA04064FF6FF72C0F201020D
:1043400012EA060405D1D0F8E0337FF036FBC0F85E
:10435000E0337EF00AFF41F2000BC2F2020B4FF491
:10436000806240F2FF7707EA0607174440F602082A
:10437000474503D3A7F50067A2EB0702C0F85C230B
:104380000BEB02094FF00007C0F600074FF400687E
:10439000A76100BF00BF00BF00BF95F811A0C4F81F
:1043A00018800BF801ABCB45F2D140F60009C4F2FE
:1043B00002094FF02007C9F8187041F20003C2F259
:1043C0000203D0F85C2303EB0209D0F8D473A7EB07
:1043D0000607974205D2002F11D003EB0709C0F85A
:1043E0005C7313F8018B82F01FFB4B45F9D1D0F8B9
:1043F0005C733E44D0F8D473BE42FFF406AFD0F8ED
:10440000E023002A0DD0C38B002BFCD14FF4806435
:104410004FF0000882F008FB013CFBD1B2F580624E
:10442000F1D14FF00D0882F0FFFA4FF01F01A0F814
:104430003A134FF00002A0F83C23FBF731BE1F29CE
:104440004BD145F20023C1F20003151FFFF482AAED
:10445000595D44297FF47EAA05F10105595D3A2989
:104460007FF478AA05F10105595D5C297FF472AAF1
:1044700005F10105595D3E297FF46CAA4FF0000259
:10448000A0F83C2390F8A31211F0010105D14FF0E0
:10449000010180F8A312FBF703BE4FF0000180F882
:1044A000A3124FF0430882F0BFFA4FF04C0882F09D
:1044B000BBFA4FF0460882F0B7FA4FF0200882F0BE
:1044C000B3FA7BF015FE4FF02001A0F83A134FF03D
:1044D0000002A0F83C23FBF7E3BD202940F09B80BD
:1044E00045F20023C1F20003151FFFF433AA595D02
:1044F00044297FF42FAA05F10105595D3A297FF47B
:1045000029AA05F10105595D5C297FF423AA05F16B
:104510000105595D3E297FF41DAAB0F88E1301F103
:104520000101A0F88E13B0F8602090F8B33313F0B7
:1045300001031CBFA1F50061B0F8B823914226D059
:1045400090F8B33313F0010318BF01F50061A0F830
:10455000001386F03CFB4FF04F0882F065FA4FF0F5
:10456000500882F061FA4FF0520882F05DFA4FF085
:10457000200882F059FA7BF0BBFD4FF01D01A0F836
:104580003A134FF00002A0F83C23FBF789BD4FF02F
:104590000002A0F83C234FF00201A0F83A134FF0BC
:1045A000440882F041FA4FF0490882F03DFA4FF09A
:1045B000520882F039FA4FF00D0882F035FA4FF0C8
:1045C0000001C0F84413D0F848134FF00C02B1FBBF
:1045D000F2F101FB02F1C0F84C136FF0000645F256
:1045E0000041C1F2000101F5007241F8046B9142F3
:1045F000FBD16FF0000645F20061C1F2000101F548
:10460000007241F8046B9142FBD14FF00801C0F8F1
:104610006813FBF745BD212921D145F20023C1F2E2
:104620000003151FFFF496A9595D44297FF492A950
:1046300005F10105595D3A297FF48CA905F10105C1
:10464000595D5C297FF486A905F10105595D3E2974
:104650007FF480A94FF00002A0F83C235DE72229F7
:1046600038D145F20023C1F20003151FFFF472A9EF
:10467000595D44297FF46EA905F10105595D3A2978
:104680007FF468A905F10105595D5C297FF462A9F1
:1046900005F10105595D3E297FF45CA94FF0000248
:1046A000A0F83C234FF0440882F0BEF94FF04C08CC
:1046B00082F0BAF94FF0460882F0B6F94FF02008C0
:1046C00082F0B2F97BF014FD4FF02301A0F83A1309
:1046D000FBF7E6BC232922D145F20023C1F20003F7
:1046E000151FFFF437A9595D44297FF433A905F15B
:1046F0000105595D3A297FF42DA905F10105595DA0
:104700005C297FF427A905F10105595D3E297FF455
:1047100021A94FF00002A0F83C23FFF750BB242949
:1047200060D145F20023C1F20003151FFFF412A966
:10473000595D44297FF40EA905F10105595D3A2917
:104740007FF408A905F10105595D5C297FF402A9F0
:1047500005F10105595D3E297FF4FCA84FF00001E9
:10476000C0F848134FF00002A0F83C234FF0250199
:10477000A0F83A134FF0440882F056F94FF0490878
:1047800082F052F94FF0520882F04EF94FF00D08C6
:1047900082F04AF94FF00001C0F84413D0F84813F2
:1047A0004FF00C02B1FBF2F101FB02F1C0F84C1327
:1047B0006FF0000645F20041C1F2000101F5007200
:1047C00041F8046B9142FBD16FF0000645F20061A5
:1047D000C1F2000101F5007241F8046B9142FBD176
:1047E000FBF75EBC252940F01E8145F20023C1F293
:1047F0000003151F58D3595D442920D105F1010547
:10480000595D3A291BD105F10105595D5C2916D185
:1048100005F10105595D3E2911D141F20046C4F26E
:104820000106376817F00F0808D03768776890F8E6
:104830006D7007F1010780F86D7093E76DE0151F4B
:1048400032D3595D2E2951D105F10105595D572902
:104850003FD105F10105595D412925D105F101053A
:10486000595D562920D1D0F8441301F10101C0F857
:104870004413D0F84C13002909D0A1F10101C0F86C
:104880004C134FF00002A0F83C23FBF709BC45F2A3
:104890000046C1F2000606F1C0073178FF2909D0B1
:1048A00006F11006BE42F8D14FF00002A0F83C23FA
:1048B000FBF7F6BB4FF00005595D06F8011B05F14B
:1048C00001059542F8D14FF00002A0F83C23FBF718
:1048D000E7BB4629E8D105F10105595D5A29E3D125
:1048E00005F10105595D5029DED1BCE72029DBD156
:1048F00005F10105595D4429D6D105F10105595D40
:104900004929D1D105F10105595D5229CCD1A5F133
:1049100003054FF02E015955A5E790F8391321F002
:10492000010180F8391345F20042C1F2000211780A
:10493000FF29B9D04FF02601A0F83A134FF000013B
:10494000A0F83E1345F20042C1F2000202F1C00499
:10495000B0F83E334FEA03131A44A24200F0CE816E
:104960001178FF2900F0CA814FF0010912F80910EF
:104970002E2902D009F10109F8E709F1010912F81D
:10498000091057290CD109F1010912F80910412920
:1049900042D109F1010912F8091056293CD10DE064
:1049A000462939D109F1010912F809105A2933D1E0
:1049B00009F1010912F8091050292DD109F1060950
:1049C00080F85F904FF0440882F02EF84FF04908CD
:1049D00082F02AF84FF0520882F026F84FF02008B3
:1049E00082F022F812F8018BB8F1FF0F04D082F0A8
:1049F0001BF812F00F01F5D14FF00D0882F014F8FA
:104A0000B0F83E1301F10101A0F83E134FF000028F
:104A1000A0F83C23FBF744BBB0F83E1301F10101C1
:104A2000A0F83E138EE7262940F0C08241F20046EE
:104A3000C4F20106376817F00F080ED037687768A0
:104A400090F86D7007F1010780F86D70D0F83E6343
:104A5000A6F10106C0F83E63D6E045F20023C1F29C
:104A60000003B2F10905C4F0B586595D2E2944F062
:104A7000B18605F10105595D572940F0878205F19E
:104A80000105595D412940F0338105F10105595D6A
:104A9000562940F02D8145F20046C1F2000606F18C
:104AA000C00790F85F90A2EB09053178FF2900F06C
:104AB0001F8113F80580884540F0158105F1010537
:104AC0007178FF2900F0918013F80580884540F047
:104AD0000A8105F10105B178FF2900F0868013F8FD
:104AE0000580884540F0FF8005F10105F178FF2938
:104AF0007BD013F80580884540F0F58005F101056D
:104B00003179FF2971D013F80580884540F0EB809A
:104B100005F101057179FF2967D013F805808845F3
:104B200040F0E18005F10105B179FF295DD013F86E
:104B30000580884540F0D78005F10105F179FF290E
:104B400053D013F80580884540F0CD8005F101056C
:104B5000317AFF2949D013F80580884540F0C38099
:104B600005F10105717AFF293FD013F805808845CA
:104B700040F0B98005F10105B17AFF2935D013F86D
:104B80000580884540F0AF8005F10105F17AFF29E5
:104B90002BD013F80580884540F0A58005F101056C
:104BA000317BFF2921D013F80580884540F09B8098
:104BB00005F10105717BFF2917D013F805808845A1
:104BC00040F0918005F10105B17BFF290DD013F86C
:104BD0000580884540F0878005F10105F17BFF29BC
:104BE00003D013F8058088457DD106F50076A2F143
:104BF00004054FF0A90106F8041B595D06F8011BD6
:104C000005F101059542F8D145F20042C1F20002DA
:104C100002F1C004B0F83E334FEA03131A44A24233
:104C20006CD01178FF2969D04FF0010912F80910F2
:104C30002E2902D009F10109F8E709F1010912F85A
:104C4000091057290CD109F1010912F8091041295D
:104C500042D109F1010912F8091056293CD10DE0A1
:104C6000462939D109F1010912F809105A2933D11D
:104C700009F1010912F8091050292DD109F106098D
:104C800080F85F904FF0440881F0CEFE4FF0490865
:104C900081F0CAFE4FF0520881F0C6FE4FF02008A6
:104CA00081F0C2FE12F8018BB8F1FF0F04D081F041
:104CB000BBFE12F00F01F5D14FF00D0881F0B4FEEC
:104CC000B0F83E1301F10101A0F83E134FF00002CD
:104CD000A0F83C23FBF7E4B9B0F83E1301F1010161
:104CE000A0F83E1390E706F11006BE427FF4D9AE5D
:104CF0004FF00002A0F83C23FBF7D2B94FF02C0193
:104D0000A0F83A134FF00002A0F83C23FBF7C8B913
:104D1000D0F848134FF00C02B1FBF2F303FB02F39F
:104D2000A1EB030145F20049C1F200094FEA01116C
:104D300089444FF0000519F80510FF293BF489A9B3
:104D40002E2902D005F10105F5E705F1010519F855
:104D5000051057290CD105F1010519F80510412955
:104D600043D105F1010519F8051056293DD10EE092
:104D700046293AD105F1010519F805105A2934D10F
:104D800005F1010519F8051050292ED187E04FF0E3
:104D90004F0881F049FE4FF0500881F045FE4FF07A
:104DA000520881F041FE4FF0200881F03DFE19F8D5
:104DB000018BB8F1FF0F04D081F036FE19F00F011E
:104DC000F5D14FF00D0881F02FFE4FF02701A0F82C
:104DD0003A1390F8391341F0010180F839134FF07C
:104DE0000002A0F83C23FBF75BB9D0F848134FF062
:104DF0000C03B1FBF3F501F10101D0F8442391421A
:104E000080F08180C0F84813B1FBF3F4A54200D1D3
:104E10007EE74FF02501A0F83A1390F8391341F0DE
:104E2000010180F839134FF0440881F0FDFD4FF087
:104E3000490881F0F9FD4FF0520881F0F5FD4FF07F
:104E40000D0881F0F1FD4FF00001C0F84413D0F8D7
:104E500048134FF00C02B1FBF2F101FB02F1C0F874
:104E60004C136FF0000645F20041C1F2000101F55C
:104E7000007241F8046B9142FBD16FF0000645F2DD
:104E80000061C1F2000101F5007241F8046B91422A
:104E9000FBD14FF00002A0F83C23FBF701B94FF41F
:104EA0000061C0F85013C0F85C134FF04F0881F058
:104EB000BBFD4FF0500881F0B7FD4FF0520881F074
:104EC000B3FD4FF0200881F0AFFD19F8018BB8F168
:104ED000FF0F04D081F0A8FD19F00F01F5D14FF0BC
:104EE0000D0881F0A1FD4FF03B01A0F83A1390F8B6
:104EF000391341F0010180F839134FF00002A0F896
:104F00003C23FBF7CDB8468AA0F81C6D86827CF066
:104F100087F84FF0430881F087FD4FF0440881F097
:104F200083FD4FF0200881F07FFD4FF02E0881F0C7
:104F30007BFD4FF02E0881F077FD4FF00D0881F0DA
:104F400073FD4FF01701A0F83A1390F8391341F0B0
:104F5000010180F8391390F85613A1F1010180F88E
:104F6000561340F20025C2F200054FEA810845447D
:104F7000D5F80080C0F848834FF00002A0F83C2329
:104F80004FF00101C0F86813FBF78AB846297FF497
:104F9000AFAE05F10105595D5A297FF4A9AE05F1BF
:104FA0000105595D50297FF4A3AE74E5272952D13C
:104FB00045F20023C1F20003151FFEF4CBAC595D8E
:104FC00044297EF4C7AC05F10105595D3A297EF408
:104FD000C1AC05F10105595D5C297EF4BBAC05F15E
:104FE0000105595D3E297EF4B5AC4FF0520881F0C1
:104FF0001BFD4FF0440881F017FD4FF0460881F08B
:1050000013FD4FF0200881F00FFD4FF04E02C0F865
:1050100050234FEA126881F007FD4FEA124808F06A
:10502000FF0881F001FD4FEA122808F0FF0881F027
:10503000FBFC02F0FF0881F0F7FC4FF00D0881F057
:10504000F3FC4FF02801A0F83A134FF00002A0F84B
:105050003C23FBF725B8282940F0648241F2004642
:10506000C4F20106376817F00F0835D03768776843
:1050700090F86D7007F1010780F86D704FF05308DC
:1050800081F0D2FC4FF0450881F0CEFC4FF04B0888
:1050900081F0CAFC4FF0200881F0C6FC4FF00008F8
:1050A00081F0C2FC4FF0000881F0BEFC4FF0000818
:1050B00081F0BAFC4FF0000881F0B6FC4FF00D080B
:1050C00081F0B2FC4FF02701A0F83A134FF0000234
:1050D000A0F83C23FAF7E4BF45F20023C1F2000335
:1050E000151FFEF437AC595D44297EF433AC05F14D
:1050F0000105595D3A297EF42DAC05F10105595D94
:105100005C297EF427AC05F10105595D3E297EF44A
:1051100021AC45F6000AC1F2000A1AF8011B522917
:1051200040F0C7811AF8011B492940F0C2811AF8E2
:10513000011B462940F0BD811AF8051B462940F0A5
:10514000B8811AF8011B572940F0B3811AF8011BE6
:10515000412940F0AE811AF8011B562940F0A9817F
:105160001AF8011B452940F0A4811AF8011B662991
:1051700040F09F811AF8011B6D2940F09A811AF8BE
:10518000011B742940F095811AF8011B202940F079
:1051900090815AF8041B102940F08B813AF8021BC9
:1051A000012940F086814FF000023AF80C1B0229D9
:1051B00008BF012280F886233AF8021B102940F02C
:1051C00078814FF0000180F8D01180F8C61F4FF0B1
:1051D0002401C0F86C1345F6000AC1F2000A0AF176
:1051E000240A9AF80010472940F09B809AF8011091
:1051F0004D2940F096809AF80210412940F09180A4
:105200009AF803104E2940F08C804FF0010180F88D
:10521000D0119AF8081080F8B0129AF8091080F8A6
:10522000B1129AF80A1080F8B2129AF80B1080F8AE
:10523000B3129AF80C1080F8B4129AF80D1080F896
:10524000B5129AF80E1080F8B6129AF80F1080F87E
:10525000B7129AF8101080F8B8129AF8111080F866
:10526000B9129AF8121080F8BA129AF8131080F84E
:10527000BB129AF8141080F8BC129AF8151080F836
:10528000BD129AF8161080F8BE129AF8171080F81E
:10529000BF124FF03C01C0F86C1345F6000AC1F292
:1052A000000ADAF83C10CAF82410DAF84010CAF8FC
:1052B000281045F6000AC1F2000A0AF13C0A9AF8E1
:1052C000001047292DD19AF80110542929D19AF8B4
:1052D0000210452925D19AF803104D2921D14FF00C
:1052E000010180F8C61F9AF808909AF8091009F091
:1052F000FF0901F0FF014FEA012149EA0109A0F885
:10530000C49F4FF04601C0F86C1345F6000AC1F285
:10531000000ADAF84610CAF82410DAF84A10CAF877
:10532000281045F6000AC1F2000A0AF1240A9AF888
:10533000001064290BD19AF80110612907D19AF85D
:105340000210742903D19AF8031061293AD0DAF8CF
:10535000041001F10801D0F86C938944C0F86C93F3
:105360004FF0530881F060FB4FF0450881F05CFB83
:105370004FF04B0881F058FB4FF0200881F054FBB0
:105380004FEA196881F050FB4FEA194808F0FF080E
:1053900081F04AFB4FEA192808F0FF0881F044FB2E
:1053A00009F0FF0881F040FB4FF00D0881F03CFB55
:1053B0004FF03001A0F83A134FF00002A0F83C2360
:1053C000FAF76EBE90F8FF1200297CF44BA990F812
:1053D000B23313F001030ED1426E4FF480414FEA15
:1053E00001418A42BCF453AAB0F86060B6F5006F80
:1053F000BCF44DAA0EE0D0F8B4234FF480414FEA3C
:1054000001418A42BCF443AAB0F8B863B6F5805FA4
:10541000BCF43DAAC0F8EC2245F60005C1F2000537
:10542000AB6A13444FF480414FEA01418B4228BFDD
:105430000B46C0F858334FF0530881F0F5FA4FF09F
:10544000450881F0F1FA4FF04B0881F0EDFA4FF08A
:10545000200881F0E9FAD0F86C6306F108064FEAFB
:10546000166881F0E1FA4FEA164808F0FF0881F06B
:10547000DBFA4FEA162808F0FF0881F0D5FA06F0AB
:10548000FF0881F0D1FA4FF00D0881F0CDFA4FF00E
:105490002901A0F83A134FF00002A0F83C234FF482
:1054A0000061C0F868134FF0000180F8BD10FAF7F2
:1054B000B3BDD0F848134FF00C02B1FBF2F303FB7D
:1054C00002F3A1EB030145F20049C1F200094FEAE2
:1054D000011189444FF0430881F0A6FA4FF04C08BF
:1054E00081F0A2FA4FF0460881F09EFA4FF02008B2
:1054F00081F09AFA19F8018BB8F1FF0F04D081F00E
:1055000093FA19F00F01F5D14FF00D0881F08CFAE4
:105510004FF02B01A0F83A134FF00002A0F83C2303
:10552000FAF7BEBD292967D145F20023C1F2000375
:10553000151FFEF40FAA595D44297EF40BAA05F14C
:105540000105595D3A297EF405AA05F10105595D69
:105550005C297EF4FFA905F10105595D3E297EF421
:10556000F9A9D0F8EC22D0F85833A3EB0203B3F535
:10557000304F05D2002B02D0C0F8503304E011E1C7
:105580004FF43043C0F85033C0F85C334FF052084A
:1055900081F04AFA4FF0440881F046FA4FF046088D
:1055A00081F042FA4FF0200881F03EFAD0F8502303
:1055B000C0F8C0204FEA126881F036FA4FEA12486C
:1055C00008F0FF0881F030FA4FEA122808F0FF08CF
:1055D00081F02AFA02F0FF0881F026FA4FF00D0858
:1055E00081F022FA4FF02A01A0F83A134FF000029E
:1055F000A0F83C23FAF754BD2A2941F0EA8041F291
:105600000046C4F20106376817F00F080ED037685D
:10561000776890F86D7007F1010780F86D7090F869
:10562000B22312F0010240F0E7847FE090F8B22349
:1056300012F0010240F0608443F2000BC2F2020B50
:10564000D0F85823446EA2EB04024FEA9212D0F82D
:10565000EC62A6EB0406B6FBF2F280F8BD20D0F8AF
:10566000EC624FF6FF72C0F2010212EA060401D1A9
:105670007EF090F944F200024FEA0242964280F036
:1056800091807DF0A3FDD0F85C934FF40067B9F5ED
:10569000006F38BF4F46C0F8F07FA9EB0709C0F88C
:1056A0005C930BEB07094FF00007C0F201074FF0C6
:1056B00001081BF801AB85F815A0A76100BF00BF6A
:1056C000C4F81880CB45F4D140F20407C0F20107BA
:1056D00040F210026A75A76140F20107C0F20407A8
:1056E00000BF00BF00BF00BFA76100BF00BF228A8C
:1056F00012F48062FBD146F62022C0F200022A603A
:1057000000BF00BF228A12F48062FBD04FF08007F6
:10571000AF61D0F8F04F2644C0F8EC62D0F85C439B
:10572000002C8DD1D0F85843A6423BD24FF05308FD
:1057300081F07AF94FF0450881F076F94FF04B0887
:1057400081F072F94FF0200881F06EF9D0F8EC6228
:10575000456EA6EB0506D0F86C5305F108052E44FE
:105760004FEA166881F060F94FEA164808F0FF0822
:1057700081F05AF94FEA162808F0FF0881F054F931
:1057800006F0FF0881F050F94FF00D0881F04CF958
:105790004FF02901A0F83A134FF00002A0F83C2383
:1057A000FAF77EBC466E4FF00101C1727EF0F2F84E
:1057B00006F101067DF00AFD40F2A9024FF0000754
:1057C000C0F201076A75A76100BF00BF00BF4FF0BC
:1057D0000107A761D0F8586306F500364FEA164274
:1057E00002F0FE024FF00007C0F201076A75A761E0
:1057F00000BF00BF00BF4FF00107A7614FEA16626C
:1058000002F01F024FF00007C0F201076A75A7619E
:1058100000BF00BF00BF4FF00107A761D0F84813D9
:105820004FF00C02B1FBF2F303FB02F3A1EB030117
:1058300045F20049C1F200094FEA011189444FF0D5
:10584000000180F8571319F8012B90F8D01111F0CE
:10585000010118BF90F8B0224FF00007C0F2010715
:105860006A75A76100BF00BF00BF4FF00107A761C5
:1058700019F8012B2E2A03D14FF0010180F857139C
:1058800090F85713012908BF202290F8D01111F089
:10589000010118BF90F8B1224FF00007C0F20107D4
:1058A0006A75A76100BF00BF00BF4FF00107A76185
:1058B00019F8012B2E2A03D14FF0010180F857135C
:1058C00090F85713012908BF202290F8D01111F049
:1058D000010118BF90F8B2224FF00007C0F2010793
:1058E0006A75A76100BF00BF00BF4FF00107A76145
:1058F00019F8012B2E2A03D14FF0010180F857131C
:1059000090F85713012908BF202290F8D01111F008
:10591000010118BF90F8B3224FF00007C0F2010751
:105920006A75A76100BF00BF00BF4FF00107A76104
:1059300019F8012B2E2A03D14FF0010180F85713DB
:1059400090F85713012908BF202290F8D01111F0C8
:10595000010118BF90F8B4224FF00007C0F2010710
:105960006A75A76100BF00BF00BF4FF00107A761C4
:1059700019F8012B2E2A03D14FF0010180F857139B
:1059800090F85713012908BF202290F8D01111F088
:10599000010118BF90F8B5224FF00007C0F20107CF
:1059A0006A75A76100BF00BF00BF4FF00107A76184
:1059B00019F8012B2E2A03D14FF0010180F857135B
:1059C00090F85713012908BF202290F8D01111F048
:1059D000010118BF90F8B6224FF00007C0F201078E
:1059E0006A75A76100BF00BF00BF4FF00107A76144
:1059F00019F8012B2E2A03D14FF0010180F857131B
:105A000090F85713012908BF202290F8D01111F007
:105A1000010118BF90F8B7224FF00007C0F201074C
:105A20006A75A76100BF00BF00BF4FF00107A76103
:105A30004FF0200290F8D01111F0010118BF90F83A
:105A4000B8224FF00007C0F201076A75A76100BFD6
:105A500000BF00BF4FF00107A7614FF0200290F890
:105A6000D01111F0010118BF90F8B9224FF00007D2
:105A7000C0F201076A75A76100BF00BF00BF4FF009
:105A80000107A7614FF0200290F8D01111F0010139
:105A900018BF90F8BA224FF00007C0F201076A75EC
:105AA000A76100BF00BF00BF4FF00107A7614FF023
:105AB000200290F8D01111F0010118BF90F8BB221C
:105AC0004FF00007C0F201076A75A76100BF00BF71
:105AD00000BF4FF00107A7614FF0200290F8D011EE
:105AE00011F0010118BF90F8BC224FF00007C0F27E
:105AF00001076A75A76100BF00BF00BF4FF0010733
:105B0000A7614FF0200290F8D01111F0010118BFE9
:105B100090F8BD224FF00007C0F201076A75A76137
:105B200000BF00BF00BF4FF00107A7614FF0200288
:105B300090F8D01111F0010118BF90F8BE224FF07B
:105B40000007C0F201076A75A76100BF00BF00BF70
:105B50004FF00107A7614FF0200290F8D01111F02B
:105B6000010118BF90F8BF224FF00007C0F20107F3
:105B70006A75A76100BF00BF00BF4FF00107A761B2
:105B8000D0F858130A464FF00007C0F201076A75B3
:105B9000A76100BF00BF00BF4FF00107A7614FEA38
:105BA00011224FF00007C0F201076A75A76100BF1C
:105BB00000BF00BF4FF00107A7614FEA11424FF04D
:105BC0000007C0F201076A75A76100BF00BF00BFF0
:105BD0004FF00107A7614FEA11624FF00007C0F2D2
:105BE00001076A75A76100BF00BF00BF4FF0010742
:105BF000A76190F8863311F0010114BFA922FF229A
:105C00004FF00007C0F201076A75A76100BF00BF2F
:105C100000BF4FF00107A76190F8C61F11F0010106
:105C200000F040814FF0FF014FF00007C0F2010784
:105C30006975A76100BF00BF00BF4FF00107A761F2
:105C400000BF00BF6FF000014FF00007C0F2010776
:105C50006975A76100BF00BF00BF4FF00107A761D2
:105C600000BF00BF4FEA11224FF00007C0F201074A
:105C70006A75A76100BF00BF00BF4FF00107A761B1
:105C800000BF00BF6FF000014FF00007C0F2010736
:105C90006975A76100BF00BF00BF4FF00107A76192
:105CA00000BF00BF4FEA11224FF00007C0F201070A
:105CB0006A75A76100BF00BF00BF4FF00107A76171
:105CC00000BF00BF6FF000014FF00007C0F20107F6
:105CD0006975A76100BF00BF00BF4FF00107A76152
:105CE00000BF00BF4FEA11224FF00007C0F20107CA
:105CF0006A75A76100BF00BF00BF4FF00107A76131
:105D000000BF00BF6FF000014FF00007C0F20107B5
:105D10006975A76100BF00BF00BF4FF00107A76111
:105D200000BF00BF4FEA11224FF00007C0F2010789
:105D30006A75A76100BF00BF00BF4FF00107A761F0
:105D400000BF00BF6FF000014FF00007C0F2010775
:105D50006975A76100BF00BF00BF4FF00107A761D1
:105D600000BF00BF4FEA11224FF00007C0F2010749
:105D70006A75A76100BF00BF00BF4FF00107A761B0
:105D800000BF00BF4FEA11424FF00007C0F2010709
:105D90006A75A76100BF00BF00BF4FF00107A76190
:105DA00000BF00BF4FEA11624FF00007C0F20107C9
:105DB0006A75A76100BF00BF00BF4FF00107A76170
:105DC00000BF00BF6FF000014FF00007C0F20107F5
:105DD0006975A76100BF00BF00BF4FF00107A76151
:105DE00000BF00BF4FEA11224FF00007C0F20107C9
:105DF0006A75A76100BF00BF00BF4FF00107A76130
:105E000000BF00BF4FEA11424FF00007C0F2010788
:105E10006A75A76100BF00BF00BF4FF00107A7610F
:105E200000BF00BF4FEA11624FF00007C0F2010748
:105E30006A75A76100BF00BF00BF4FF00107A761EF
:105E400000BF00BF4FF0A9014FF00007C0F20107EB
:105E50006975A76100BF00BF00BF4FF00107A761D0
:105E600000BF00BFB0F8C42F4FF00007C0F2010719
:105E70006A75A76100BF00BF00BF4FF00107A761AF
:105E800000BF00BF4FEA12214FF00007C0F2010728
:105E90006975A76100BF00BF00BF4FF00107A76190
:105EA00000BF00BF40F20407C0F2010740F2100239
:105EB0006A75A76140F20107C0F20407A76100BF3D
:105EC00000BF228A12F48062FBD146F62022C0F283
:105ED00000022A60228A12F48062FBD04FF0000197
:105EE000C1724FF08007AF617DF0BFFB4FF0000241
:105EF000A0F83C23FFF7DDBA43F2000BC2F2020B1D
:105F0000D0F85823D0F8B443A2EB04024FEA92121F
:105F1000D0F8EC62A6EB0406B6FBF2F280F8BD20E6
:105F2000D0F8EC624FF6FF72C0F2010212EA0604EA
:105F300001D17DF042FD44F200024FEA0242964256
:105F400080F097807DF003FAD0F85C934FF40067FF
:105F5000B9F5006F38BF4F46C0F8F07FA9EB0709CD
:105F6000C0F85C930BEB07094FF00007C0F2010784
:105F70004FF001081BF801AB85F815A0A76100BF21
:105F800000BFC4F81880CB45F4D140F20407C0F23A
:105F9000010740F210026A75A76140F20107C0F2E2
:105FA000040700BF00BF00BF00BFA76100BF00BF64
:105FB000228A12F48062FBD146F62022C0F200024F
:105FC0002A6000BF00BF228A12F48062FBD040F634
:105FD0000009C4F202094FF02007C9F81870D0F880
:105FE000F04F2644C0F8EC62D0F85C43002C87D117
:105FF000D0F85843A6423CD24FF0530880F014FD2D
:106000004FF0450880F010FD4FF04B0880F00CFD7C
:106010004FF0200880F008FDD0F8EC62D0F8B453BF
:10602000A6EB0506D0F86C5305F108052E444FEA9F
:10603000166880F0F9FC4FEA164808F0FF0880F077
:10604000F3FC4FEA162808F0FF0880F0EDFC06F09C
:10605000FF0880F0E9FC4FF00D0880F0E5FC4FF000
:106060002901A0F83A134FF00002A0F83C23FAF7F8
:1060700017B8D0F8B4634FF00101C1727DF09DFCF8
:1060800006F101067DF063F940F2A9024FF0000726
:10609000C0F201076A75A76100BF00BF00BF4FF0E3
:1060A0000107A761D0F8586306F500364FEA16429B
:1060B00002F0FE024FF00007C0F201076A75A76107
:1060C00000BF00BF00BF4FF00107A7614FEA166293
:1060D00002F01F024FF00007C0F201076A75A761C6
:1060E00000BF00BF00BF4FF00107A761D0F8481301
:1060F0004FF00C02B1FBF2F303FB02F3A1EB03013F
:1061000045F20049C1F200094FEA011189444FF0FC
:10611000000180F8571319F8012B90F8D01111F0F5
:10612000010118BF90F8B0224FF00007C0F201073C
:106130006A75A76100BF00BF00BF4FF00107A761EC
:1061400019F8012B2E2A03D14FF0010180F85713C3
:1061500090F85713012908BF202290F8D01111F0B0
:10616000010118BF90F8B1224FF00007C0F20107FB
:106170006A75A76100BF00BF00BF4FF00107A761AC
:1061800019F8012B2E2A03D14FF0010180F8571383
:1061900090F85713012908BF202290F8D01111F070
:1061A000010118BF90F8B2224FF00007C0F20107BA
:1061B0006A75A76100BF00BF00BF4FF00107A7616C
:1061C00019F8012B2E2A03D14FF0010180F8571343
:1061D00090F85713012908BF202290F8D01111F030
:1061E000010118BF90F8B3224FF00007C0F2010779
:1061F0006A75A76100BF00BF00BF4FF00107A7612C
:1062000019F8012B2E2A03D14FF0010180F8571302
:1062100090F85713012908BF202290F8D01111F0EF
:10622000010118BF90F8B4224FF00007C0F2010737
:106230006A75A76100BF00BF00BF4FF00107A761EB
:1062400019F8012B2E2A03D14FF0010180F85713C2
:1062500090F85713012908BF202290F8D01111F0AF
:10626000010118BF90F8B5224FF00007C0F20107F6
:106270006A75A76100BF00BF00BF4FF00107A761AB
:1062800019F8012B2E2A03D14FF0010180F8571382
:1062900090F85713012908BF202290F8D01111F06F
:1062A000010118BF90F8B6224FF00007C0F20107B5
:1062B0006A75A76100BF00BF00BF4FF00107A7616B
:1062C00019F8012B2E2A03D14FF0010180F8571342
:1062D00090F85713012908BF202290F8D01111F02F
:1062E000010118BF90F8B7224FF00007C0F2010774
:1062F0006A75A76100BF00BF00BF4FF00107A7612B
:106300004FF0200290F8D01111F0010118BF90F861
:10631000B8224FF00007C0F201076A75A76100BFFD
:1063200000BF00BF4FF00107A7614FF0200290F8B7
:10633000D01111F0010118BF90F8B9224FF00007F9
:10634000C0F201076A75A76100BF00BF00BF4FF030
:106350000107A7614FF0200290F8D01111F0010160
:1063600018BF90F8BA224FF00007C0F201076A7513
:10637000A76100BF00BF00BF4FF00107A7614FF04A
:10638000200290F8D01111F0010118BF90F8BB2243
:106390004FF00007C0F201076A75A76100BF00BF98
:1063A00000BF4FF00107A7614FF0200290F8D01115
:1063B00011F0010118BF90F8BC224FF00007C0F2A5
:1063C00001076A75A76100BF00BF00BF4FF001075A
:1063D000A7614FF0200290F8D01111F0010118BF11
:1063E00090F8BD224FF00007C0F201076A75A7615F
:1063F00000BF00BF00BF4FF00107A7614FF02002B0
:1064000090F8D01111F0010118BF90F8BE224FF0A2
:106410000007C0F201076A75A76100BF00BF00BF97
:106420004FF00107A7614FF0200290F8D01111F052
:10643000010118BF90F8BF224FF00007C0F201071A
:106440006A75A76100BF00BF00BF4FF00107A761D9
:10645000D0F858130A464FF00007C0F201076A75DA
:10646000A76100BF00BF00BF4FF00107A7614FEA5F
:1064700011224FF00007C0F201076A75A76100BF43
:1064800000BF00BF4FF00107A7614FEA11424FF074
:106490000007C0F201076A75A76100BF00BF00BF17
:1064A0004FF00107A7614FEA11624FF00007C0F2F9
:1064B00001076A75A76100BF00BF00BF4FF0010769
:1064C000A76190F8863311F0010114BFA922FF22C1
:1064D0004FF00007C0F201076A75A76100BF00BF57
:1064E00000BF4FF00107A76190F8C61F11F001012E
:1064F00000F040814FF0FF014FF00007C0F20107AC
:106500006975A76100BF00BF00BF4FF00107A76119
:1065100000BF00BF6FF000014FF00007C0F201079D
:106520006975A76100BF00BF00BF4FF00107A761F9
:1065300000BF00BF4FEA11224FF00007C0F2010771
:106540006A75A76100BF00BF00BF4FF00107A761D8
:1065500000BF00BF6FF000014FF00007C0F201075D
:106560006975A76100BF00BF00BF4FF00107A761B9
:1065700000BF00BF4FEA11224FF00007C0F2010731
:106580006A75A76100BF00BF00BF4FF00107A76198
:1065900000BF00BF6FF000014FF00007C0F201071D
:1065A0006975A76100BF00BF00BF4FF00107A76179
:1065B00000BF00BF4FEA11224FF00007C0F20107F1
:1065C0006A75A76100BF00BF00BF4FF00107A76158
:1065D00000BF00BF6FF000014FF00007C0F20107DD
:1065E0006975A76100BF00BF00BF4FF00107A76139
:1065F00000BF00BF4FEA11224FF00007C0F20107B1
:106600006A75A76100BF00BF00BF4FF00107A76117
:1066100000BF00BF6FF000014FF00007C0F201079C
:106620006975A76100BF00BF00BF4FF00107A761F8
:1066300000BF00BF4FEA11224FF00007C0F2010770
:106640006A75A76100BF00BF00BF4FF00107A761D7
:1066500000BF00BF4FEA11424FF00007C0F2010730
:106660006A75A76100BF00BF00BF4FF00107A761B7
:1066700000BF00BF4FEA11624FF00007C0F20107F0
:106680006A75A76100BF00BF00BF4FF00107A76197
:1066900000BF00BF6FF000014FF00007C0F201071C
:1066A0006975A76100BF00BF00BF4FF00107A76178
:1066B00000BF00BF4FEA11224FF00007C0F20107F0
:1066C0006A75A76100BF00BF00BF4FF00107A76157
:1066D00000BF00BF4FEA11424FF00007C0F20107B0
:1066E0006A75A76100BF00BF00BF4FF00107A76137
:1066F00000BF00BF4FEA11624FF00007C0F2010770
:106700006A75A76100BF00BF00BF4FF00107A76116
:1067100000BF00BF4FF0A9014FF00007C0F2010712
:106720006975A76100BF00BF00BF4FF00107A761F7
:1067300000BF00BFB0F8C42F4FF00007C0F2010740
:106740006A75A76100BF00BF00BF4FF00107A761D6
:1067500000BF00BF4FEA12214FF00007C0F201074F
:106760006975A76100BF00BF00BF4FF00107A761B7
:1067700000BF00BF40F20407C0F2010740F2100260
:106780006A75A76140F20107C0F20407A76100BF64
:1067900000BF228A12F48062FBD146F62022C0F2AA
:1067A00000022A60228A12F48062FBD04FF00001BE
:1067B000C17240F60009C4F202094FF02007C9F87F
:1067C00018707CF052FF4FF00002A0F83C23FEF757
:1067D00070BE2B291ED145F20023C1F20003151F04
:1067E000FDF4B8A8595D44297DF4B4A805F101056C
:1067F000595D3A297DF4AEA805F10105595D5C2982
:106800007DF4A8A805F10105595D3E297DF4A2A8F3
:10681000FEF7EBBA2C2909D14FF02601A0F83A1364
:106820004FF00002A0F83C23FEF772BA2D2960D188
:1068300045F20023C1F20003151FFDF48BA8595D3A
:1068400044297DF487A805F10105595D3A297DF4B5
:1068500081A805F10105595D5C297DF47BA805F14E
:106860000105595D3E297DF475A84FF00002A0F89E
:106870003C234FF00201A0F83A134FF0440880F097
:10688000D3F84FF0490880F0CFF84FF0520880F06D
:10689000CBF84FF00D0880F0C7F84FF00001C0F8BA
:1068A0004413D0F848134FF00C02B1FBF2F101FB96
:1068B00002F1C0F84C136FF0000645F20041C1F23E
:1068C000000101F5007241F8046B9142FBD16FF0B9
:1068D000000645F20061C1F2000101F5007241F8C5
:1068E000046B9142FBD14FF00101C0F86813F9F736
:1068F000D7BB2E2952D145F20023C1F20003151F48
:10690000FDF428A8595D44297DF424A805F101056A
:10691000595D3A297DF41EA805F10105595D5C29F0
:106920007DF418A805F10105595D3E297DF412A8F2
:106930004FF0520880F078F84FF0440880F074F877
:106940004FF0460880F070F84FF0200880F06CF8A7
:106950004FF00802C0F850234FEA126880F064F844
:106960004FEA124808F0FF0880F05EF84FEA12285C
:1069700008F0FF0880F058F802F0FF0880F054F8A3
:106980004FF00D0880F050F84FF02F01A0F83A13A7
:106990004FF00002A0F83C23F9F782BB2F2962D107
:1069A00041F20046C4F20106376817F00F083BD0E9
:1069B0003768776890F86D7007F1010780F86D709F
:1069C0004FF0530880F030F84FF0450880F02CF875
:1069D0004FF04B0880F028F84FF0200880F024F8A2
:1069E000D0F86C934FEA196880F01EF84FEA194806
:1069F00008F0FF0880F018F84FEA192808F0FF089F
:106A000080F012F809F0FF0880F00EF84FF00D0842
:106A100080F00AF84FF02E01A0F83A134FF0000270
:106A2000A0F83C23F9F73CBB45F20023C1F2000378
:106A3000151FFCF48FAF595D44297CF48BAF05F131
:106A40000105595D3A297CF485AF05F10105595DD1
:106A50005C297CF47FAF05F10105595D3E297CF48A
:106A600079AFFAF7AFBA302952D145F20023C1F21B
:106A70000003151FFCF46EAF595D44297CF46AAF26
:106A800005F10105595D3A297CF464AF05F1010572
:106A9000595D5C297CF45EAF05F10105595D3E2925
:106AA0007CF458AF4FF052087FF0BEFF4FF044081F
:106AB0007FF0BAFF4FF046087FF0B6FF4FF0200896
:106AC0007FF0B2FF4FF00802C0F850234FEA12687F
:106AD0007FF0AAFF4FEA124808F0FF087FF0A4FFFA
:106AE0004FEA122808F0FF087FF09EFF02F0FF082F
:106AF0007FF09AFF4FF00D087FF096FF4FF03101C5
:106B0000A0F83A134FF00002A0F83C23F9F7C8BAF6
:106B1000312962D141F20046C4F20106376817F00C
:106B20000F083BD03768776890F86D7007F1010760
:106B300080F86D704FF053087FF076FF4FF04508F6
:106B40007FF072FF4FF04B087FF06EFF4FF0200890
:106B50007FF06AFFD0F86C934FEA19687FF064FF0A
:106B60004FEA194808F0FF087FF05EFF4FEA192846
:106B700008F0FF087FF058FF09F0FF087FF054FF8E
:106B80004FF00D087FF050FF4FF03001A0F83A139E
:106B90004FF00002A0F83C23F9F782BA45F2002337
:106BA000C1F20003151FFCF4D5AE595D44297CF4F5
:106BB000D1AE05F10105595D3A297CF4CBAE05F162
:106BC0000105595D5C297CF4C5AE05F10105595DEF
:106BD0003E297CF4BFAEFEF7A4BB322940F0EC8026
:106BE00045F20023C1F20003151F21D3595D44294A
:106BF0001ED105F10105595D3A2919D105F10105AB
:106C0000595D5C2914D105F10105595D3E290FD16B
:106C10004FF00002A0F83C234FF40051C0F8681375
:106C200090F8391321F0010180F83913F9F7F4B91C
:106C300045F20025C1F2000515F8011B43297CF43B
:106C400089AE15F8011B6F297CF484AE15F8011B81
:106C50006D297CF47FAE15F8011B6D297CF47AAEAA
:106C600015F8011B61297CF475AE15F8011B6E291E
:106C70007CF470AE15F8011B64297CF46BAE15F83A
:106C8000011B20297CF466AE15F8011B46297CF413
:106C900061AE15F8011B61297CF45CAE15F8011B8F
:106CA00069297CF457AE15F8011B6C297CF452AEAF
:106CB00015F8011B65297CF44DAE15F8011B6429FC
:106CC0007CF448AE4FF00002A0F83C234FF04F0890
:106CD0007FF0AAFE4FF050087FF0A6FE4FF0570855
:106CE0007FF0A2FE4FF020087FF09EFEB0F81C6DF2
:106CF0004FEA961606F141087FF096FEB0F81C6D3B
:106D000006F03F0606F101064FF000080A3E08F1C2
:106D10000108FBD206F10A06A8F1010808F13008C3
:106D20007FF082FE06F130087FF07EFE41F2000423
:106D3000C2F2000494F892807AF028F97FF074FE91
:106D400094F894807AF022F97FF06EFE94F89680A1
:106D50007AF01CF97FF068FE94F898807AF016F9C2
:106D60007FF062FE94F89A807AF010F97FF05CFE72
:106D70004FF02E087FF058FE4FF046087FF054FE8B
:106D80004FF05A087FF050FE4FF050087FF04CFE55
:106D90004FF00D087FF048FE4FF03301A0F83A1392
:106DA00090F8391341F0010180F839134FF4804114
:106DB000C0F86813F9F730B933297BD145F20023C5
:106DC000C1F20003151FFCF4C5AD595D44297CF4E4
:106DD000C1AD05F10105595D3A297CF4BBAD05F162
:106DE0000105595D5C297CF4B5AD05F10105595DDE
:106DF0003E297CF4AFAD4FF057087FF015FE4FF001
:106E000052087FF011FE4FF046087FF00DFE4FF064
:106E100020087FF009FE4FF488324FEA12687FF0B5
:106E200003FE4FEA124808F0FF087FF0FDFD4FEA2D
:106E3000122808F0FF087FF0F7FD904608F0FF08E1
:106E40007FF0F2FD4FF00D087FF0EEFD41F2000300
:106E5000C2F2000303F58056C28B002AFCD103F571
:106E6000806913F8018B7FF0DFFD4B45F9D1B34208
:106E7000F2D340F20003C2F2010303F58036C28B65
:106E8000002AFCD103F5806913F8018B7FF0CCFD5B
:106E90004B45F9D1B342F2D34FF00D087FF0C4FD5A
:106EA0004FF03401A0F83A134FF00002A0F83C2351
:106EB000F9F7F6B8342940F09C8045F20023C1F27E
:106EC0000003151FFCF446AD595D44297CF442AD26
:106ED00005F10105595D3A297CF43CAD05F1010548
:106EE000595D5C297CF436AD05F10105595D3E29FB
:106EF0007CF430AD4FF00002A0F83C2390F8A312D0
:106F000011F0010105D14FF0010180F8A312F9F74A
:106F1000C7B84FF0000180F8A3124FF043087FF08C
:106F200083FD4FF04C087FF07FFD4FF046087FF067
:106F30007BFD4FF020087FF077FDB0F81C6D4FEA25
:106F4000961606F141087FF06FFDB0F81C6D06F053
:106F50003F0606F101064FF000080A3E08F101085D
:106F6000FBD206F10A06A8F1010808F130087FF00B
:106F70005BFD06F130087FF057FD41F20004C2F2DC
:106F8000000494F892807AF001F87FF04DFD94F8B7
:106F9000948079F0FBFF7FF047FD94F8968079F0BC
:106FA000F5FF7FF041FD94F8988079F0EFFF7FF0D6
:106FB0003BFD94F89A8079F0E9FF7FF035FD4FF0C2
:106FC0002E087FF031FD4FF046087FF02DFD4FF089
:106FD0005A087FF029FD4FF050087FF025FD4FF053
:106FE0000D087FF021FD4FF03501A0F83A13F9F7B5
:106FF00057B8352960D145F20023C1F20003151FAF
:10700000FCF4A8AC595D44297CF4A4AC05F101055D
:10701000595D3A297CF49EAC05F10105595D5C2966
:107020007CF498AC05F10105595D3E297CF492ACE5
:107030004FF00002A0F83C234FF00201A0F83A13F1
:107040004FF044087FF0F0FC4FF049087FF0ECFC73
:107050004FF052087FF0E8FC4FF00D087FF0E4FCA1
:107060004FF00001C0F84413D0F848134FF00C0261
:10707000B1FBF2F101FB02F1C0F84C136FF0000616
:1070800045F20041C1F2000101F5007241F8046BC4
:107090009142FBD16FF0000645F20061C1F20001A0
:1070A00001F5007241F8046B9142FBD14FF00801E9
:1070B000C0F86813F8F7F4BF362940F08D8045F228
:1070C0000023C1F20003151FFCF444AC595D4429B0
:1070D0007CF440AC05F10105595D3A297CF43AACE9
:1070E00005F10105595D5C297CF434AC05F101051D
:1070F000595D3E297CF42EAC4FF00002A0F83C23F1
:107100004FF044087FF090FC4FF04C087FF08CFC6F
:107110004FF046087FF088FC4FF020087FF084FC99
:10712000B0F81C6D4FEA961606F141087FF07CFC22
:10713000B0F81C6D06F03F0606F101064FF000089E
:107140000A3E08F10108FBD206F10A06A8F101087F
:1071500008F130087FF068FC06F130087FF064FC2D
:1071600041F20004C2F2000494F8928079F00EFF1C
:107170007FF05AFC94F8948079F008FF7FF054FC7B
:1071800094F8968079F002FF7FF04EFC94F8988096
:1071900079F0FCFE7FF048FC94F89A8079F0F6FED6
:1071A0007FF042FC4FF02E087FF03EFC4FF0460887
:1071B0007FF03AFC4FF05A087FF036FC4FF0500851
:1071C0007FF032FC4FF00D087FF02EFC4FF03701BE
:1071D000A0F83A13F8F764BF372921D145F200230C
:1071E000C1F20003151FFCF4B5AB595D44297CF4D2
:1071F000B1AB05F10105595D3A297CF4ABAB05F162
:107200000105595D5C297CF4A5AB05F10105595DCB
:107210003E297CF49FAB4FF00002A0F83C2355E5DB
:1072200038295CD145F20023C1F20003151FFCF49C
:1072300091AB595D44297CF48DAB05F10105595D95
:107240003A297CF487AB05F10105595D5C297CF492
:1072500081AB05F10105595D3E297CF47BAB4FF014
:1072600052087FF0E1FB4FF044087FF0DDFB4FF068
:1072700046087FF0D9FB4FF020087FF0D5FB4FF494
:107280000062C0F85023C0F85C234FEA12687FF018
:10729000CBFB4FEA124808F0FF087FF0C5FB4FEA2E
:1072A000122808F0FF087FF0BFFB02F0FF087FF014
:1072B000BBFB4FF00D087FF0B7FB4FF03901A0F892
:1072C0003A134FF00002A0F83C234FF40061C0F8DD
:1072D00068134FF0000180F8BD10F8F79DBE392902
:1072E00040F0CC8041F20046C4F20106376817F046
:1072F0000F080ED03768776890F86D7007F10107B6
:1073000080F86D70D0F85C63A6F50066C0F85C6329
:107310002AE045F20023C1F20003151FFCF41AAB6A
:10732000595D44297CF416AB05F10105595D3A29F4
:107330007CF410AB05F10105595D5C297CF40AABC6
:1073400005F10105595D3E297CF404ABD0F85C637E
:1073500040F24041B6FBF1F180F8BD10D0F85C631B
:107360004FF488318E4233D24FF053087FF05CFBEC
:107370004FF045087FF058FB4FF04B087FF054FB6F
:107380004FF020087FF050FBD0F85C634FEA16689E
:107390007FF04AFB4FEA164808F0FF087FF044FBF5
:1073A0004FEA162808F0FF087FF03EFB06F0FF08C2
:1073B0007FF03AFB4FF00D087FF036FB4FF03D01B8
:1073C000A0F83A134FF00002A0F83C23F8F768BE8B
:1073D00078F020FE4FF0010180F847114FF4004192
:1073E000A0F8FA14A0F8FA15A0F8FA16A0F8FA17FF
:1073F000A0F8FA18A0F8FA19A0F8FA1AA0F8FA1BDF
:1074000090F8FC1341764FF0000180F8FC1384F0F3
:107410006CFA4FF0010180F8FC1384F066FA4FF02B
:10742000020180F8FC1384F060FA4FF0030180F849
:10743000FC1384F05AFA4FF0040180F8FC1384F036
:1074400054FA4FF0050180F8FC1384F04EFA4FF027
:10745000060180F8FC1384F048FA4FF0070180F829
:10746000FC1384F042FA417E80F8FC13B0F86E10F1
:1074700041F00101A0F86E10F9F786BF3A2905D155
:107480004FF00002A0F83C23F8F70ABE3B295CD17C
:1074900045F20023C1F20003151FFCF45BAA595DFD
:1074A00044297CF457AA05F10105595D3A297CF479
:1074B00051AA05F10105595D5C297CF44BAA05F13F
:1074C0000105595D3E297CF445AA4FF052087FF032
:1074D000ABFA4FF044087FF0A7FA4FF046087FF070
:1074E000A3FA4FF020087FF09FFA4FF40062C0F833
:1074F0005023C0F85C234FEA12687FF095FA4FEAF8
:10750000124808F0FF087FF08FFA4FEA122808F0BF
:10751000FF087FF089FA02F0FF087FF085FA4FF04C
:107520000D087FF081FA4FF03C01A0F83A134FF0BC
:107530000002A0F83C234FF40061C0F868134FF03C
:10754000000180F8BD10F8F767BD3C2940F0DD80F0
:1075500041F20046C4F20106376817F00F080ED05A
:107560003768776890F86D7007F1010780F86D70E3
:10757000D0F85C63A6F50066C0F85C632AE045F2CB
:107580000023C1F20003151FFCF4E4A9595D44294E
:107590007CF4E0A905F10105595D3A297CF4DAA9EA
:1075A00005F10105595D5C297CF4D4A905F10105BB
:1075B000595D3E297CF4CEA9D0F85C6340F240418D
:1075C000B6FBF1F180F8BD10D0F85C634FF4883160
:1075D0008E4233D24FF053087FF026FA4FF0450821
:1075E0007FF022FA4FF04B087FF01EFA4FF0200890
:1075F0007FF01AFAD0F85C634FEA16687FF014FA4D
:107600004FEA164808F0FF087FF00EFA4FEA1628F6
:1076100008F0FF087FF008FA06F0FF087FF004FA90
:107620004FF00D087FF000FA4FF03E01A0F83A133A
:107630004FF00002A0F83C23F8F732BD78F0EAFCE6
:107640004FF0010180F847114FF40041A0F8FA14FF
:10765000A0F8FA15A0F8FA16A0F8FA17A0F8FA1888
:10766000A0F8FA19A0F8FA1AA0F8FA1B90F8FC137F
:1076700041764FF0000180F8FC1384F036F94FF0AA
:10768000010180F8FC1384F030F94FF0020180F81A
:10769000FC1384F02AF94FF0030180F8FC1384F006
:1076A00024F94FF0040180F8FC1384F01EF94FF028
:1076B000050180F8FC1384F018F94FF0060180F8FA
:1076C000FC1384F012F94FF0070180F8FC1384F0EA
:1076D0000CF9417E80F8FC13B0F8421081824FF023
:1076E000010780F85E707BF01DF94FF0000780F80D
:1076F0005E70B0F8421001F1010140F2FF3701EA7B
:107700000701A0F84210FDF7D4BE3D2959D145F23A
:107710000023C1F20003151FFCF41CA9595D442984
:107720007CF418A905F10105595D3A297CF412A9E8
:1077300005F10105595D5C297CF40CA905F10105F1
:10774000595D3E297CF406A94FF40063C0F850331C
:10775000D0F85C131944C0F85C134FF052087FF066
:1077600063F94FF044087FF05FF94FF046087FF06F
:107770005BF94FF020087FF057F9D0F850234FEA1B
:1077800012687FF051F94FEA124808F0FF087FF0C5
:107790004BF94FEA122808F0FF087FF045F902F094
:1077A000FF087FF041F94FF00D087FF03DF94FF0F1
:1077B0003901A0F83A134FF00002A0F83C23F8F783
:1077C0006FBC3E2959D145F20023C1F20003151FB9
:1077D000FCF4C0A8595D44297CF4BCA805F101055E
:1077E000595D3A297CF4B6A805F10105595D5C297B
:1077F0007CF4B0A805F10105595D3E297CF4AAA8E6
:107800004FF40063C0F85033D0F85C131944C0F84B
:107810005C134FF052087FF007F94FF044087FF0F7
:1078200003F94FF046087FF0FFF84FF020087FF093
:10783000FBF8D0F850234FEA12687FF0F5F84FEAD2
:10784000124808F0FF087FF0EFF84FEA122808F01E
:10785000FF087FF0E9F802F0FF087FF0E5F84FF04D
:107860000D087FF0E1F84FF03C01A0F83A134FF01B
:107870000002A0F83C23F8F713BC3F2940F0F58044
:1078800045F20023C1F20003151F2CD3595D442992
:1078900029D105F10105595D3A2924D105F10105E8
:1078A000595D5C291FD105F10105595D3E291AD1A9
:1078B0004FF00002A0F83C2390F8331111F00102C0
:1078C00005D011F0020221F0E38120F015BE4FF443
:1078D0008031C0F8681390F8391321F0010180F865
:1078E0003913F8F799BB45F20025C1F2000515F8E8
:1078F000011B43297CF42EA815F8011B6F297CF489
:1079000029A815F8011B6D297CF424A815F8011B82
:107910006D297CF41FA815F8011B61297CF41AA8B5
:1079200015F8011B6E297CF415A815F8011B6429B4
:107930007CF410A815F8011B20297CF40BA815F87D
:10794000011B46297CF406A815F8011B61297CF46B
:1079500001A815F8011B69297BF4FCAF15F8011B80
:107960006C297BF4F7AF15F8011B65297BF4F2AFA6
:1079700015F8011B64297BF4EDAF4FF00002A0F86D
:107980003C234FF04F087FF04FF84FF050087FF046
:107990004BF84FF057087FF047F84FF020087FF082
:1079A00043F8468A4FEA961606F141087FF03CF804
:1079B000468A06F03F0606F101064FF000080A3E2F
:1079C00008F10108FBD206F10A06A8F1010808F146
:1079D00030087FF029F806F130087FF025F841F2F1
:1079E0000004C2F2000494F8928079F0CFFA7FF09C
:1079F0001BF894F8948079F0C9FA7FF015F894F8A0
:107A0000968079F0C3FA7FF00FF894F8988079F0B7
:107A1000BDFA7FF009F894F89A8079F0B7FA7FF010
:107A200003F84FF02E087EF0FFFF4FF046087EF07F
:107A3000FBFF4FF05A087EF0F7FF4FF050087EF042
:107A4000F3FF4FF00D087EF0EFFF4FF04001A0F87C
:107A50003A1390F8391341F0010180F839134FF4CB
:107A60000031C0F86813F8F7D7BA40297BD145F246
:107A70000023C1F20003151FFBF46CAF595D4429CC
:107A80007BF468AF05F10105595D3A297BF462AFDB
:107A900005F10105595D5C297BF45CAF05F1010539
:107AA000595D3E297BF456AF4FF057087EF0BCFF7E
:107AB0004FF052087EF0B8FF4FF046087EF0B4FF5A
:107AC0004FF020087EF0B0FF4FF488324FEA126882
:107AD0007EF0AAFF4FEA124808F0FF087EF0A4FFEC
:107AE0004FEA122808F0FF087EF09EFF904608F04B
:107AF000FF087EF099FF4FF00D087EF095FF41F2F0
:107B00000003C2F2000303F58056C28B002AFCD1A9
:107B100003F5806913F8018B7EF086FF4B45F9D1A0
:107B2000B342F2D340F20003C2F2010303F5803600
:107B3000C28B002AFCD103F5806913F8018B7EF01B
:107B400073FF4B45F9D1B342F2D34FF00D087EF0ED
:107B50006BFF4FF04101A0F83A134FF00002A0F87C
:107B60003C23F8F79DBA412940F09A8045F2002362
:107B7000C1F20003151FFBF4EDAE595D44297BF4FF
:107B8000E9AE05F10105595D3A297BF4E3AE05F153
:107B90000105595D5C297BF4DDAE05F10105595DF8
:107BA0003E297BF4D7AE4FF00002A0F83C2390F8BA
:107BB000A31211F0010105D14FF0010180F8A312C9
:107BC000F8F76EBA4FF0000180F8A3124FF04308A7
:107BD0007EF02AFF4FF04C087EF026FF4FF046085B
:107BE0007EF022FF4FF020087EF01EFF468A4FEA0B
:107BF000961606F141087EF017FF468A06F03F060A
:107C000006F101064FF000080A3E08F10108FBD218
:107C100006F10A06A8F1010808F130087EF004FF19
:107C200006F130087EF000FF41F20004C2F20004C9
:107C300094F8928079F0AAF97EF0F6FE94F8948098
:107C400079F0A4F97EF0F0FE94F8968079F09EF930
:107C50007EF0EAFE94F8988079F098F97EF0E4FEE0
:107C600094F89A8079F092F97EF0DEFE4FF02E08BB
:107C70007EF0DAFE4FF046087EF0D6FE4FF05A084E
:107C80007EF0D2FE4FF050087EF0CEFE4FF00D0891
:107C90007EF0CAFE4FF04201A0F83A13F8F700BA9E
:107CA000422940F00B8145F20023C1F20003151F69
:107CB000FBF450AE595D44297BF44CAE05F101054F
:107CC000595D3A297BF446AE05F10105595D5C2901
:107CD0007BF440AE05F10105595D3E297BF43AAED7
:107CE000418A01F10101418211F4806240F09680E5
:107CF00079F096F94FF0005041F20004C2F200040E
:107D00002188A92916D0A82914D0A72912D0A629DC
:107D100010D0A5290ED0A4290CD0A3290AD0A229BD
:107D200008D0A12906D0AA2904D0AB2902D0AC29B9
:107D300000D0D5E74FF04F087EF076FE4FF05008A8
:107D40007EF072FE4FF052087EF06EFE4FF020087B
:107D50007EF06AFE468A4FEA961606F141087EF0EA
:107D600063FE468A06F03F0606F101064FF0000862
:107D70000A3E08F10108FBD206F10A06A8F1010843
:107D800008F130087EF050FE06F130087EF04CFE1F
:107D900041F20004C2F2000494F8928079F0F6F8FF
:107DA0007EF042FE94F8948079F0F0F87EF03CFE8C
:107DB00094F8968079F0EAF87EF036FE94F8988090
:107DC00079F0E4F87EF030FE94F89A8079F0DEF8ED
:107DD0007EF02AFE4FF02E087EF026FE4FF0460879
:107DE0007EF022FE4FF05A087EF01EFE4FF0500843
:107DF0007EF01AFE4FF00D087EF016FE4FF03F01A8
:107E0000A0F83A134FF00002A0F83C2390F8391381
:107E100041F0010180F83913F8F742B94FF0000240
:107E2000A0F83C23B0F81C1D418281824FF008016C
:107E3000C0F8681379F0F4F84FF000504FF00201E9
:107E4000A0F83A134FF044087EF0EEFD4FF04908D9
:107E50007EF0EAFD4FF052087EF0E6FD4FF00D088F
:107E60007EF0E2FD4FF00001C0F84413D0F8481353
:107E70004FF00C02B1FBF2F101FB02F1C0F84C1320
:107E80006FF0000645F20041C1F2000101F50072F9
:107E900041F8046B9142FBD16FF0000645F200619E
:107EA000C1F2000101F5007241F8046B9142FBD16F
:107EB0004FF00801C0F86813F8F7F2B8432940F012
:107EC0008B8045F20023C1F20003151FFBF442AD85
:107ED000595D44297BF43EAD05F10105595D3A2910
:107EE0007BF438AD05F10105595D5C297BF432ADB9
:107EF00005F10105595D3E297BF42CAD4FF00002E0
:107F0000A0F83C234FF044087EF08EFD4FF04C0863
:107F10007EF08AFD4FF046087EF086FD4FF0200887
:107F20007EF082FD468A4FEA961606F141087EF001
:107F30007BFD468A06F03F0606F101064FF0000879
:107F40000A3E08F10108FBD206F10A06A8F1010871
:107F500008F130087EF068FD06F130087EF064FD1F
:107F600041F20004C2F2000494F8928079F00EF815
:107F70007EF05AFD94F8948079F008F87EF054FD74
:107F800094F8968079F002F87EF04EFD94F898808F
:107F900078F0FCFF7EF048FD94F89A8078F0F6FFC8
:107FA0007EF042FD4FF02E087EF03EFD4FF0460879
:107FB0007EF03AFD4FF05A087EF036FD4FF0500843
:107FC0007EF032FD4FF00D087EF02EFD4FF04401A3
:107FD000A0F83A13F8F764B8442921D145F20023F8
:107FE000C1F20003151FFBF4B5AC595D44297BF4C5
:107FF000B1AC05F10105595D3A297BF4ABAC05F153
:108000000105595D5C297BF4A5AC05F10105595DBD
:108010003E297BF49FAC4FF00002A0F83C23B0E473
:10802000452921D145F20023C1F20003151FFBF4BD
:1080300091AC595D44297BF48DAC05F10105595D86
:108040003A297BF487AC05F10105595D5C297BF485
:1080500081AC05F10105595D3E297BF47BAC4FF005
:108060000002A0F83C233BE6462960D145F20023FC
:10807000C1F20003151FFBF46DAC595D44297BF47C
:1080800069AC05F10105595D3A297BF463AC05F152
:108090000105595D5C297BF45DAC05F10105595D75
:1080A0003E297BF457AC4FF00001C0F848134FF065
:1080B0000002A0F83C234FF04701A0F83A134FF01C
:1080C00044087EF0B1FC4FF049087EF0ADFC4FF063
:1080D00052087EF0A9FC4FF00D087EF0A5FC4FF091
:1080E0000001C0F84413D0F848134FF00C02B1FB64
:1080F000F2F101FB02F1C0F84C136FF0000645F2FB
:108100000041C1F2000101F5007241F8046B914297
:10811000FBD16FF0000645F20061C1F2000101F5EC
:10812000007241F8046B9142FBD1F7F7B9BF4729C0
:1081300040F0E78045F20023C1F20003151F4AD347
:10814000595D442920D105F10105595D3A291BD11A
:1081500005F10105595D5C2916D105F10105595D4F
:108160003E2911D141F20046C4F20106376817F0EA
:108170000F0808D03768776890F86D7007F101072D
:1081800080F86D7093E73BE0151F24D3595D2E29CD
:1081900021D105F10105595D48291CD105F10105E1
:1081A000595D452917D105F10105595D582912D1AD
:1081B000D0F8441301F10101C0F8441345F2004620
:1081C000C1F2000606F1C0073178FF2909D006F197
:1081D0001006BE42F8D14FF00002A0F83C23F7F79A
:1081E0005FBF4FF00005595D06F8011B05F1010561
:1081F0009542F8D14FF00002A0F83C23F7F750BFAA
:1082000090F8391321F0010180F8391345F200424A
:10821000C1F200021178FF2969D04FF04801A0F89F
:108220003A134FF00001A0F83E1345F20042C1F2AC
:10823000000202F1C004B0F83E334FEA03131A44BF
:10824000A24200F0C0811178FF2900F0BC814FF0FC
:10825000010912F809102E2902D009F10109F8E7E5
:1082600009F1010912F80910482939D109F1010968
:1082700012F80910452933D109F1010912F8091042
:1082800058292DD109F1060980F85F904FF0440874
:108290007EF0CAFB4FF049087EF0C6FB4FF0520853
:1082A0007EF0C2FB4FF020087EF0BEFB12F8018B7F
:1082B000B8F1FF0F04D07EF0B7FB12F00F01F5D13B
:1082C0004FF00D087EF0B0FBB0F83E1301F1010154
:1082D000A0F83E134FF00002A0F83C23F7F7E0BEF1
:1082E000B0F83E1301F10101A0F83E139DE74FF4F1
:1082F0000021C0F868134FF00002A0F83C23F7F704
:108300008BBE482940F0358241F20046C4F2010696
:10831000376817F00F080ED03768776890F86D70DF
:1083200007F1010780F86D70D0F83E63A6F10106F1
:10833000C0F83E63DCE045F20023C1F20003B2F175
:108340000905C1F04782595D2E2941F0438205F1AC
:108350000105595D482940F0308105F10105595D5D
:10836000452940F02A8105F10105595D582940F061
:10837000248145F20046C1F2000606F1C00790F8DC
:108380005F90A2EB09053178FF2900F0168113F800
:108390000580884540F00C8105F101057178FF29C1
:1083A00000F0908013F80580884540F0018105F1C8
:1083B0000105B178FF2900F0858013F80580884514
:1083C00040F0F68005F10105F178FF297AD013F825
:1083D0000580884540F0EC8005F101053179FF29E1
:1083E00070D013F80580884540F0E28005F1010562
:1083F0007179FF2966D013F80580884540F0D88050
:1084000005F10105B179FF295CD013F80580884595
:1084100040F0CE8005F10105F179FF2952D013F823
:108420000580884540F0C48005F10105317AFF29B7
:1084300048D013F80580884540F0BA8005F1010561
:10844000717AFF293ED013F80580884540F0B0804E
:1084500005F10105B17AFF2934D013F8058088456C
:1084600040F0A68005F10105F17AFF292AD013F822
:108470000580884540F09C8005F10105317BFF298E
:1084800020D013F80580884540F0928005F1010561
:10849000717BFF2916D013F80580884540F088804D
:1084A00005F10105B17BFF290CD013F80580884543
:1084B0007ED105F10105F17BFF2903D013F805807A
:1084C000884575D106F50076A2F10405595943F6A1
:1084D000442AC3F65C6A51456FD04FF0A90106F8F3
:1084E000041B595D06F8011B05F101059542F8D101
:1084F00045F20042C1F2000202F1C004B0F83E337E
:108500004FEA03131A44A2425DD01178FF295AD0D2
:108510004FF0010912F809102E2902D009F10109C2
:10852000F8E709F1010912F80910482939D109F1D0
:10853000010912F80910452933D109F1010912F88E
:10854000091058292DD109F1060980F85F904FF0E4
:1085500044087EF069FA4FF049087EF065FA4FF062
:1085600052087EF061FA4FF020087EF05DFA12F8B2
:10857000018BB8F1FF0F04D07EF056FA12F00F0114
:10858000F5D14FF00D087EF04FFAB0F83E1301F12F
:108590000101A0F83E134FF00002A0F83C23F7F7CA
:1085A0007FBDB0F83E1301F10101A0F83E139FE733
:1085B00006F11006BE427FF4E2AE4FF00002A0F8D2
:1085C0003C23F7F76DBD4FF04901A0F83A134FF087
:1085D0000002A0F83C23F7F763BD45F20063C1F247
:1085E000000303F1C0041978A92904D003F1100392
:1085F000A34231D2F7E7A3F5007211784629F5D1ED
:1086000051785F29F2D19778312FEFD3342FEDD203
:10861000D1785F29EAD111793029E7D33A29E5D217
:1086200051793029E2D33A29E0D291793029DDD34A
:108630003A29DBD2D1793029D8D33A29D6D290F849
:108640007452A7F131074FF0010606FA07F645EA22
:10865000060580F87452C9E790F87452002D3FF473
:1086600046AE4FF48011C0F868134FF00002A0F836
:108670003C234EF60022C2F200024FF0000122F825
:10868000021B22F8021B22F8021B22F8021B22F80E
:10869000021B22F8021B22F8021B22F8021B4FF6D3
:1086A000FF7122F8021B4FF0000122F8021B4FF06D
:1086B000000122F8021B4FF0000122F8021B46F2D3
:1086C0000042C4F20202D2F8A01041F00101C2F847
:1086D000A010F7F7A1BCD0F8481301F10101D0F8C0
:1086E0004423914202D2C0F8481376E7468AA0F8A4
:1086F0001C6D868278F094FC4FF043087EF094F96C
:108700004FF044087EF090F94FF020087EF08CF98D
:108710004FF02E087EF088F94FF02E087EF084F995
:108720004FF00D087EF080F94FF01701A0F83A13D2
:1087300090F8391341F0010180F8391390F856137D
:10874000A1F1010180F8561340F20025C2F20005A4
:108750004FEA81084544D5F80080C0F848834FF0BF
:108760000002A0F83C234FF00101C0F86813F7F7AE
:1087700097BC492908D14FF04801A0F83A134FF0AF
:108780000002A0F83C2328E74A295ED145F20023E5
:10879000C1F20003151FFBF4DDA8595D44297BF4E9
:1087A000D9A805F10105595D3A297BF4D3A805F153
:1087B0000105595D5C297BF4CDA805F10105595DE2
:1087C0003E297BF4C7A84FF052087EF02DF94FF0F8
:1087D00044087EF029F94FF046087EF025F94FF065
:1087E00020087EF021F94FF40062D0F8F833D0F879
:1087F0005843A4EB0304B4F5006F38BF2246C0F819
:108800005023C0F8C0204FEA12687EF00DF94FEAFD
:10881000124808F0FF087EF007F94FEA122808F026
:10882000FF087EF001F902F0FF087EF0FDF84FF03E
:108830000D087EF0F9F84FF04B01A0F83A134FF015
:108840000002A0F83C23F7F72BBC4B2940F0A38093
:1088500041F20046C4F20106376817F00F0842D013
:108860003768776890F86D7007F1010780F86D70D0
:10887000D0F8F823D0F858339A4280F04C824FF069
:1088800053087EF0D1F84FF045087EF0CDF84FF058
:108890004B087EF0C9F84FF020087EF0C5F8D0F8FC
:1088A000F8234FEA12687EF0BFF84FEA124808F04A
:1088B000FF087EF0B9F84FEA122808F0FF087EF0B2
:1088C000B3F802F0FF087EF0AFF84FF00D087EF02D
:1088D000ABF84FF04A01A0F83A134FF00002A0F8AD
:1088E0003C23F7F7DDBB45F20023C1F20003151F5F
:1088F000FBF430A8595D44297BF42CA805F101054F
:10890000595D3A297BF426A805F10105595D5C29DA
:108910007BF420A805F10105595D3E297BF41AA8D6
:10892000D0F8F823D0F858339A4280F0F4814FF011
:1089300053087EF079F84FF045087EF075F84FF057
:108940004B087EF071F84FF020087EF06DF8D0F8FB
:10895000F8234FEA12687EF067F84FEA124808F0F1
:10896000FF087EF061F84FEA122808F0FF087EF059
:108970005BF802F0FF087EF057F84FF00D087EF02C
:1089800053F84FF04C01A0F83A134FF00002A0F852
:108990003C23F7F785BB4C295ED145F20023C1F299
:1089A0000003151FFAF4D6AF595D44297AF4D2AF0B
:1089B00005F10105595D3A297AF4CCAF05F10105BD
:1089C000595D5C297AF4C6AF05F10105595D3E2970
:1089D0007AF4C0AF4FF052087EF026F84FF044080A
:1089E0007EF022F84FF046087EF01EF84FF0200887
:1089F0007EF01AF84FF40062D0F8F833D0F85843FC
:108A0000A4EB0304B4F5006F38BF2246C0F850232E
:108A1000C0F8C0204FEA12687EF006F84FEA12480C
:108A200008F0FF087EF000F84FEA122808F0FF086F
:108A30007DF0FAFF02F0FF087DF0F6FF4FF00D0821
:108A40007DF0F2FF4FF04D01A0F83A134FF0000215
:108A5000A0F83C23F7F724BB4D2940F0F88441F2FD
:108A60000046C4F20106376817F00F0842D0376895
:108A7000776890F86D7007F1010780F86D70D0F895
:108A8000F823D0F858339A4280F045814FF05308CC
:108A90007DF0CAFF4FF045087DF0C6FF4FF04B0850
:108AA0007DF0C2FF4FF020087DF0BEFFD0F8F82324
:108AB0004FEA12687DF0B8FF4FEA124808F0FF084D
:108AC0007DF0B2FF4FEA122808F0FF087DF0ACFFFE
:108AD00002F0FF087DF0A8FF4FF00D087DF0A4FF25
:108AE0004FF04C01A0F83A134FF00002A0F83C23DD
:108AF000F7F7D6BA45F20023C1F20003151FFAF4C6
:108B000029AF595D44297AF425AF05F10105595D76
:108B10003A297AF41FAF05F10105595D5C297AF411
:108B200019AF05F10105595D3E297AF413AF47F2FB
:108B30000002C2F2000202F5006402F5006352F87E
:108B4000045B53F8046BB5427FF492AEA242F6D3B5
:108B500047F20002C2F2000202F50064D0F8DC53D2
:108B600049F20001C2F20001C0F8DC538D4280F0EE
:108B7000D68011783A2904D002F10102A242F8D33A
:108B8000BDE0117A312900F0C68092F80180B8F179
:108B9000410F2CBFA8F13708A8F1300808F00F08E2
:108BA0004FEA0818917841292CBF3739303901F044
:108BB0000F0148EA01084FEA480808F10D089044FF
:108BC000A04580F09C80117A302903D04246A2F162
:108BD0000102C5E702F101024FF0000712F8016B34
:108BE000412E2CBF373E303E06F00F064FEA0616E8
:108BF00012F8011B41292CBF3739303901F00F0120
:108C000046EA0106374412F8013B412B2CBF373BA3
:108C1000303B03F00F034FEA031312F8011B412905
:108C20002CBF3739303901F00F0143EA01031F44EB
:108C300012F8013B412B2CBF373B303B03F00F03B5
:108C40004FEA031312F8011B41292CBF3739303981
:108C500001F00F0143EA01031F4412F8013B412BCD
:108C60002CBF373B303B03F00F034FEA031312F8DE
:108C7000011B41292CBF3739303901F00F0143EA7C
:108C800001031F44002E19D012F8013B412B2CBFC9
:108C9000373B303B03F00F034FEA031312F8011B7D
:108CA00041292CBF3739303901F00F0143EA010364
:108CB00005F8013B1F44A6F10106E3E712F8018B1A
:108CC000B8F1410F2CBFA8F13708A8F1300808F01F
:108CD0000F084FEA081812F8011B41292CBF373939
:108CE000303901F00F0148EA01086FEA070707F180
:108CF000010707F0FF0747453FF432AFB8E547F2F9
:108D00000001C2F20001A2EB0102D0F8F8939144F5
:108D1000C0F8F893ACE54FF0010180F8A71247F2D4
:108D20000001C2F20001A2EB0102D0F8F8939144D5
:108D3000C0F8F89390F8741211F0010200F043812A
:108D400072B64FF0005043F60042C4F20202D0F86F
:108D5000A063002E34D1D16811F48031FBD140F2F0
:108D60002311C4F26751516000BF00BF00BF00BFB4
:108D7000D16811F48031FBD148F6AB11CCF6EF513C
:108D8000516000BF00BF00BF00BFD16811F4803147
:108D9000FBD148F20001C0F200011161116941F4F8
:108DA0008031116100BF00BF00BF00BFD16811F466
:108DB0008031FBD14FF00006C0F61006C0F8A0636A
:108DC00048F20005C2F2000505F5805740F2012186
:108DD000C0F20001116100BF00BF55F8041B46F846
:108DE000041B00BF00BF00BF00BFD16811F4803179
:108DF000FBD1BD42F1D3C0F8A063116921F001019C
:108E0000116162B64FF00001C0F61E018E4280F083
:108E1000C08290F8A71211F0010140F0BA8248F226
:108E20000005C2F2000505F580564FF0000145F837
:108E3000041BB542FBD348F20001C2F20001D0F896
:108E4000DC23A2F58052C0F8DC23914207D201F561
:108E5000805313F8015B01F8015B9142F9D307E5F8
:108E6000D0F8481345F20049C1F200094FEA011158
:108E700089444FF043087DF0D7FD4FF04C087DF05A
:108E8000D3FD4FF046087DF0CFFD4FF020087DF078
:108E9000CBFD19F8018BB8F1FF0F04D07DF0C4FDB4
:108EA00019F00F01F5D14FF00D087DF0BDFD4FF029
:108EB0004E01A0F83A1390F8741221F0020180F8E4
:108EC00074124FF00002A0F83C23F7F7E9B890F8CD
:108ED000A71211F0010124D148F20005C2F20005E9
:108EE00005F580564FF0000145F8041BB542FBD351
:108EF00048F20001C2F20001D0F8DC23A2F5805252
:108F0000C0F8DC23914207D201F5805313F8015BCE
:108F100001F8015B9142F9D34FF00003C0F8A03390
:108F2000A6E44EF60022C2F20002D0F87C424FEADC
:108F3000146102F8011B4FEA144102F8011B4FEAC9
:108F4000142102F8011B214602F8011B4FF0000119
:108F500002F8011B02F8011B02F8011B02F8011BB9
:108F600002F8011B02F8011B02F8011B02F8011BA9
:108F700002F8011B02F8011B02F8011B02F8011B99
:108F80004FF6FF7122F8021B4FF0000122F8021B7E
:108F90004FF0040122F8021B4FF0000122F8021BDF
:108FA00046F20042C4F20202D2F8A01041F00101E0
:108FB000C2F8A010F7F774B8D0F8A033A3F11003EB
:108FC000C0F8A03303E011F0020200F0488148F23B
:108FD0000004C2F20004D0F8A0334EF60022C2F220
:108FE00000024FF00007E15C02F8011B0F4403F19F
:108FF0000103E15C02F8011B0F4403F10103E15C92
:1090000002F8011B0F4403F10103E15C02F8011BAC
:109010000F4403F10103E15C02F8011B0F4403F16B
:109020000103E15C02F8011B0F4403F10103E15C61
:1090300002F8011B0F4403F10103E15C02F8011B7C
:109040000F4403F10103E15C02F8011B0F4403F13B
:109050000103E15C02F8011B0F4403F10103E15C31
:1090600002F8011B0F4403F10103E15C02F8011B4C
:109070000F4403F10103E15C02F8011B0F4403F10B
:109080000103E15C02F8011B0F4403F10103E15C01
:1090900002F8011B0F4403F10103E15C02F8011B1C
:1090A0000F4403F10103C0F8A0334FF6FF7122F81B
:1090B000021B6FEA070707F1010707F0FF0722F815
:1090C000027B4FF00201B3F5805F08BF032122F855
:1090D000021B4FF0000122F8021B46F20042C4F2CC
:1090E0000202D2F8A01041F00101C2F8A010F6F778
:1090F000D7BFD0F8481345F20049C1F200094FEA42
:10910000011189444FF043087DF08EFC4FF04C086C
:109110007DF08AFC4FF046087DF086FC4FF0200879
:109120007DF082FC19F8018BB8F1FF0F04D07DF0BF
:109130007BFC19F00F01F5D14FF00D087DF074FCA8
:109140004FF04E01A0F83A1390F8741221F0040188
:1091500080F874124FF00002A0F83C23F6F7A0BF8D
:1091600090F8A71211F0010125D148F20005C2F2D2
:10917000000505F580564FF0000145F8041BB54287
:10918000FBD348F20001C2F20001D0F8DC23A2F5C3
:109190008052C0F8DC23914207D201F5805313F8C6
:1091A000015B01F8015B9142F9D34FF00003C0F875
:1091B000A033FFF75DBB4EF60022C2F20002D0F8EA
:1091C0007C424FEA146102F8011B4FEA144102F895
:1091D000011B4FEA142102F8011B214602F8011B72
:1091E0004FF0000102F8011B02F8011B02F8011BFD
:1091F00002F8011B02F8011B02F8011B02F8011B17
:1092000002F8011B02F8011B02F8011B02F8011B06
:1092100002F8011B4FF6FF7122F8021B4FF000010C
:1092200022F8021B4FF0040141F4004122F8021B16
:109230004FF0000122F8021B46F20042C4F2020283
:10924000D2F8A01041F00101C2F8A010F6F728BF33
:10925000D0F8A033A3F11003C0F8A03303E011F05D
:10926000040200F0948048F20004C2F20004D0F836
:10927000A0334EF60022C2F200024FF00007E15C7C
:1092800002F8011B0F4403F10103E15C02F8011B2A
:109290000F4403F10103E15C02F8011B0F4403F1E9
:1092A0000103E15C02F8011B0F4403F10103E15CDF
:1092B00002F8011B0F4403F10103E15C02F8011BFA
:1092C0000F4403F10103E15C02F8011B0F4403F1B9
:1092D0000103E15C02F8011B0F4403F10103E15CAF
:1092E00002F8011B0F4403F10103E15C02F8011BCA
:1092F0000F4403F10103E15C02F8011B0F4403F189
:109300000103E15C02F8011B0F4403F10103E15C7E
:1093100002F8011B0F4403F10103E15C02F8011B99
:109320000F4403F10103E15C02F8011B0F4403F158
:109330000103E15C02F8011B0F4403F10103C0F8D3
:10934000A0334FF6FF7122F8021B6FEA070707F1FF
:10935000010707F0FF0722F8027B4FF00201B3F587
:10936000805F08BF032141F4004122F8021B4FF047
:10937000000122F8021B46F20042C4F20202D2F8B7
:10938000A01041F00101C2F8A010F6F789BEF6F76F
:1093900087BE72B64FF0005043F60042C4F202029C
:1093A0004FF6F076C0F61D0640F20121C0F2000132
:1093B000116100BF00BFD0F87C1246F8041B00BF4B
:1093C00000BF00BF00BFD16811F48031FBD111692B
:1093D00021F001011161116941F00041116162B692
:1093E000D0F8481345F20049C1F200094FEA0111D3
:1093F00089444FF043087DF017FB4FF04C087DF097
:1094000013FB4FF046087DF00FFB4FF020087DF076
:109410000BFB19F8018BB8F1FF0F04D07DF004FBB2
:1094200019F00F01F5D14FF00D087DF0FDFA4FF066
:109430004E01A0F83A1390F8741221F0010180F85F
:1094400074124FF00002A0F83C23F6F729BE4E2913
:1094500040F0BA8145F20023C1F20003151FFAF46F
:1094600079AA595D44297AF475AA05F10105595D77
:109470003A297AF46FAA05F10105595D5C297AF45D
:1094800069AA05F10105595D3E297AF463AA4FF0F6
:109490000002A0F83C2390F8741211F0020209D1E6
:1094A00011F0040240F0C6804FF40011C0F86813B8
:1094B000F6F7B2BD90F8741211F0020200F0BA8013
:1094C0004FF00001C0F8F813C0F8A01380F8A712FD
:1094D00048F20001C2F20001C0F8DC1348F20005B6
:1094E000C2F2000505F580564FF0000145F8041B57
:1094F000B542FBD34FF00001C0F84813D0F8481331
:1095000045F20049C1F200094FEA0111894499F876
:109510000010462940F0828099F801105F297DD122
:1095200099F80270322F79D199F803105F2975D11B
:1095300099F80410302971D33A296FD211F0FF0243
:109540004FEA026299F80510302967D33A2965D2AB
:1095500011F0FF014FEA014142EA010299F80610B9
:1095600030295BD33A2959D211F0FF014FEA01218A
:1095700042EA010299F8071030294FD33A294DD217
:1095800011F0FF0142EA010299F808102E2945D195
:1095900099F80910482941D199F80A1045293DD177
:1095A00099F80B10582939D1C0F87C2209F5017AB5
:1095B000DAF80010C0F858134FF04F087DF034FA75
:1095C0004FF050087DF030FA4FF052087DF02CFA41
:1095D0004FF020087DF028FA19F8018BB8F1FF0F41
:1095E00004D07DF021FA19F00F01F5D14FF00D08EC
:1095F0007DF01AFA4FF04A01A0F83A1390F83913A7
:1096000041F0010180F839134FF08071C0F8681300
:109610004FF00002A0F83C23F6F7FEBCD0F8481348
:1096200001F10101D0F8442391429FF01883C0F862
:10963000481363E790F8741211F0040200F0BA8046
:109640004FF00001C0F8F813C0F8A01380F8A7127B
:1096500048F20001C2F20001C0F8DC1348F2000534
:10966000C2F2000505F580564FF0000145F8041BD5
:10967000B542FBD34FF00001C0F84813D0F84813AF
:1096800045F20049C1F200094FEA0111894499F8F5
:109690000010462940F0828099F801105F297DD1A1
:1096A00099F80270332F79D199F803105F2975D199
:1096B00099F80410302971D33A296FD211F0FF02C2
:1096C0004FEA026299F80510302967D33A2965D22A
:1096D00011F0FF014FEA014142EA010299F8061038
:1096E00030295BD33A2959D211F0FF014FEA012109
:1096F00042EA010299F8071030294FD33A294DD296
:1097000011F0FF0142EA010299F808102E2945D113
:1097100099F80910482941D199F80A1045293DD1F5
:1097200099F80B10582939D1C0F87C2209F5017A33
:10973000DAF80010C0F858134FF04F087DF074F9B4
:109740004FF050087DF070F94FF052087DF06CF941
:109750004FF020087DF068F919F8018BB8F1FF0F80
:1097600004D07DF061F919F00F01F5D14FF00D082B
:109770007DF05AF94FF04A01A0F83A1390F83913E6
:1097800041F0010180F839134FF00071C0F86813FF
:109790004FF00002A0F83C23F6F73EBCD0F8481387
:1097A00001F10101D0F8442391429FF05882C0F8A2
:1097B000481363E74FF40011C0F868134FF000023C
:1097C000A0F83C23F6F728BC4FF00002A0F83C2399
:1097D000F6F766BC45F20023C1F20003B0F83C2363
:1097E0009C5402F10102B2F5007F36F459ACA0F8A6
:1097F0003C23F6F755BC4FF00050D0F8781211F02A
:10980000010200F0C48021F00101C0F8781290F844
:10981000741211F001023FF44DAE4FF00001C0F898
:10982000F813C0F8A01380F8A71248F20001C2F2A2
:109830000001C0F8DC1348F20005C2F2000505F58E
:1098400080564FF0000145F8041BB542FBD34FF0A2
:109850000001C0F84813D0F8481345F20049C1F29E
:1098600000094FEA0111894499F80010462940F097
:10987000828099F801105F297DD199F80270312F0B
:1098800079D199F803105F2975D199F8041030291E
:1098900071D33A296FD211F0FF024FEA026299F8B0
:1098A0000510302967D33A2965D211F0FF014FEA3C
:1098B000014142EA010299F8061030295BD33A29A6
:1098C00059D211F0FF014FEA012142EA010299F851
:1098D000071030294FD33A294DD211F0FF0142EA47
:1098E000010299F808102E2945D199F80910482944
:1098F00041D199F80A1045293DD199F80B10582902
:1099000039D1C0F87C2209F5017ADAF80010C0F8E4
:1099100058134FF04F087DF087F84FF050087DF056
:1099200083F84FF052087DF07FF84FF020087DF06B
:109930007BF819F8018BB8F1FF0F04D07DF074F8B3
:1099400019F00F01F5D14FF00D087DF06DF84FF0D3
:109950004A01A0F83A1390F8391341F0010180F858
:1099600039134FF48001C0F868134FF00002A0F8DB
:109970003C23F6F751BBD0F8481301F10101D0F8B0
:10998000442391429FF06B81C0F8481363E7D0F8FD
:10999000781211F0020205D021F00201C0F878120D
:1099A000FFF715BBD0F8781211F0040205D021F0B2
:1099B0000401C0F87812FFF78ABAD0F8781211F0D3
:1099C000080205D021F00801C0F87812FFF7F4BAB8
:1099D000D0F8781211F0100205D021F01001C0F873
:1099E0007812FFF73DBAD0F8781211F0200204D0B7
:1099F00021F02001C0F8781235E4D0F8781211F087
:109A0000400205D021F04001C0F87812FFF7A8BB52
:109A1000D0F8781211F0800204D021F08001C0F853
:109A2000781215E4D0F8781211F4807205D021F480
:109A30008071C0F87812FFF75CBB4FF0005046F21F
:109A40000009C4F20209D9F88C10A1F10101B0F8A3
:109A5000D6A0514514D0AAF1010140F2FF3201EA2B
:109A60000201A0F8D6106FEA0A0A0AEA020A4AF2CC
:109A7000000BC2F2000B1BF80A407BF006FADCE791
:109A80004FF00050B0F8DEA04BF2000BC2F2000B1A
:109A90001BF80A4040F2FF0104EA01048C420ED098
:109AA00040F2FF010BF80A100AF1010A40F2FF31FF
:109AB0000AEA010AA0F8DEA07CF0DBFFE0E74FF045
:109AC0000050D0F8681311F4800206D111F08072B2
:109AD00003D111F0007200F0D980D0F8F8434FEABA
:109AE000943404F0FF0490F81313A14200F0CE80E8
:109AF00080F813434FF023087AF084FE4FF04608B5
:109B00007AF080FE4FF05A087AF07CFE4FF008069B
:109B10007AF090FF4FF02C087AF074FE4FF00106B7
:109B20007AF088FF4FF02C087AF06CFE4FF0230893
:109B30007AF068FE4FF05A087AF064FE4FF046085B
:109B40007AF060FE4FF005067AF074FF4FF02C08B3
:109B50007AF058FE4FF023087AF054FE4FF05A087E
:109B60007AF050FE4FF042087AF04CFE4FF08C062F
:109B70007AF060FF4FF02C087AF044FE4FF0C806F0
:109B80007AF058FF4FF02C087AF03CFE40F2C806FD
:109B90007AF050FF4FF02C087AF034FE4FF0D206E6
:109BA0007AF048FF4FF02C087AF02CFE4FF0310885
:109BB0007AF028FE4FF02C087AF024FE26467AF040
:109BC00039FE4FF000087AF01DFE4FF023087AF0BE
:109BD00019FE4FF05A087AF015FE4FF042087AF05D
:109BE00011FE4FF08C067AF025FF4FF02C087AF02A
:109BF00009FE4FF0B4067AF01DFF4FF02C087AF002
:109C000001FE40F2C8067AF015FF4FF02C087AF0FA
:109C1000F9FD4FF0BE067AF00DFF4FF02C087AF0F8
:109C2000F1FD4FF031087AF0EDFD4FF02C087AF09D
:109C3000E9FD4FF053087AF0E5FD4FF069087AF03E
:109C4000E1FD4FF07A087AF0DDFD4FF065087AF01B
:109C5000D9FD4FF03A087AF0D5FD4FF020087AF0A0
:109C6000D1FDD0F858434FEA14667AF0E3FD4FEA8D
:109C700014467AF0DFFD4FEA14267AF0DBFD264623
:109C80007AF0D8FD4FF000087AF0BCFDB0F8026F12
:109C9000B0F81E7DBE420BD04682A0F81C6D8682B5
:109CA00077F0BEF9B0F8026FA0F81E6DF6F7B4B900
:109CB00090F8066F477CBE421DD080F8206D467438
:109CC00040F265018E4201D340F26406142E38BF83
:109CD00014264FF023087AF095FD4FF059087AF0DA
:109CE00091FD4FF048087AF08DFD7AF0A3FE4FF019
:109CF0002C087AF087FD90F8046F90F8BF70BE4290
:109D000003D080F8216D80F8BF6090F86A1011F0E0
:109D1000010217D090F8164F14F0800212D014F000
:109D200040020FD021F0010180F86A1014F0020205
:109D300002D014F0040205D14FF00063C0F868337C
:109D4000F6F76AB990F8FD1311F0010215D090F8FA
:109D5000F71311F0010205D021F0010180F8F7138B
:109D60007AF018F890F8F71311F0020205D021F0FC
:109D7000020180F8F71379F007FF826DD0F8805266
:109D8000D0F8846222F000425FEA32025FEA3505D1
:109D90005FEA36064FEA9251134681EA030161F306
:109DA0009E728265C0F88052C0F8846290F88B136E
:109DB00011F0020100F0EE80D0F81481D0F80471A7
:109DC0006FEA070708EA0708B8F1000F26D04BF63C
:109DD0000606C2F200064FF0010918F0010209D18F
:109DE00019F000421AD14FEA580806F108064FEA66
:109DF0004909F2E74FF0000333806FEA0902D0F817
:109E0000143103EA0203C0F81431D0F8F43003EA45
:109E10000203C0F8F4307AF08DF8E1E7D0F8188149
:109E2000D0F808716FEA070708EA0708B8F1000FD1
:109E300026D04BF60616C2F200064FF0010918F0C4
:109E4000010209D119F000421AD14FEA580806F16F
:109E500008064FEA4909F2E74FF0000333806FEA42
:109E60000902D0F8183103EA0203C0F81831D0F81B
:109E7000F83003EA0203C0F8F8307AF05BF8E1E763
:109E8000D0F81C81D0F80C716FEA070708EA0708C0
:109E9000B8F1000F26D04BF60626C2F200064FF0AE
:109EA000010918F0010209D119F000421AD14FEA54
:109EB000580806F108064FEA4909F2E74FF0000397
:109EC00033806FEA0902D0F81C3103EA0203C0F8BC
:109ED0001C31D0F8FC3003EA0203C0F8FC307AF001
:109EE00029F8E1E7D0F82081D0F810716FEA070770
:109EF00008EA0708B8F1000F26D04BF60636C2F282
:109F000000064FF0010918F0010209D119F00042D2
:109F10001AD14FEA580806F108064FEA4909F2E754
:109F20004FF0000333806FEA0902D0F8203103EAD2
:109F30000203C0F82031D0F8003103EA0203C0F870
:109F4000003179F0F7FFE1E74FF00001C0F80411AC
:109F5000C0F80811C0F80C11C0F81011C0F8F410C6
:109F6000C0F8F810C0F8FC10C0F80011C0F81411C7
:109F7000C0F81811C0F81C11C0F82011468AA0F8CA
:109F80001C6D868277F04CF84FF0000180F88B133F
:109F9000F6F742B84FF0005090F87B1311F0010132
:109FA00017D090F8F11011F0010112D190F847117B
:109FB00011F001010DD1B0F8F210002909D14FF0D4
:109FC000000180F87B1380F839137FF06DFCF6F701
:109FD00023B84FF00050D0F81863D0F82043A4EB1A
:109FE0000604002C27D0B0F8CA23B0F8C8334FEAD3
:109FF000432343EA02024FEA8232A4FB02231E44B7
:10A0000026F00106C0F8D063D0F81863D0F82043DA
:10A01000A4EB0604B0F8CE23B0F8CC334FEA4323C8
:10A0200043EA02024FEA8232A4FB02231E4426F0D6
:10A030000106C0F8D4634FF0005090F8681011F09A
:10A04000010100F0968041F20001C2F20001B1F876
:10A05000307AB1F840AA4FF00050B0F8F85115F03E
:10A06000010508BF83F0A7FA41F20001C2F2000126
:10A07000B1F8327AB1F842AA4FF00050B0F8F85176
:10A0800015F0020500F5807008BF83F094FA41F2E4
:10A090000001C2F20001B1F8347AB1F844AA4FF0DD
:10A0A0000050B0F8F85115F0040500F5007008BF35
:10A0B00083F081FA41F20001C2F20001B1F8367A70
:10A0C000B1F846AA4FF00050B0F8F85115F0080565
:10A0D00000F5407008BF83F06EFA41F20001C2F251
:10A0E0000001B1F8387AB1F848AA4FF00050B0F842
:10A0F000F85115F0100500F5806008BF83F05BFA99
:10A1000041F20001C2F20001B1F83A7AB1F84AAA6C
:10A110004FF00050B0F8F85115F0200500F5A060A0
:10A1200008BF83F048FA41F20001C2F20001B1F821
:10A130003C7AB1F84CAA4FF00050B0F8F85115F045
:10A14000400500F5C06008BF83F035FA41F2000118
:10A15000C2F20001B1F83E7AB1F84EAA4FF00050B9
:10A16000B0F8F85115F0800500F5E06008BF83F005
:10A1700022FA40F20044C4F20204228A12F48062FD
:10A1800000F04E864FF0005041F20004C2F200048D
:10A1900090F8122312F0020100F0CF8022F00202A8
:10A1A00080F81223B0F80013B1F5006F60D2D0F838
:10A1B0001C63D0F81C1312F0800312D06FF08003E0
:10A1C00002EA030280F8122340F20003CFF6FE7386
:10A1D00006EA03064FF60063CFF6FF7301EA0301B8
:10A1E0000BE04FF60063CFF6FF7301EA030106EAC6
:10A1F000030601F5007106F500764FF6FF72C0F216
:10A20000010212EA060409D179F0C4FB01EA020155
:10A210006FEA020206EA020646EA010644F200027A
:10A220004FEA024296421ED278F0B9FE41F6000B88
:10A23000C2F2020B0BF500794FF00007C0F60007E1
:10A240004FF40068A76100BF00BF00BF00BF95F8D2
:10A2500011A0C4F818800BF801ABCB45F2D14FF038
:10A260008007AF6103E04FF0000280F8122364E042
:10A27000D0F81C63D0F81C1312F0800312D06FF0DA
:10A28000800302EA030280F8122340F20003CFF6B3
:10A29000FE7306EA03064FF60063CFF6FF7301EA8A
:10A2A00003010BE04FF60063CFF6FF7301EA0301F1
:10A2B00006EA030601F5007106F500764FF6FF7217
:10A2C000C0F2010212EA060409D179F076FB01EA34
:10A2D00002016FEA020206EA020646EA010644F2B9
:10A2E00000024FEA0242964223D278F03EFF41F646
:10A2F000000BC2F2020B0BF500794FF00007C0F61D
:10A3000000074FF40068A76100BF00BF00BF00BF97
:10A3100095F811A0C4F818800BF801ABCB45F2D129
:10A3200040F60009C4F202094FF02007C9F818707E
:10A3300003E04FF0000280F8122390F8122312F08D
:10A34000040100F0CF8022F0040280F81223B0F85C
:10A350000013B1F5006F60D2D0F81C63D0F81C1365
:10A3600012F0800312D06FF0800302EA030280F83B
:10A37000122340F20003CFF6FE7306EA03064FF6FF
:10A380000063CFF6FF7301EA03010BE04FF60063B1
:10A39000CFF6FF7301EA030106EA030601F5007137
:10A3A00006F500764FF6FF72C0F2010212EA0604CB
:10A3B00009D179F0EFFA01EA02016FEA020206EA36
:10A3C000020646EA010644F200024FEA02429642C1
:10A3D0001ED278F0E4FD41F6002BC2F2020B0BF521
:10A3E00000794FF00007C0F600074FF40068A7613E
:10A3F00000BF00BF00BF00BF95F811A0C4F81880CF
:10A400000BF801ABCB45F2D14FF08007AF6103E011
:10A410004FF0000280F8122364E0D0F81C63D0F8FB
:10A420001C1312F0800312D06FF0800302EA0302C3
:10A4300080F8122340F20003CFF6FE7306EA03060B
:10A440004FF60063CFF6FF7301EA03010BE04FF60E
:10A450000063CFF6FF7301EA030106EA030601F584
:10A46000007106F500764FF6FF72C0F2010212EAA3
:10A47000060409D179F0A1FA01EA02016FEA0202A9
:10A4800006EA020646EA010644F200024FEA0242E8
:10A49000964223D278F069FE41F6002BC2F2020BFD
:10A4A0000BF500794FF00007C0F600074FF4006885
:10A4B000A76100BF00BF00BF00BF95F811A0C4F89E
:10A4C00018800BF801ABCB45F2D140F60009C4F27D
:10A4D00002094FF02007C9F8187003E04FF000029E
:10A4E00080F812234FF0005090F8681011F001012D
:10A4F00001F0CE834FF0005090F8FF2212F00201DD
:10A5000000F0B78022F0020280F8FF22D0F8C46287
:10A5100090F8B31311F0010153D14FF6FF72C0F25E
:10A52000010212EA060401D179F034FA44F2000281
:10A530004FEA024296423DD278F048FE41F2000BCB
:10A54000C2F2020B0BF500794FF00007C0F20107D1
:10A550004FF001081BF801AB85F815A0A76100BFFB
:10A5600000BFC4F81880CB45F4D140F20407C0F214
:10A57000010740F210026A75A76140F20107C0F2BC
:10A58000040700BF00BF00BF00BFA76100BF00BF3E
:10A59000228A12F48062FBD146F62022C0F2000229
:10A5A0002A6000BF00BF4FF08007AF614FF4007416
:10A5B000264403E04FF0000180F8FF12C0F8C462A7
:10A5C00057E04FF6FF72C0F2010212EA060401D111
:10A5D00079F0F3F944F200024FEA0242964242D285
:10A5E00078F0B5FE41F2000BC2F2020B0BF50079D8
:10A5F0004FF00007C0F201074FF001081BF801AB54
:10A6000085F815A0A76100BF00BFC4F81880CB452E
:10A61000F4D140F20407C0F2010740F210026A755B
:10A62000A76140F20107C0F2040700BF00BF00BFEE
:10A6300000BFA76100BF00BF228A12F48062FBD175
:10A6400046F62022C0F200022A6000BF00BF40F69A
:10A650000009C4F202094FF02007C9F818704FF43E
:10A660000074264403E04FF0000180F8FF12C0F8A8
:10A67000C46290F8FF2212F0040100F0B78022F0CB
:10A68000040280F8FF22D0F8C46290F8B31311F0EE
:10A69000010153D14FF6FF72C0F2010212EA060423
:10A6A00001D179F077F944F200024FEA0242964272
:10A6B0003DD278F08BFD41F2002BC2F2020B0BF57C
:10A6C00000794FF00007C0F201074FF001081BF8B6
:10A6D00001AB85F815A0A76100BF00BFC4F81880C2
:10A6E000CB45F4D140F20407C0F2010740F210025A
:10A6F0006A75A76140F20107C0F2040700BF00BFFE
:10A7000000BF00BFA76100BF00BF228A12F48062B1
:10A71000FBD146F62022C0F200022A6000BF00BF33
:10A720004FF08007AF614FF40074264403E04FF010
:10A73000000180F8FF12C0F8C46257E04FF6FF72C4
:10A74000C0F2010212EA060401D179F036F944F2AE
:10A7500000024FEA0242964242D278F0F8FD41F2FE
:10A76000002BC2F2020B0BF500794FF00007C0F28C
:10A7700001074FF001081BF801AB85F815A0A76190
:10A7800000BF00BFC4F81880CB45F4D140F20407E5
:10A79000C0F2010740F210026A75A76140F201079A
:10A7A000C0F2040700BF00BF00BF00BFA76100BF29
:10A7B00000BF228A12F48062FBD146F62022C0F24A
:10A7C00000022A6000BF00BF40F60009C4F202097F
:10A7D0004FF02007C9F818704FF40074264403E0C6
:10A7E0004FF0000180F8FF12C0F8C4624FF0005033
:10A7F00090F8A62212F0020100F0B78022F00202C7
:10A8000080F8A62290F8B31311F0010154D1D0F8CA
:10A81000C862D0F8C81212F080030ED022F0800275
:10A8200080F8A622D0F8CC62C0F8C862314640F267
:10A830000003CFF6FE7306EA03064FF6FF72C0F27E
:10A84000010212EA060409D179F0A4F801EA020132
:10A850006FEA020206EA020646EA010644F2000234
:10A860004FEA0242964220D278F099FB41F2000B67
:10A87000C2F2020B0BF500794FF00007C0F600079B
:10A880004FF40068A76100BF00BF00BF00BF95F88C
:10A8900011A0C4F818800BF801ABCB45F2D14FF0F2
:10A8A0008007AF6106F5007603E04FF0000180F805
:10A8B000A612C0F8C86258E0D0F8C862D0F8C81232
:10A8C00012F080030ED022F0800280F8A622D0F889
:10A8D000CC62C0F8C862314640F20003CFF6FE7386
:10A8E00006EA03064FF6FF72C0F2010212EA0604FE
:10A8F00009D179F062F801EA02016FEA020206EA80
:10A90000020646EA010644F200024FEA024296427B
:10A9100025D278F02AFC41F2000BC2F2020B0BF5B3
:10A9200000794FF00007C0F600074FF40068A761F8
:10A9300000BF00BF00BF00BF95F811A0C4F8188089
:10A940000BF801ABCB45F2D140F60009C4F2020985
:10A950004FF02007C9F8187006F5007603E04FF0B5
:10A96000000180F8A612C0F8C8624FF0005090F8BD
:10A97000A62212F0040100F0B78022F0040280F851
:10A98000A62290F8B31311F0010154D1D0F8C86297
:10A99000D0F8C81212F080030ED022F0800280F8A6
:10A9A000A622D0F8CC62C0F8C862314640F200035B
:10A9B000CFF6FE7306EA03064FF6FF72C0F20102FD
:10A9C00012EA060409D178F0E5FF01EA02016FEA14
:10A9D000020206EA020646EA010644F200024FEAD3
:10A9E0000242964220D278F0DAFA41F2002BC2F20B
:10A9F000020B0BF500794FF00007C0F600074FF48B
:10AA00000068A76100BF00BF00BF00BF95F811A09C
:10AA1000C4F818800BF801ABCB45F2D14FF080079A
:10AA2000AF6106F5007603E04FF0000180F8A61252
:10AA3000C0F8C86258E0D0F8C862D0F8C81212F066
:10AA400080030ED022F0800280F8A622D0F8CC62DB
:10AA5000C0F8C862314640F20003CFF6FE7306EA42
:10AA600003064FF6FF72C0F2010212EA060409D192
:10AA700078F0A3FF01EA02016FEA020206EA020689
:10AA800046EA010644F200024FEA0242964225D20B
:10AA900078F06BFB41F2002BC2F2020B0BF5007950
:10AAA0004FF00007C0F600074FF40068A76100BF31
:10AAB00000BF00BF00BF95F811A0C4F818800BF8C4
:10AAC00001ABCB45F2D140F60009C4F202094FF0C8
:10AAD0002007C9F8187006F5007603E04FF0000172
:10AAE00080F8A612C0F8C8624FF0005041F200048E
:10AAF000C2F20004B4F80821062A01D0022A23D1A8
:10AB000090F8FE2412F0020109D022F0020280F82F
:10AB1000FE2443F2000BC2F2020B78F02CF84FF047
:10AB2000005041F20004C2F2000490F8FE2412F03A
:10AB3000040109D022F0040280F8FE2443F6000B41
:10AB4000C2F2020B78F017F84FF0005000F5807059
:10AB500041F20014C2F20004B4F80821062A01D020
:10AB6000022A25D190F8FE2412F0020109D022F029
:10AB7000020280F8FE2444F2000BC2F2020B77F0CE
:10AB8000FAFF4FF0005000F5807041F20014C2F25D
:10AB9000000490F8FE2412F0040109D022F004020F
:10ABA00080F8FE2444F6000BC2F2020B77F0E3FFBC
:10ABB0004FF0005000F5007041F20024C2F2000492
:10ABC000B4F80821062A01D0022A25D190F8FE24E3
:10ABD00012F0020109D022F0020280F8FE2445F2B0
:10ABE000000BC2F2020B77F0C6FF4FF0005000F5E9
:10ABF000007041F20024C2F2000490F8FE2412F02A
:10AC0000040109D022F0040280F8FE2445F6000B6E
:10AC1000C2F2020B77F0AFFF4FF0005000F540702A
:10AC200041F20034C2F20004B4F80821062A01D02F
:10AC3000022A25D190F8FE2412F0020109D022F058
:10AC4000020280F8FE2446F2000BC2F2020B77F0FB
:10AC500092FF4FF0005000F5407041F20034C2F214
:10AC6000000490F8FE2412F0040109D022F004023E
:10AC700080F8FE2446F6000BC2F2020B77F07BFF51
:10AC80004FF0005000F5806041F20044C2F2000431
:10AC9000B4F80821062A01D0022A25D190F8FE2412
:10ACA00012F0020109D022F0020280F8FE2447F2DD
:10ACB000000BC2F2020B77F05EFF4FF0005000F580
:10ACC000806041F20044C2F2000490F8FE2412F0C9
:10ACD000040109D022F0040280F8FE2447F6000B9C
:10ACE000C2F2020B77F047FF4FF0005000F5A06072
:10ACF00041F20054C2F20004B4F80821062A01D03F
:10AD0000022A25D190F8FE2412F0020109D022F087
:10AD1000020280F8FE2448F2000BC2F2020B77F028
:10AD20002AFF4FF0005000F5A06041F20054C2F23B
:10AD3000000490F8FE2412F0040109D022F004026D
:10AD400080F8FE2448F6000BC2F2020B77F013FFE6
:10AD50004FF0005000F5C06041F20064C2F2000400
:10AD6000B4F80821062A01D0022A25D190F8FE2441
:10AD700012F0020109D022F0020280F8FE2449F20A
:10AD8000000BC2F2020B77F0F6FE4FF0005000F518
:10AD9000C06041F20064C2F2000490F8FE2412F098
:10ADA000040109D022F0040280F8FE2449F6000BC9
:10ADB000C2F2020B77F0DFFE4FF0005000F5E060CA
:10ADC00041F20074C2F20004B4F80821062A01D04E
:10ADD000022A25D190F8FE2412F0020109D022F0B7
:10ADE000020280F8FE244AF2000BC2F2020B77F056
:10ADF000C2FE4FF0005000F5E06041F20074C2F274
:10AE0000000490F8FE2412F0040109D022F004029C
:10AE100080F8FE244AF6000BC2F2020B77F0ABFE7C
:10AE20004FF0005041F20001C2F20001B1F8B2301F
:10AE30004FEA8353C0F8A433B1F8B4304FEA8353D8
:10AE4000C0F8A833B1F8B63080F8D1304FF00050D8
:10AE500041F20004C2F2000447F20009C1F2000905
:10AE600040F60007C4F200077EF00CFF4FF00050E0
:10AE700041F20001C2F2000147F20007C1F20007EF
:10AE80007FF03CFA4FF0005041F20001C2F20001A5
:10AE900047F20007C1F200077FF044FB4FF000507B
:10AEA00041F20001C2F2000147F20007C1F20007BF
:10AEB0007FF08FFB4FF0005000F5807041F20014DE
:10AEC000C2F2000447F20019C1F2000940F2004743
:10AED000C4F200077EF0D6FE4FF0005000F58070FF
:10AEE00041F20011C2F2000147F20017C1F200075F
:10AEF0007FF004FA4FF0005000F5807041F200112D
:10AF0000C2F2000147F20017C1F200077FF00AFB0E
:10AF10004FF0005000F5807041F20011C2F20001C4
:10AF200047F20017C1F200077FF053FB4FF00050CB
:10AF300000F5007041F20024C2F2000447F200293B
:10AF4000C1F2000940F20007C4F201077EF09AFE48
:10AF50004FF0005000F5007041F20021C2F20001F4
:10AF600047F20027C1F200077FF0C8F94FF0005008
:10AF700000F5007041F20021C2F2000147F2002703
:10AF8000C1F200077FF0CEFA4FF0005000F50070DC
:10AF900041F20021C2F2000147F20027C1F200078E
:10AFA0007FF017FB4FF0005000F5407041F2003485
:10AFB000C2F2000447F20039C1F2000944F200076E
:10AFC000C4F201077EF05EFE4FF0005000F54070C5
:10AFD00041F20031C2F2000147F20037C1F200072E
:10AFE0007FF08CF94FF0005000F5407041F20031D5
:10AFF000C2F2000147F20037C1F200077FF092FA77
:10B000004FF0005000F5407041F20031C2F20001F3
:10B0100047F20037C1F200077FF0DBFA4FF0005033
:10B0200000F5806041F20044C2F2000447F200499A
:10B03000C1F2000944F20047C4F201077EF022FE8B
:10B040004FF0005000F5806041F20041C2F2000173
:10B0500047F20047C1F200077FF050F94FF000506F
:10B0600000F5806041F20041C2F2000147F2004762
:10B07000C1F200077FF056FA4FF0005000F58060F3
:10B0800041F20041C2F2000147F20047C1F200075D
:10B090007FF09FFA4FF0005000F5A06041F200549D
:10B0A000C2F2000447F20059C1F2000944F6000759
:10B0B000C4F201077EF0E6FD4FF0005000F5A060FD
:10B0C00041F20051C2F2000147F20057C1F20007FD
:10B0D0007FF014F94FF0005000F5A06041F20051EC
:10B0E000C2F2000147F20057C1F200077FF01AFADE
:10B0F0004FF0005000F5A06041F20051C2F2000193
:10B1000047F20057C1F200077FF063FA4FF000509A
:10B1100000F5C06041F20064C2F2000447F2006929
:10B12000C1F200094FF000077EF0ACFD4FF0005077
:10B1300000F5C06041F20061C2F2000147F2006711
:10B14000C1F200077FF0DAF84FF0005000F5C06060
:10B1500041F20061C2F2000147F20067C1F200074C
:10B160007FF0E0F94FF0005000F5C06041F200615F
:10B17000C2F2000147F20067C1F200077FF029FA2E
:10B180004FF0005000F5E06041F20074C2F200049C
:10B1900047F20079C1F200094FF000077EF072FD1E
:10B1A0004FF0005000F5E06041F20071C2F2000182
:10B1B00047F20077C1F200077FF0A0F84FF000508F
:10B1C00000F5E06041F20071C2F2000147F2007741
:10B1D000C1F200077FF0A6F94FF0005000F5E060E3
:10B1E00041F20071C2F2000147F20077C1F200079C
:10B1F0007FF0EFF94FF0005090F85D10002928D152
:10B2000001F1010180F85D1041F20011C2F200016C
:10B21000B1F88C2112F001031AD012F4807217D009
:10B220000B4601F580714FF000040C2C0BD0142C50
:10B2300009D0162C07D08C2C05D0942C03D0962C3A
:10B2400001D01A5B0A5304F10204B4F5807FECD3F9
:10B25000FEE0012928D101F1010180F85D1041F2E1
:10B260000021C2F20001B1F88C2112F001031AD0C2
:10B2700012F4807217D00B4601F580714FF0000474
:10B280000C2C0BD0142C09D0162C07D08C2C05D0EC
:10B29000942C03D0962C01D01A5B0A5304F10204BB
:10B2A000B4F5807FECD3D3E0022928D101F101016C
:10B2B00080F85D1041F20031C2F20001B1F88C213A
:10B2C00012F001031AD012F4807217D00B4601F568
:10B2D00080714FF000040C2C0BD0142C09D0162CCC
:10B2E00007D08C2C05D0942C03D0962C01D01A5B5F
:10B2F0000A5304F10204B4F5807FECD3A8E00329DB
:10B3000028D101F1010180F85D1041F20041C2F243
:10B310000001B1F88C2112F001031AD012F48072EE
:10B3200017D00B4601F580714FF000040C2C0BD0A8
:10B33000142C09D0162C07D08C2C05D0942C03D0BB
:10B34000962C01D01A5B0A5304F10204B4F5807FF5
:10B35000ECD37DE0042928D101F1010180F85D10D2
:10B3600041F20051C2F20001B1F88C2112F0010348
:10B370001AD012F4807217D00B4601F580714FF08D
:10B3800000040C2C0BD0142C09D0162C07D08C2CBC
:10B3900005D0942C03D0962C01D01A5B0A5304F1EB
:10B3A0000204B4F5807FECD352E0052928D101F1E5
:10B3B000010180F85D1041F20061C2F20001B1F8B4
:10B3C0008C2112F001031AD012F4807217D00B46B0
:10B3D00001F580714FF000040C2C0BD0142C09D017
:10B3E000162C07D08C2C05D0942C03D0962C01D091
:10B3F0001A5B0A5304F10204B4F5807FECD327E012
:10B400004FF0000180F85D1041F20071C2F20001BE
:10B41000B1F88C2112F001031AD012F4807217D007
:10B420000B4601F580714FF000040C2C0BD0142C4E
:10B4300009D0162C07D08C2C05D0942C03D0962C38
:10B4400001D01A5B0A5304F10204B4F5807FECD3F7
:10B450004FF0005041F20001C2F20001B1F8942116
:10B46000A0F8242D47F20004C1F20004A1694FEABC
:10B47000116180F80A1D216A4FEA116180F8121DDE
:10B48000A16B4FEA116180F8021D216C4FEA116136
:10B4900080F8501DA16C4FEA116180F8511D216D9B
:10B4A0004FEA116180F8521DA16D4FEA116180F8D9
:10B4B000531D216E4FEA116180F8541DA16E4FEAB1
:10B4C000116180F8551D216F4FEA116180F8561DFA
:10B4D000A16F4FEA116180F8571DD4F880104FEA30
:10B4E000116180F8581DD4F888104FEA116180F876
:10B4F000591DD4F890104FEA116180F85A1DD4F804
:10B5000098104FEA116180F85B1DD4F8A0104FEA43
:10B51000116180F85C1DD4F8A8104FEA116180F821
:10B520005D1DD4F8B0104FEA116180F85E1DD4F8AB
:10B53000B8104FEA116180F85F1DD4F8C0104FEACF
:10B54000116180F8601DD4F8C8104FEA116180F8CD
:10B55000611DD4F8D0104FEA116180F8621DD4F853
:10B56000D8104FEA116180F8631D04F58074A16959
:10B570004FEA116180F80B1D216A4FEA116180F8D2
:10B58000131DA16B4FEA116180F8031D216C4FEA76
:10B59000116180F8701DA16C4FEA116180F8711D76
:10B5A000216D4FEA116180F8721DA16D4FEA1161A2
:10B5B00080F8731D216E4FEA116180F8741DA16E31
:10B5C0004FEA116180F8751D216F4FEA116180F813
:10B5D000761DA16F4FEA116180F8771DD4F88010B5
:10B5E0004FEA116180F8781DD4F888104FEA116194
:10B5F00080F8791DD4F890104FEA116180F87A1D17
:10B60000D4F898104FEA116180F87B1DD4F8A0108F
:10B610004FEA116180F87C1DD4F8A8104FEA11613F
:10B6200080F87D1DD4F8B0104FEA116180F87E1DBE
:10B63000D4F8B8104FEA116180F87F1DD4F8C0101B
:10B640004FEA116180F8801DD4F8C8104FEA1161EB
:10B6500080F8811DD4F8D0104FEA116180F8821D66
:10B66000D4F8D8104FEA116180F8831D04F5807476
:10B67000A1694FEA116180F80C1D216A4FEA11613E
:10B6800080F8141DA16B4FEA116180F8041D216C34
:10B690004FEA116180F8901DA16C4FEA116180F8AA
:10B6A000911D216D4FEA116180F8921DA16D4FEA45
:10B6B000116180F8931D216E4FEA116180F8941D8D
:10B6C000A16E4FEA116180F8951D216F4FEA11615B
:10B6D00080F8961DA16F4FEA116180F8971DD4F88C
:10B6E00080104FEA116180F8981DD4F888104FEA55
:10B6F000116180F8991DD4F890104FEA116180F81B
:10B700009A1DD4F898104FEA116180F89B1DD4F867
:10B71000A0104FEA116180F89C1DD4F8A8104FEAE0
:10B72000116180F89D1DD4F8B0104FEA116180F8C6
:10B730009E1DD4F8B8104FEA116180F89F1DD4F80F
:10B74000C0104FEA116180F8A01DD4F8C8104FEA6C
:10B75000116180F8A11DD4F8D0104FEA116180F872
:10B76000A21DD4F8D8104FEA116180F8A31D04F58A
:10B770008074A1694FEA116180F80D1D216A4FEABA
:10B78000116180F8151DA16B4FEA116180F8051D4C
:10B79000216C4FEA116180F8B01DA16C4FEA116174
:10B7A00080F8B11D216D4FEA116180F8B21DA16DC5
:10B7B0004FEA116180F8B31D216E4FEA116180F8E4
:10B7C000B41DA16E4FEA116180F8B51D216F4FEADB
:10B7D000116180F8B61DA16F4FEA116180F8B71DA5
:10B7E000D4F880104FEA116180F8B81DD4F88810A1
:10B7F0004FEA116180F8B91DD4F890104FEA116139
:10B8000080F8BA1DD4F898104FEA116180F8BB1D7A
:10B81000D4F8A0104FEA116180F8BC1DD4F8A8102C
:10B820004FEA116180F8BD1DD4F8B0104FEA1161E4
:10B8300080F8BE1DD4F8B8104FEA116180F8BF1D22
:10B84000D4F8C0104FEA116180F8C01DD4F8C810B8
:10B850004FEA116180F8C11DD4F8D0104FEA116190
:10B8600080F8C21DD4F8D8104FEA116180F8C31DCA
:10B8700004F58074A1694FEA116180F80E1D216AF8
:10B880004FEA116180F8161DA16B4FEA116180F833
:10B89000061D216C4FEA116180F8D01DA16C4FEAA2
:10B8A000116180F8D11D216D4FEA116180F8D21D20
:10B8B000A16D4FEA116180F8D31D216E4FEA11612D
:10B8C00080F8D41DA16E4FEA116180F8D51D216F5B
:10B8D0004FEA116180F8D61DA16F4FEA116180F81F
:10B8E000D71DD4F880104FEA116180F8D81DD4F824
:10B8F00088104FEA116180F8D91DD4F890104FEAF2
:10B90000116180F8DA1DD4F898104FEA116180F8BF
:10B91000DB1DD4F8A0104FEA116180F8DC1DD4F8CB
:10B92000A8104FEA116180F8DD1DD4F8B0104FEA7D
:10B93000116180F8DE1DD4F8B8104FEA116180F86B
:10B94000DF1DD4F8C0104FEA116180F8E01DD4F873
:10B95000C8104FEA116180F8E11DD4F8D0104FEA09
:10B96000116180F8E21DD4F8D8104FEA116180F817
:10B97000E31D04F58074A1694FEA116180F80F1D81
:10B98000216A4FEA116180F8171DA16B4FEA11611E
:10B9900080F8071D216C4FEA116180F8F01DA16C41
:10B9A0004FEA116180F8F11D216D4FEA116180F8B5
:10B9B000F21DA16D4FEA116180F8F31D216E4FEA6F
:10B9C000116180F8F41DA16E4FEA116180F8F51D38
:10B9D000216F4FEA116180F8F61DA16F4FEA1161E6
:10B9E00080F8F71DD4F880104FEA116180F8F81D37
:10B9F000D4F888104FEA116180F8F91DD4F890103E
:10BA00004FEA116180F8FA1DD4F898104FEA1161DD
:10BA100080F8FB1DD4F8A0104FEA116180F8FC1DDE
:10BA2000D4F8A8104FEA116180F8FD1DD4F8B010C9
:10BA30004FEA116180F8FE1DD4F8B8104FEA116189
:10BA400080F8FF1DD4F8C0104FEA116180F8001E85
:10BA5000D4F8C8104FEA116180F8011ED4F8D01054
:10BA60004FEA116180F8021ED4F8D8104FEA116134
:10BA700080F8031E04F58074A1694FEA116180F813
:10BA8000101D216A4FEA116180F8181DA16B4FEA61
:10BA9000116180F8081DB0F8FA1A4FEA112180F8F8
:10BAA0001A1D216C4FEA116180F8101EA16C4FEA3B
:10BAB000116180F8111E216D4FEA116180F8121E8C
:10BAC000A16D4FEA116180F8131E216E4FEA1161DA
:10BAD00080F8141EA16E4FEA116180F8151E216FC7
:10BAE0004FEA116180F8161EA16F4FEA116180F8CC
:10BAF000171ED4F880104FEA116180F8181ED4F890
:10BB000088104FEA116180F8191ED4F890104FEA9E
:10BB1000116180F81A1ED4F898104FEA116180F86C
:10BB20001B1ED4F8A0104FEA116180F81C1ED4F837
:10BB3000A8104FEA116180F81D1ED4F8B0104FEA2A
:10BB4000116180F81E1ED4F8B8104FEA116180F818
:10BB50001F1ED4F8C0104FEA116180F8201ED4F8DF
:10BB6000C8104FEA116180F8211ED4F8D0104FEAB6
:10BB7000116180F8221ED4F8D8104FEA116180F8C4
:10BB8000231E04F58074A1694FEA116180F8111D2C
:10BB9000216A4FEA116180F8191DA16B4FEA11610A
:10BBA00080F8091DB0F8FA1B4FEA112180F81B1D1F
:10BBB000216C4FEA116180F8301EA16C4FEA1161CF
:10BBC00080F8311E216D4FEA116180F8321EA16D9F
:10BBD0004FEA116180F8331E216E4FEA116180F83F
:10BBE000341EA16E4FEA116180F8351E216F4FEAB5
:10BBF000116180F8361EA16F4FEA116180F8371E7F
:10BC0000D4F880104FEA116180F8381ED4F88810FB
:10BC10004FEA116180F8391ED4F890104FEA116193
:10BC200080F83A1ED4F898104FEA116180F83B1E54
:10BC3000D4F8A0104FEA116180F83C1ED4F8A81087
:10BC40004FEA116180F83D1ED4F8B0104FEA11613F
:10BC500080F83E1ED4F8B8104FEA116180F83F1EFC
:10BC6000D4F8C0104FEA116180F8401ED4F8C81013
:10BC70004FEA116180F8411ED4F8D0104FEA1161EB
:10BC800080F8421ED4F8D8104FEA116180F8431EA4
:10BC90004FF00050B0F86E1011F0010174F4BCA91F
:10BCA00090F8A01211F0010100F00C814FF000019A
:10BCB00080F8A0124FF0230878F0A4FD4FF046085A
:10BCC00078F0A0FD4FF05A0878F09CFD4FF0330853
:10BCD00078F098FD4FF02C0878F094FD4FF0320882
:10BCE00078F090FD4FF0330878F08CFD4FF02C0881
:10BCF00078F088FD4FF0230878F084FD4FF05A0863
:10BD000078F080FD4FF0460878F07CFD4FF0310868
:10BD100078F078FD4FF0330878F074FD4FF02C0880
:10BD200078F070FD4FF0230878F06CFD4FF05A0862
:10BD300078F068FD4FF04C0878F064FD4FF0310862
:10BD400078F060FD4FF0320878F05CFD4FF030087D
:10BD500078F058FD4FF02C0878F054FD4FF0310882
:10BD600078F050FD4FF0300878F04CFD4FF030087F
:10BD700078F048FD4FF02C0878F044FD4FF0530860
:10BD800078F040FD4FF0790878F03CFD4FF07308F3
:10BD900078F038FD4FF0450878F034FD4FF0780822
:10BDA00078F030FD4FF0000878F02CFD4FF02308BC
:10BDB00078F028FD4FF05A0878F024FD4FF04C0839
:10BDC00078F020FD4FF0310878F01CFD4FF032087C
:10BDD00078F018FD4FF0300878F014FD4FF02C0883
:10BDE00078F010FD4FF0310878F00CFD4FF033087B
:10BDF00078F008FD4FF0300878F004FD4FF02C0883
:10BE000078F000FD4FF0420878F0FCFC4FF0750828
:10BE100078F0F8FC4FF0660878F0F4FC4FF0660814
:10BE200078F0F0FC4FF0650878F0ECFC4FF0720809
:10BE300078F0E8FC4FF0000878F0E4FC4FF02308BD
:10BE400078F0E0FC4FF05A0878F0DCFC4FF04C083A
:10BE500078F0D8FC4FF0310878F0D4FC4FF032087D
:10BE600078F0D0FC4FF0300878F0CCFC4FF02C0884
:10BE700078F0C8FC4FF0310878F0C4FC4FF0360879
:10BE800078F0C0FC4FF0300878F0BCFC4FF02C0884
:10BE900078F0B8FC4FF0460878F0B4FC4FF0750825
:10BEA00078F0B0FC4FF06C0878F0ACFC4FF06C0808
:10BEB00078F0A8FC4FF0210878F0A4FC4FF00008BF
:10BEC00078F0A0FC4FF00050B0F82E1100291BD0E4
:10BED0004FF00002A0F82E21B1FA81F26FEA0202BF
:10BEE00002F00F024FEA420241F61024C2F20004AF
:10BEF00040F25425C2F2000534F8029025F8029071
:10BF000009F07F091FF085BC90F8701011F0030153
:10BF100040F0568143F20004C4F2010490F870101E
:10BF200011F0040216D0238913F0020600F04881B4
:10BF300013F0800640F0448140F20046C4F202064D
:10BF40004FF04007B761227B80F82C2121F00401DB
:10BF500080F8701090F82B11002919D190F82C213D
:10BF60001B2A1BD040F20046C4F20206318A11F0AF
:10BF700080017ED14FF0010180F82B114FF0FF08B6
:10BF8000B0F87210B0F87420914240F0EE80FAE000
:10BF9000012916D190F82C211B2A0DD14FF0020156
:10BFA00080F82B114FF0FF08B0F87210B0F8742031
:10BFB000914240F0DA80E6E04FF0000180F82B116A
:10BFC00057E0022911D190F82C21412AF4D14FF0E9
:10BFD000030180F82B114FF0FF08B0F87210B0F891
:10BFE0007420914240F0C180CDE0032911D190F836
:10BFF0002C21012AE0D14FF0040180F82B114FF0E1
:10C00000FF08B0F87210B0F87420914240F0AD8093
:10C01000B9E04FF0000180F82B1190F82C21502A44
:10C0200015D2A2F10A0280F82D214FEA420241F610
:10C030001024C2F2000440F25425C2F2000534F884
:10C04000029025F8029009F07F091FF0E2BBA2F1EF
:10C0500050024FEA420240F2FF0580F82D5140F2B3
:10C060005425C2F2000535F8029009F07F0908F066
:10C070004ABBB0F87210B0F87420914275D190F8B4
:10C080007A13012919F05E8402291AF0B48390F81A
:10C09000BE13012915F0D48090F8391311F0010175
:10C0A00040F08E80D0F8C41311F0040200F08880B4
:10C0B00021F00401C0F8C41311F0010257F06A81A5
:10C0C00011F0020256F0748411F0100259F0E7806A
:10C0D00011F0200256F0418711F0400254F0B7846D
:10C0E00011F0800254F0AB8711F4807254F0DD85BA
:10C0F00011F400725CF0568311F4806256F05A839A
:10C1000011F4006256F0AF8711F480525CF045875D
:10C1100011F400525CF0D68211F480425CF0BF83CF
:10C1200011F4004257F0428011F480325CF07E83BB
:10C1300011F4003257F0038011F4802256F09D86EE
:10C1400011F400225CF0628211F4801254F0E68354
:10C1500011F4001254F03D8711F480025EF0108754
:10C1600011F400025EF001852AE040F20001C1F204
:10C17000000111F8028002F1010243F6FF7102EAA8
:10C180000102A0F874204FF0870380F8703040F26D
:10C190000046C4F202064FF00007C0F24007B76144
:10C1A00084F80C8042F20002C4F2000240F28501E1
:10C1B000C0F20001116040F20101C0F200015161C2
:10C1C0004FF0005041F20001C2F20001B1F81080BE
:10C1D00008F101084DF2847AC0F2170ABAFBF8FAA6
:10C1E00040F60042C4F20002C2F82CA04FF000500A
:10C1F00090F8F11011F0010144F0178490F8471104
:10C2000011F0010144F0118441F20001C2F2000179
:10C21000B0F8CE20002A04F00884A2F10102A0F8B0
:10C22000CE2090F86C2112F001020FD190F8212D50
:10C2300012F0040303D040F2F8087AF0D0FB12F0B9
:10C24000080303D040F2F8087AF097FE40F2B013EA
:10C25000C2F2000390F8C4404FEA44041A5BA0F80D
:10C26000D22090F8D530012B43F0418640F2B01532
:10C27000C2F2000590F8C4604FEA4606AA5B90F847
:10C280006C3113F0010318BF90F86D21002A16D10C
:10C2900090F86C3113F001030CD190F8BA6316F0EA
:10C2A000010236D016F0020204D090F8F06016F0C9
:10C2B00001022ED04FF0140580F8BC5329E090F80D
:10C2C000BB63B2FBF6F505FB06F5A2EB0506002EF7
:10C2D0001FD14FF06006B2FBF6F505FB06F5A2EBA9
:10C2E0000506002ED4D090F86C3113F001030CD168
:10C2F00090F8BA6316F001020BD016F0020204D0D7
:10C3000090F8F06016F0010203D04FF0280580F895
:10C31000BC5390F86C3113F001030BD090F86D31E1
:10C3200003F10103C02B08BF1CF00DBF80F86D3175
:10C3300004F07BBB90F8F02012F0010200F0B38112
:10C3400090F8942312F0010200F0AD81B0F8D220F1
:10C35000002A40F09C8190F8944314F002042FD1FD
:10C3600090F8B23380F8B33313F001030ED1426E6C
:10C370004FF480414FEA01418A429DF04D86B0F86A
:10C380006060B6F5006F9DF047860EE0D0F8B423EC
:10C390004FF480414FEA01418A429DF03D86B0F85A
:10C3A000B863B6F5805F9DF03786C0F8C422C0F848
:10C3B000EC2290F8FF1241F0010180F8FF1272E1C7
:10C3C0004FF0000180F8F0104FF0000180F8941356
:10C3D00073F0F7FE90F83D10002940F0548190F87A
:10C3E0002A11002940F04F8190F8D813002904D178
:10C3F00090F87110002940F046814FF0230878F042
:10C4000001FA4FF0460878F0FDF94FF05A0878F03D
:10C41000F9F94FF0380878F0F5F94FF02C0878F07A
:10C42000F1F94FF0310878F0EDF94FF0350878F078
:10C43000E9F94FF02C0878F0E5F94FF0230878F08F
:10C44000E1F94FF05A0878F0DDF94FF0460878F03E
:10C45000D9F94FF0310878F0D5F94FF0300878F07D
:10C46000D1F94FF02C0878F0CDF94FF0230878F08F
:10C47000C9F94FF05A0878F0C5F94FF0520878F032
:10C48000C1F94FF0340878F0BDF94FF0380878F072
:10C49000B9F94FF0300878F0B5F94FF02C0878F082
:10C4A000B1F94FF0310878F0ADF94FF0300878F07D
:10C4B000A9F94FF0300878F0A5F94FF02C0878F082
:10C4C000A1F94FF0520878F09DF94FF0650878F027
:10C4D00099F94FF0730878F095F94FF0650878F006
:10C4E00091F94FF0740878F08DF94FF0000878F06A
:10C4F00089F990F8B81011F0010100F0C48090F8AB
:10C500008F1211F0010140F0BE8090F8891311F0F4
:10C51000010140F0B88090F88C1311F0010140F057
:10C52000B28090F88D1311F0010140F0AC804FF013
:10C53000230878F067F94FF0460878F063F94FF078
:10C540005A0878F05FF94FF0380878F05BF94FF04F
:10C550002C0878F057F94FF0310878F053F94FF084
:10C560002C0878F04FF94FF0230878F04BF94FF092
:10C570005A0878F047F94FF0460878F043F94FF041
:10C58000310878F03FF94FF0300878F03BF94FF080
:10C590002C0878F037F94FF0230878F033F94FF092
:10C5A0005A0878F02FF94FF0520878F02BF94FF035
:10C5B000340878F027F94FF0380878F023F94FF075
:10C5C000300878F01FF94FF02C0878F01BF94FF085
:10C5D000310878F017F94FF0380878F013F94FF078
:10C5E000300878F00FF94FF02C0878F00BF94FF085
:10C5F000200878F007F94FF0200878F003F94FF0A1
:10C60000470878F0FFF84FF0720878F0FBF84FF029
:10C61000690878F0F7F84FF0640878F0F3F84FF015
:10C62000000878F0EFF84FF0230878F0EBF84FF0BF
:10C630005A0878F0E7F84FF0520878F0E3F84FF036
:10C64000300878F0DFF84FF02C0878F0DBF84FF086
:10C65000320878F0D7F84FF0300878F0D3F84FF080
:10C660002C0878F0CFF84FF0490878F0CBF84FF06D
:10C670006E0878F0C7F84FF0730878F0C3F84FF001
:10C68000000878F0BFF873F0C5FC1EF061B890F8B0
:10C69000944344F0020480F8944390F8FE4244F03E
:10C6A000010480F8FE4241F20001C2F20001B0F83C
:10C6B000B02140F20005C2F20105B1F8C0602E447D
:10C6C000B0F87041254443F2000CC2F2000CB542B0
:10C6D00061D24FEA94083CF80830934256D35AD1BD
:10C6E0004FF0000AB1F8007CD0F8803240F2FF1918
:10C6F00003EA09039F4207D2B1F8607C002F45D0BE
:10C700004FEA07674AEA070AB1F8207C4FEA970721
:10C71000836D03F07F0303FB07F34FEAD31303F0AA
:10C720007F034FEA03434AEA030AB1F8407CD0F89A
:10C73000843240F2FF1903EA090303FB07F34FEACF
:10C740001333B1F8807C17F001070CD141F6904902
:10C75000C2F20009877B4FEA4707B944B9F8007075
:10C760003B444AEA030A6B79002B0FD090F8D17151
:10C7700017F0050718BF80F8D231B1F8947117F09F
:10C78000010703D1B1F8523077F022FC05F108051A
:10C7900004F108049BE7A0F87041B0F8B22140F220
:10C7A0000005C2F20105B1F8C2602E44B1F8C040E4
:10C7B0002544B0F87241254443F2000CC2F2000C4B
:10C7C000B1F8C0704FEA9707BC44B54267D24FEA50
:10C7D00094083CF8083093425CD360D14FF0000AD3
:10C7E000B1F8027CD0F880324FEA530340F2FF19CF
:10C7F00003EA09039F4207D2B1F8627C002F49D0B7
:10C800004FEA07674AEA070AB1F8227C4FEA97071E
:10C81000836D4FEA530303F07F0303FB07F34FEAF3
:10C82000D31303F07F034FEA03434AEA030AB1F844
:10C83000427CD0F884324FEA530340F2FF1903EAF6
:10C84000090303FB07F34FEA1333B1F8807C17F0B9
:10C8500002070CD141F69049C2F20009877B4FEAEA
:10C860004707B944B9F800703B444AEA030A6B79B8
:10C87000002B0FD090F8D17117F0050718BF80F882
:10C88000D331B1F8947117F0020703D1B1F85430E5
:10C8900077F09EFB05F1080504F1080495E7A0F880
:10C8A0007241B0F8B42140F20005C2F20105B1F8BE
:10C8B000C4602E44B1F8C2402544B0F87441254408
:10C8C00043F2000CC2F2000CB1F8C2704FEA9707B5
:10C8D000BC44B54267D24FEA94083CF80830934212
:10C8E0005CD360D14FF0000AB1F8047CD0F88032FC
:10C8F0004FEA930340F2FF1903EA09039F4207D26C
:10C90000B1F8647C002F49D04FEA07674AEA070A6A
:10C91000B1F8247C4FEA9707836D4FEA930303F045
:10C920007F0303FB07F34FEAD31303F07F034FEAC0
:10C9300003434AEA030AB1F8447CD0F884324FEA50
:10C94000930340F2FF1903EA090303FB07F34FEADD
:10C950001333B1F8807C17F004070CD141F69049ED
:10C96000C2F20009877B4FEA4707B944B9F8007063
:10C970003B444AEA030A6B79002B0FD090F8D1713F
:10C9800017F0050718BF80F8D431B1F8947117F08B
:10C99000040703D1B1F8563077F01AFB05F108050A
:10C9A00004F1080495E7A0F87441B0F8B62140F20C
:10C9B0000005C2F20105B1F8C6602E44B1F8C440CA
:10C9C0002544B0F87641254443F2000CC2F2000C35
:10C9D000B1F8C4704FEA9707BC44B54267D24FEA3A
:10C9E00094083CF8083093425CD360D14FF0000AC1
:10C9F000B1F8067CD0F880324FEAD30340F2FF1939
:10CA000003EA09039F4207D2B1F8667C002F49D0A0
:10CA10004FEA07674AEA070AB1F8267C4FEA970708
:10CA2000836D4FEAD30303F07F0303FB07F34FEA61
:10CA3000D31303F07F034FEA03434AEA030AB1F832
:10CA4000467CD0F884324FEAD30340F2FF1903EA60
:10CA5000090303FB07F34FEA1333B1F8807C17F0A7
:10CA600008070CD141F69049C2F20009877B4FEAD2
:10CA70004707B944B9F800703B444AEA030A6B79A6
:10CA8000002B0FD090F8D17117F0050718BF80F870
:10CA9000D531B1F8947117F0080703D1B1F85830C7
:10CAA00077F096FA05F1080504F1080495E7A0F877
:10CAB0007641B0F8B82140F20005C2F20105B1F8A4
:10CAC000C8602E44B1F8C6402544B0F878412544EA
:10CAD00043F2000CC2F2000CB1F8C6704FEA97079F
:10CAE000BC44B54267D24FEA94083CF80830934200
:10CAF0005CD360D14FF0000AB1F8087CD0F88032E6
:10CB00004FEA131340F2FF1903EA09039F4207D2C9
:10CB1000B1F8687C002F49D04FEA07674AEA070A54
:10CB2000B1F8287C4FEA9707836D4FEA131303F09F
:10CB30007F0303FB07F34FEAD31303F07F034FEAAE
:10CB400003434AEA030AB1F8487CD0F884324FEA3A
:10CB5000131340F2FF1903EA090303FB07F34FEA3B
:10CB60001333B1F8807C17F010070CD141F69049CF
:10CB7000C2F20009877B4FEA4707B944B9F8007051
:10CB80003B444AEA030A6B79002B0FD090F8D1712D
:10CB900017F0050718BF80F8D631B1F8947117F077
:10CBA000100703D1B1F85A3077F012FA05F10805F1
:10CBB00004F1080495E7A0F87841B0F8BA2140F2F2
:10CBC0000005C2F20105B1F8CA602E44B1F8C840B0
:10CBD0002544B0F87A41254443F2000CC2F2000C1F
:10CBE000B1F8C8704FEA9707BC44B54267D24FEA24
:10CBF00094083CF8083093425CD360D14FF0000AAF
:10CC0000B1F80A7CD0F880324FEA531340F2FF1992
:10CC100003EA09039F4207D2B1F86A7C002F49D08A
:10CC20004FEA07674AEA070AB1F82A7C4FEA9707F2
:10CC3000836D4FEA531303F07F0303FB07F34FEABF
:10CC4000D31303F07F034FEA03434AEA030AB1F820
:10CC50004A7CD0F884324FEA531340F2FF1903EABA
:10CC6000090303FB07F34FEA1333B1F8807C17F095
:10CC700020070CD141F69049C2F20009877B4FEAA8
:10CC80004707B944B9F800703B444AEA030A6B7994
:10CC9000002B0FD090F8D17117F0050718BF80F85E
:10CCA000D731B1F8947117F0200703D1B1F85C3097
:10CCB00077F08EF905F1080504F1080495E7A0F86E
:10CCC0007A41B0F8BC2140F20005C2F20105B1F88A
:10CCD000CC602E44B1F8CA402544B0F87C412544CC
:10CCE00043F2000CC2F2000CB1F8CA704FEA970789
:10CCF000BC44B54267D24FEA94083CF808309342EE
:10CD00005CD360D14FF0000AB1F80C7CD0F88032CF
:10CD10004FEA931340F2FF1903EA09039F4207D237
:10CD2000B1F86C7C002F49D04FEA07674AEA070A3E
:10CD3000B1F82C7C4FEA9707836D4FEA931303F009
:10CD40007F0303FB07F34FEAD31303F07F034FEA9C
:10CD500003434AEA030AB1F84C7CD0F884324FEA24
:10CD6000931340F2FF1903EA090303FB07F34FEAA9
:10CD70001333B1F8807C17F040070CD141F690498D
:10CD8000C2F20009877B4FEA4707B944B9F800703F
:10CD90003B444AEA030A6B79002B0FD090F8D1711B
:10CDA00017F0050718BF80F8D831B1F8947117F063
:10CDB000400703D1B1F85E3077F00AF905F10805B4
:10CDC00004F1080495E7A0F87C41B0F8BE2140F2D8
:10CDD0000005C2F20105B1F8CE602E44B1F8CC4096
:10CDE0002544B0F87E41254443F2000CC2F2000C09
:10CDF000B1F8CC704FEA9707BC44B54267D24FEA0E
:10CE000094083CF8083093425CD360D14FF0000A9C
:10CE1000B1F80E7CD0F880324FEAD31340F2FF19FC
:10CE200003EA09039F4207D2B1F86E7C002F49D074
:10CE30004FEA07674AEA070AB1F82E7C4FEA9707DC
:10CE4000836D4FEAD31303F07F0303FB07F34FEA2D
:10CE5000D31303F07F034FEA03434AEA030AB1F80E
:10CE60004E7CD0F884324FEAD31340F2FF1903EA24
:10CE7000090303FB07F34FEA1333B1F8807C17F083
:10CE800080070CD141F69049C2F20009877B4FEA36
:10CE90004707B944B9F800703B444AEA030A6B7982
:10CEA000002B0FD090F8D17117F0050718BF80F84C
:10CEB000D931B1F8947117F0800703D1B1F860301F
:10CEC00077F086F805F1080504F1080495E7A0F865
:10CED0007E41B0F8C02140F20005C2F20105B1F870
:10CEE000D0602E44B1F8CE402544B0F880412544AE
:10CEF00043F2000CC2F2000CB1F8CE704FEA970773
:10CF0000BC44B5426CD24FEA94083CF808309342D6
:10CF100061D365D14FF0000AB1F8107CD0F88032AF
:10CF20004FEA132340F2FF1903EA09039F4207D295
:10CF3000B1F8707C002F4ED04FEA07674AEA070A23
:10CF4000B1F8307C4FEA9707836D4FEA132303F063
:10CF50007F0303FB07F34FEAD31303F07F034FEA8A
:10CF600003434AEA030AB1F8507CD0F884324FEA0E
:10CF7000132340F2FF1903EA090303FB07F34FEA07
:10CF80001333B1F8807C17F480770CD141F69049C7
:10CF9000C2F20009877B4FEA4707B944B9F800702D
:10CFA0003B444AEA030A6B79002B14D0B1F8B870FD
:10CFB00017F001070BD190F8D17117F0050718BFD2
:10CFC00080F8DA31B1F8947117F4807703D1B1F8B1
:10CFD000623076F0FDFF05F1080504F1080490E7E2
:10CFE000A0F88041B0F8C22140F20005C2F201056C
:10CFF000B1F8D2602E44B1F8D0402544B0F8824157
:10D00000254443F2000CC2F2000CB1F8D0704FEA94
:10D010009707BC44B5426CD24FEA94083CF80830FC
:10D02000934261D365D14FF0000AB1F8127CD0F879
:10D0300080324FEA532340F2FF1903EA09039F426B
:10D0400007D2B1F8727C002F4ED04FEA07674AEA48
:10D05000070AB1F8327C4FEA9707836D4FEA5323F2
:10D0600003F07F0303FB07F34FEAD31303F07F03BF
:10D070004FEA03434AEA030AB1F8527CD0F88432FB
:10D080004FEA532340F2FF1903EA090303FB07F3B6
:10D090004FEA1333B1F8807C17F400770CD141F6D6
:10D0A0009049C2F20009877B4FEA4707B944B9F8B3
:10D0B00000703B444AEA030A6B79002B14D0B1F8A4
:10D0C000B87017F002070BD190F8D17117F005076F
:10D0D00018BF80F8DB31B1F8947117F4007703D1F1
:10D0E000B1F8643076F074FF05F1080504F1080426
:10D0F00090E7A0F88241B0F8C42140F20005C2F2E6
:10D100000105B1F8D4602E44B1F8D2402544B0F8FE
:10D110008441254443F2000CC2F2000CB1F8D270F5
:10D120004FEA9707BC44B5426CD24FEA94083CF8EA
:10D130000830934261D365D14FF0000AB1F8147CF6
:10D14000D0F880324FEA932340F2FF1903EA090333
:10D150009F4207D2B1F8747C002F4ED04FEA076788
:10D160004AEA070AB1F8347C4FEA9707836D4FEA21
:10D17000932303F07F0303FB07F34FEAD31303F07A
:10D180007F034FEA03434AEA030AB1F8547CD0F81C
:10D1900084324FEA932340F2FF1903EA090303FBA9
:10D1A00007F34FEA1333B1F8807C17F480670CD192
:10D1B00041F69049C2F20009877B4FEA4707B9441C
:10D1C000B9F800703B444AEA030A6B79002B14D08B
:10D1D000B1F8B87017F004070BD190F8D17117F0BF
:10D1E000050718BF80F8DC31B1F8947117F4806737
:10D1F00003D1B1F8663076F0EBFE05F1080504F1D5
:10D20000080490E7A0F88441B0F8C62140F2000578
:10D21000C2F20105B1F8D6602E44B1F8D4402544DD
:10D22000B0F88641254443F2000CC2F2000CB1F87C
:10D23000D4704FEA9707BC44B5426CD24FEA9408C9
:10D240003CF80830934261D365D14FF0000AB1F841
:10D25000167CD0F880324FEAD32340F2FF1903EA5C
:10D2600009039F4207D2B1F8767C002F4ED04FEAD7
:10D2700007674AEA070AB1F8367C4FEA9707836DD9
:10D280004FEAD32303F07F0303FB07F34FEAD313E3
:10D2900003F07F034FEA03434AEA030AB1F8567CDE
:10D2A000D0F884324FEAD32340F2FF1903EA09038E
:10D2B00003FB07F34FEA1333B1F8807C17F40067E0
:10D2C0000CD141F69049C2F20009877B4FEA47072B
:10D2D000B944B9F800703B444AEA030A6B79002B61
:10D2E00014D0B1F8B87017F008070BD190F8D171CD
:10D2F00017F0050718BF80F8DD31B1F8947117F405
:10D30000006703D1B1F8683076F062FE05F10805D8
:10D3100004F1080490E7A0F88641B0F8C82140F273
:10D320000005C2F20105B1F8D8602E44B1F8D6402C
:10D330002544B0F88841254443F2000CC2F2000CA9
:10D34000B1F8D6704FEA9707BC44B5426CD24FEAA9
:10D3500094083CF80830934261D365D14FF0000A3D
:10D36000B1F8187CD0F880324FEA133340F2FF193D
:10D3700003EA09039F4207D2B1F8787C002F4ED010
:10D380004FEA07674AEA070AB1F8387C4FEA97077D
:10D39000836D4FEA133303F07F0303FB07F34FEA78
:10D3A000D31303F07F034FEA03434AEA030AB1F8B9
:10D3B000587CD0F884324FEA133340F2FF1903EA65
:10D3C000090303FB07F34FEA1333B1F8807C17F42A
:10D3D00080570CD141F69049C2F20009877B4FEA91
:10D3E0004707B944B9F800703B444AEA030A6B792D
:10D3F000002B14D0B1F8B87017F010070BD190F8CB
:10D40000D17117F0050718BF80F8DE31B1F89471BB
:10D4100017F4805703D1B1F86A3076F0D9FD05F1E1
:10D42000080504F1080490E7A0F88841B0F8CA2183
:10D4300040F20005C2F20105B1F8DA602E44B1F8FD
:10D44000D8402544B0F88A41254443F2000CC2F28A
:10D45000000CB1F8D8704FEA9707BC44B5426CD2C3
:10D460004FEA94083CF80830934261D365D14FF0FD
:10D47000000AB1F81A7CD0F880324FEA533340F2F8
:10D48000FF1903EA09039F4207D2B1F87A7C002F03
:10D490004ED04FEA07674AEA070AB1F83A7C4FEAEA
:10D4A0009707836D4FEA533303F07F0303FB07F3C2
:10D4B0004FEAD31303F07F034FEA03434AEA030A18
:10D4C000B1F85A7CD0F884324FEA533340F2FF1956
:10D4D00003EA090303FB07F34FEA1333B1F8807C37
:10D4E00017F400570CD141F69049C2F20009877B2E
:10D4F0004FEA4707B944B9F800703B444AEA030AC7
:10D500006B79002B14D0B1F8B87017F020070BD14D
:10D5100090F8D17117F0050718BF80F8DF31B1F826
:10D52000947117F4005703D1B1F86C3076F050FDC8
:10D5300005F1080504F1080490E7A0F88A41B0F865
:10D54000CC2140F20005C2F20105B1F8DC602E44A6
:10D55000B1F8DA402544B0F88C41254443F2000C80
:10D56000C2F2000CB1F8DA704FEA9707BC44B5423A
:10D570006CD24FEA94083CF80830934261D365D1ED
:10D580004FF0000AB1F81C7CD0F880324FEA933398
:10D5900040F2FF1903EA09039F4207D2B1F87C7CED
:10D5A000002F4ED04FEA07674AEA070AB1F83C7CE1
:10D5B0004FEA9707836D4FEA933303F07F0303FB32
:10D5C00007F34FEAD31303F07F034FEA03434AEA1A
:10D5D000030AB1F85C7CD0F884324FEA933340F20E
:10D5E000FF1903EA090303FB07F34FEA1333B1F80A
:10D5F000807C17F480470CD141F69049C2F20009B3
:10D60000877B4FEA4707B944B9F800703B444AEAC0
:10D61000030A6B79002B14D0B1F8B87017F04007EB
:10D620000BD190F8D17117F0050718BF80F8E031E1
:10D63000B1F8947117F4804703D1B1F86E3076F0E9
:10D64000C7FC05F1080504F1080490E7A0F88C4137
:10D65000B0F8CE2140F20005C2F20105B1F8DE605B
:10D660002E44B1F8DC402544B0F88E41254443F205
:10D67000000CC2F2000CB1F8DC704FEA9707BC4412
:10D68000B5426CD24FEA94083CF80830934261D31B
:10D6900065D14FF0000AB1F81E7CD0F880324FEA15
:10D6A000D33340F2FF1903EA09039F4207D2B1F8CE
:10D6B0007E7C002F4ED04FEA07674AEA070AB1F88E
:10D6C0003E7C4FEA9707836D4FEAD33303F07F0325
:10D6D00003FB07F34FEAD31303F07F034FEA03433F
:10D6E0004AEA030AB1F85E7CD0F884324FEAD333B9
:10D6F00040F2FF1903EA090303FB07F34FEA133370
:10D70000B1F8807C17F400470CD141F69049C2F281
:10D710000009877B4FEA4707B944B9F800703B44DA
:10D720004AEA030A6B79002B14D0B1F8B87017F0ED
:10D7300080070BD190F8D17117F0050718BF80F85A
:10D74000E131B1F8947117F4004703D1B1F87030AA
:10D7500076F03EFC05F1080504F1080490E7A0F816
:10D760008E41B0F8F84114F4807515D024F480741B
:10D77000A0F8F841B0F8C0214EF68075C2F200055D
:10D780006B79002B08D06B889A4205D14FF0000AC4
:10D79000B1F8623076F01CFCB0F8F84114F4007572
:10D7A00015D024F40074A0F8F841B0F8C2214EF668
:10D7B0008875C2F200056B79002B08D06B889A42FD
:10D7C00005D14FF0000AB1F8643076F001FCB0F8F2
:10D7D000F84114F4806515D024F48064A0F8F84171
:10D7E000B0F8C4214EF69075C2F200056B79002B9B
:10D7F00008D06B889A4205D14FF0000AB1F8663024
:10D8000076F0E6FBB0F8F84114F4006515D024F486
:10D810000064A0F8F841B0F8C6214EF69875C2F23F
:10D8200000056B79002B08D06B889A4205D14FF028
:10D83000000AB1F8683076F0CBFBB0F8F84114F488
:10D84000805515D024F48054A0F8F841B0F8C821D0
:10D850004EF6A075C2F200056B79002B08D06B88DC
:10D860009A4205D14FF0000AB1F86A3076F0B0FB69
:10D87000B0F8F84114F4005515D024F40054A0F881
:10D88000F841B0F8CA214EF6A875C2F200056B79CE
:10D89000002B08D06B889A4205D14FF0000AB1F8EE
:10D8A0006C3076F095FBB0F8F84114F4804515D053
:10D8B00024F48044A0F8F841B0F8CC214EF6B075BD
:10D8C000C2F200056B79002B08D06B889A4205D113
:10D8D0004FF0000AB1F86E3076F07AFBB0F8F841FC
:10D8E00014F4004515D024F40044A0F8F841B0F831
:10D8F000CE214EF6B875C2F200056B79002B08D028
:10D900006B889A4205D14FF0000AB1F8703076F07A
:10D910005FFB90F8B94014F0010426D040F2B01536
:10D92000C2F2000590F8C4604FEA4606AA5B4EF6C4
:10D930000075C2F2000505F140066B79002B10D08E
:10D940006B889A420DD14FF0000A41F25207C2F2A1
:10D95000000790F8C4804FEA480837F8083076F09E
:10D9600037FB05F10805B542E7D390F88D4314F075
:10D97000010404D190F88F4214F001042FD0B1F8C3
:10D98000944190F8C46024FA06F414F0010426D1FE
:10D9900040F2B015C2F2000590F8C4604FEA4606A6
:10D9A000AA5B4EF60075C2F2000505F140066B79E0
:10D9B000002B10D02B889A420DD14FF0000A41F273
:10D9C0005207C2F2000790F8C4804FEA480837F8BF
:10D9D000083076F034FD05F10805B542E7D3B0F81C
:10D9E000B02140F20005C2F20105B1F8E0602E441A
:10D9F000B1F8DE402544B0F890412544B54280F0AE
:10DA00001C816B889342C0F0138140F01681B1F8FD
:10DA1000947117F0010740F00B816F78032F2BD121
:10DA2000B1F8969119F0010922D1B1F8329019F0AC
:10DA300010080ED109F00F0909F1E00878F0CFFFC6
:10DA400095F8048078F0CBFF95F8058078F0C7FF53
:10DA5000EEE009F00F0909F1E00879F08EFA95F887
:10DA6000048079F08AFA95F8058079F086FADFE08B
:10DA70004B8E80F075FBDBE0042F2BD1B1F8969133
:10DA800019F0010922D1B1F8329019F010080ED125
:10DA900009F00F0909F1B00878F0A1FF95F80480AA
:10DAA00078F09DFF95F8058078F099FFC0E009F0C7
:10DAB0000F0909F1B00879F060FA95F8048079F05F
:10DAC0005CFA95F8058079F058FAB1E04B8E7FF05A
:10DAD000DCFDADE0052F20D1B1F8969119F00109D8
:10DAE0001AD1B1F8329019F010080AD109F00F09D3
:10DAF00009F1C00878F073FF95F8048078F06FFFA3
:10DB000096E009F00F0909F1C00879F036FA95F8A6
:10DB1000048079F032FA8BE08AE0062F23D1B1F845
:10DB2000969119F001091AD1B1F8329019F0100844
:10DB30000AD109F00F0909F1D00878F050FF95F8E3
:10DB4000048078F04CFF73E009F00F0909F1D00868
:10DB500079F013FA95F8048079F00FFA68E04B8EAB
:10DB600080F0ACF864E0072F28D1B1F8969119F055
:10DB7000010922D1B1F8329019F010080ED109F044
:10DB80000F0909F1A00878F02AFF95F8048078F0D1
:10DB900026FF95F8058078F022FF49E009F00F098B
:10DBA00009F1A00879F0E9F995F8048079F0E5F930
:10DBB00095F8058079F0E1F93AE039E00A2F19D1BA
:10DBC00095F8048078F00BFF95F8058078F007FF52
:10DBD000B8F1F70F2CD095F8068078F000FFB8F177
:10DBE000F70F25D095F8078078F0F9FEB8F1F70F18
:10DBF0001ED01DE00B2F1BD195F8048078F0EFFEAE
:10DC0000B8F1F70F14D095F8058078F0E8FEB8F178
:10DC1000F70F0DD095F8068078F0E1FEB8F1F70F18
:10DC200006D095F8078078F0DAFEB8F1F70FFFD04C
:10DC300005F1080504F10804E0E6A0F89041B0F809
:10DC4000B22140F20005C2F20105B1F8E2602E44B3
:10DC5000B1F8E0402544B0F892412544B54280F047
:10DC6000E1806B889342C0F0D88040F0DB80B1F84F
:10DC7000947117F0020740F0D0806F78032F2BD1FA
:10DC8000B1F8969119F0020922D1B1F8349019F047
:10DC900010080ED109F00F0909F1E00878F09FFE95
:10DCA00095F8048078F09BFE95F8058078F097FE53
:10DCB000B3E009F00F0909F1E00879F05EF995F891
:10DCC000048079F05AF995F8058079F056F9A4E0C6
:10DCD0008B8E80F045FAA0E0042F2BD1B1F89691FD
:10DCE00019F0020922D1B1F8349019F010080ED1C0
:10DCF00009F00F0909F1B00878F071FE95F8048079
:10DD000078F06DFE95F8058078F069FE85E009F001
:10DD10000F0909F1B00879F030F995F8048079F02D
:10DD20002CF995F8058079F028F976E08B8E7FF054
:10DD3000ACFC72E0052F20D1B1F8969119F00209E0
:10DD40001AD1B1F8349019F010080AD109F00F096E
:10DD500009F1C00878F043FE95F8048078F03FFEA2
:10DD60005BE009F00F0909F1C00879F006F995F8B0
:10DD7000048079F002F950E04FE0062F23D1B1F88A
:10DD8000969119F002091AD1B1F8349019F01008DF
:10DD90000AD109F00F0909F1D00878F020FE95F8B2
:10DDA000048078F01CFE38E009F00F0909F1D00872
:10DDB00079F0E3F895F8048079F0DFF82DE08B8EA8
:10DDC0007FF07CFF29E0072F27D1B1F8969119F059
:10DDD000020922D1B1F8349019F010080ED109F0DF
:10DDE0000F0909F1A00878F0FAFD95F8048078F0A1
:10DDF000F6FD95F8058078F0F2FD0EE009F00F09C8
:10DE000009F1A00879F0B9F895F8048079F0B5F82F
:10DE100095F8058079F0B1F8FFE705F1080504F100
:10DE200008041BE7A0F89241B0F8B42140F20005C5
:10DE3000C2F20105B1F8E4602E44B1F8E240254495
:10DE4000B0F894412544B54280F0E1806B8893425C
:10DE5000C0F0D88040F0DB80B1F8947117F004076F
:10DE600040F0D0806F78032F2BD1B1F8969119F044
:10DE7000040922D1B1F8369019F010080ED109F03A
:10DE80000F0909F1E00878F0AAFD95F8048078F010
:10DE9000A6FD95F8058078F0A2FDB3E009F00F0922
:10DEA00009F1E00879F069F895F8048079F065F8EF
:10DEB00095F8058079F061F8A4E0CB8E80F050F9F8
:10DEC000A0E0042F2BD1B1F8969119F0040922D1CA
:10DED000B1F8369019F010080ED109F00F0909F1C8
:10DEE000B00878F07CFD95F8048078F078FD95F81E
:10DEF000058078F074FD85E009F00F0909F1B0089C
:10DF000079F03BF895F8048079F037F895F80580BA
:10DF100079F033F876E0CB8E7FF0B7FB72E0052F17
:10DF200020D1B1F8969119F004091AD1B1F83690C0
:10DF300019F010080AD109F00F0909F1C00878F0AA
:10DF40004EFD95F8048078F04AFD5BE009F00F097A
:10DF500009F1C00879F011F895F8048079F00DF80E
:10DF600050E04FE0062F23D1B1F8969119F0040943
:10DF70001AD1B1F8369019F010080AD109F00F093A
:10DF800009F1D00878F02BFD95F8048078F027FD92
:10DF900038E009F00F0909F1D00878F0EEFF95F8A4
:10DFA000048078F0EAFF2DE0CB8E7FF087FE29E039
:10DFB000072F27D1B1F8969119F0040922D1B1F8B1
:10DFC000369019F010080ED109F00F0909F1A008D8
:10DFD00078F005FD95F8048078F001FD95F805804E
:10DFE00078F0FDFC0EE009F00F0909F1A00878F0C7
:10DFF000C4FF95F8048078F0C0FF95F8058078F0AC
:10E00000BCFFFFE705F1080504F108041BE7A0F8D1
:10E010009441B0F8B62140F20005C2F20105B1F812
:10E02000E6602E44B1F8E4402544B0F8964125441A
:10E03000B54280F0E1806B889342C0F0D88040F018
:10E04000DB80B1F8947117F0080740F0D0806F784A
:10E05000032F2BD1B1F8969119F0080922D1B1F80C
:10E06000389019F010080ED109F00F0909F1E008F5
:10E0700078F0B5FC95F8048078F0B1FC95F805804F
:10E0800078F0ADFCB3E009F00F0909F1E00878F091
:10E0900074FF95F8048078F070FF95F8058078F0AB
:10E0A0006CFFA4E00B8F80F05BF8A0E0042F2BD175
:10E0B000B1F8969119F0080922D1B1F8389019F009
:10E0C00010080ED109F00F0909F1B00878F087FCAB
:10E0D00095F8048078F083FC95F8058078F07FFC53
:10E0E00085E009F00F0909F1B00878F046FF95F8CE
:10E0F000048078F042FF95F8058078F03EFF76E0E6
:10E100000B8F7FF0C2FA72E0052F20D1B1F8969103
:10E1100019F008091AD1B1F8389019F010080AD18D
:10E1200009F00F0909F1C00878F059FC95F804804E
:10E1300078F055FC5BE009F00F0909F1C00878F0B0
:10E140001CFF95F8048078F018FF50E04FE0062F90
:10E1500023D1B1F8969119F008091AD1B1F8389085
:10E1600019F010080AD109F00F0909F1D00878F068
:10E1700036FC95F8048078F032FC38E009F00F099D
:10E1800009F1D00878F0F9FE95F8048078F0F5FEF2
:10E190002DE00B8F7FF092FD29E0072F27D1B1F8FA
:10E1A000969119F0080922D1B1F8389019F01008A9
:10E1B0000ED109F00F0909F1A00878F010FC95F8CC
:10E1C000048078F00CFC95F8058078F008FC0EE0EF
:10E1D00009F00F0909F1A00878F0CFFE95F8048046
:10E1E00078F0CBFE95F8058078F0C7FEFFE705F1E3
:10E1F000080504F108041BE7A0F89641B0F8B8211F
:10E2000040F20005C2F20105B1F8E8602E44B1F811
:10E21000E6402544B0F898412544B54280F0E180BD
:10E220006B889342C0F0D88040F0DB80B1F89471E5
:10E2300017F0100740F0D0806F78032F2BD1B1F882
:10E24000969119F0100922D1B1F83A9019F01008FE
:10E250000ED109F00F0909F1E00878F0C0FB95F83C
:10E26000048078F0BCFB95F8058078F0B8FBB3E04B
:10E2700009F00F0909F1E00878F07FFE95F80480B5
:10E2800078F07BFE95F8058078F077FEA4E04B8F60
:10E290007FF066FFA0E0042F2BD1B1F8969119F022
:10E2A000100922D1B1F83A9019F010080ED109F0F6
:10E2B0000F0909F1B00878F092FB95F8048078F026
:10E2C0008EFB95F8058078F08AFB85E009F00F0950
:10E2D00009F1B00878F051FE95F8048078F04DFE11
:10E2E00095F8058078F049FE76E04B8F7FF0CDF908
:10E2F00072E0052F20D1B1F8969119F010091AD1CA
:10E30000B1F83A9019F010080AD109F00F0909F193
:10E31000C00878F064FB95F8048078F060FB5BE05F
:10E3200009F00F0909F1C00878F027FE95F804807C
:10E3300078F023FE50E04FE0062F23D1B1F89691FC
:10E3400019F010091AD1B1F83A9019F010080AD151
:10E3500009F00F0909F1D00878F041FB95F8048025
:10E3600078F03DFB38E009F00F0909F1D00878F0AA
:10E3700004FE95F8048078F000FE2DE04B8F7FF0CE
:10E380009DFC29E0072F27D1B1F8969119F01009CB
:10E3900022D1B1F83A9019F010080ED109F00F0906
:10E3A00009F1A00878F01BFB95F8048078F017FBC2
:10E3B00095F8058078F013FB0EE009F00F0909F1DC
:10E3C000A00878F0DAFD95F8048078F0D6FD95F88D
:10E3D000058078F0D2FDFFE705F1080504F1080497
:10E3E0001BE7A0F89841B0F8BA2140F20005C2F24C
:10E3F0000105B1F8EA602E44B1F8E8402544B0F8D0
:10E400009A412544B54280F0E1806B889342C0F088
:10E41000D88040F0DB80B1F8947117F0200740F00D
:10E42000D0806F78032F2BD1B1F8969119F0200985
:10E4300022D1B1F83C9019F010080ED109F00F0963
:10E4400009F1E00878F0CBFA95F8048078F0C7FA83
:10E4500095F8058078F0C3FAB3E009F00F0909F1E7
:10E46000E00878F08AFD95F8048078F086FD95F84C
:10E47000058078F082FDA4E08B8F7FF071FEA0E034
:10E48000042F2BD1B1F8969119F0200922D1B1F8BF
:10E490003C9019F010080ED109F00F0909F1B008ED
:10E4A00078F09DFA95F8048078F099FA95F805804F
:10E4B00078F095FA85E009F00F0909F1B00878F0D5
:10E4C0005CFD95F8048078F058FD95F8058078F0AB
:10E4D00054FD76E08B8F7FF0D8F872E0052F20D1C5
:10E4E000B1F8969119F020091AD1B1F83C9019F0C1
:10E4F00010080AD109F00F0909F1C00878F06FFA85
:10E5000095F8048078F06BFA5BE009F00F0909F1E7
:10E51000C00878F032FD95F8048078F02EFD50E0C8
:10E520004FE0062F23D1B1F8969119F020091AD1A6
:10E53000B1F83C9019F010080AD109F00F0909F15F
:10E54000D00878F04CFA95F8048078F048FA38E072
:10E5500009F00F0909F1D00878F00FFD95F8048053
:10E5600078F00BFD2DE08B8F7FF0A8FB29E0072FC3
:10E5700027D1B1F8969119F0200922D1B1F83C9039
:10E5800019F010080ED109F00F0909F1A00878F070
:10E5900026FA95F8048078F022FA95F8058078F04C
:10E5A0001EFA0EE009F00F0909F1A00878F0E5FC69
:10E5B00095F8048078F0E1FC95F8058078F0DDFCB2
:10E5C000FFE705F1080504F108041BE7A0F89A41EC
:10E5D000B0F8BC2140F20005C2F20105B1F8EC60D0
:10E5E0002E44B1F8EA402544B0F89C412544B54298
:10E5F00080F0E1806B889342C0F0D88040F0DB80EF
:10E60000B1F8947117F0400740F0D0806F78032F75
:10E610002BD1B1F8969119F0400922D1B1F83E9072
:10E6200019F010080ED109F00F0909F1E00878F08F
:10E63000D6F995F8048078F0D2F995F8058078F04D
:10E64000CEF9B3E009F00F0909F1E00878F095FC84
:10E6500095F8048078F091FC95F8058078F08DFCB1
:10E66000A4E0CB8F7FF07CFDA0E0042F2BD1B1F88C
:10E67000969119F0400922D1B1F83E9019F0100896
:10E680000ED109F00F0909F1B00878F0A8F995F852
:10E69000048078F0A4F995F8058078F0A0F985E079
:10E6A00009F00F0909F1B00878F067FC95F80480CB
:10E6B00078F063FC95F8058078F05FFC76E0CB8F0E
:10E6C0007EF0E3FF72E0052F20D1B1F8969119F0AA
:10E6D00040091AD1B1F83E9019F010080AD109F09A
:10E6E0000F0909F1C00878F07AF995F8048078F0FC
:10E6F00076F95BE009F00F0909F1C00878F03DFCFC
:10E7000095F8048078F039FC50E04FE0062F23D1D3
:10E71000B1F8969119F040091AD1B1F83E9019F06C
:10E7200010080AD109F00F0909F1D00878F057F95B
:10E7300095F8048078F053F938E009F00F0909F1F1
:10E74000D00878F01AFC95F8048078F016FC2DE0DB
:10E75000CB8F7FF0B3FA29E0072F27D1B1F896913C
:10E7600019F0400922D1B1F83E9019F010080ED1ED
:10E7700009F00F0909F1A00878F031F995F8048043
:10E7800078F02DF995F8058078F029F90EE009F078
:10E790000F0909F1A00878F0F0FB95F8048078F0F3
:10E7A000ECFB95F8058078F0E8FBFFE705F108053C
:10E7B00004F108041BE7A0F89C41B0F8BE2140F228
:10E7C0000005C2F20105B1F8EE602E44B1F8EC404C
:10E7D0002544B0F89E412544B54280F0E4806B8822
:10E7E0009342C0F0DB8040F0DE80B1F8947117F006
:10E7F000800740F0D3806F78032F2CD1B1F8969129
:10E8000019F0800922D1B1F8409019F010080ED10A
:10E8100009F00F0909F1E00878F0E1F895F80480B3
:10E8200078F0DDF895F8058078F0D9F8B6E009F0D1
:10E830000F0909F1E00878F0A0FB95F8048078F062
:10E840009CFB95F8058078F098FBA7E0B1F8403084
:10E850007FF086FCA2E0042F2CD1B1F8969119F03C
:10E86000800922D1B1F8409019F010080ED109F0BA
:10E870000F0909F1B00878F0B2F895F8048078F043
:10E88000AEF895F8058078F0AAF887E009F00F094E
:10E8900009F1B00878F071FB95F8048078F06DFB11
:10E8A00095F8058078F069FB78E0B1F840307EF0AB
:10E8B000ECFE73E0052F20D1B1F8969119F0800994
:10E8C0001AD1B1F8409019F010080AD109F00F09D7
:10E8D00009F1C00878F083F895F8048078F07FF8A3
:10E8E0005CE009F00F0909F1C00878F046FB95F8E3
:10E8F000048078F042FB51E050E0062F24D1B1F8BB
:10E90000969119F080091AD1B1F8409019F01008C9
:10E910000AD109F00F0909F1D00878F060F895F8EC
:10E92000048078F05CF839E009F00F0909F1D008AB
:10E9300078F023FB95F8048078F01FFB2EE0B1F807
:10E9400040307FF0BBF929E0072F27D1B1F896912D
:10E9500019F0800922D1B1F8409019F010080ED1B9
:10E9600009F00F0909F1A00878F039F895F804804A
:10E9700078F035F895F8058078F031F80EE009F078
:10E980000F0909F1A00878F0F8FA95F8048078F0FA
:10E99000F4FA95F8058078F0F0FAFFE705F108053C
:10E9A00004F1080418E7A0F89E41B0F8C02140F235
:10E9B0000005C2F20105B1F8F0602E44B1F8EE4056
:10E9C0002544B0F8A0412544B54280F0E4806B882E
:10E9D0009342C0F0DB8040F0DE80B1F8947117F410
:10E9E000807740F0D3806F78032F2CD1B1F89691C7
:10E9F00019F4807922D1B1F8429019F010080ED1A3
:10EA000009F00F0909F1E00877F0E9FF95F80480B3
:10EA100077F0E5FF95F8058077F0E1FFB6E009F0C3
:10EA20000F0909F1E00878F0A8FA95F8048078F069
:10EA3000A4FA95F8058078F0A0FAA7E0B1F8423082
:10EA40007FF08EFBA2E0042F2CD1B1F8969119F43F
:10EA5000807922D1B1F8429019F010080ED109F056
:10EA60000F0909F1B00877F0BAFF95F8048077F044
:10EA7000B6FF95F8058077F0B2FF87E009F00F093F
:10EA800009F1B00878F079FA95F8048078F075FA11
:10EA900095F8058078F071FA78E0B1F842307EF0B0
:10EAA000F4FD73E0052F20D1B1F8969119F4807927
:10EAB0001AD1B1F8429019F010080AD109F00F09E3
:10EAC00009F1C00877F08BFF95F8048077F087FF95
:10EAD0005CE009F00F0909F1C00878F04EFA95F8EA
:10EAE000048078F04AFA51E050E0062F24D1B1F8C2
:10EAF000969119F480791AD1B1F8429019F0100862
:10EB00000AD109F00F0909F1D00877F068FF95F8EC
:10EB1000048077F064FF39E009F00F0909F1D008AB
:10EB200078F02BFA95F8048078F027FA2EE0B1F807
:10EB300042307FF0C3F829E0072F27D1B1F8969132
:10EB400019F4807922D1B1F8429019F010080ED151
:10EB500009F00F0909F1A00877F041FF95F804804A
:10EB600077F03DFF95F8058077F039FF0EE009F06A
:10EB70000F0909F1A00878F000FA95F8048078F000
:10EB8000FCF995F8058078F0F8F9FFE705F108053C
:10EB900004F1080418E7A0F8A041B0F8C22140F23F
:10EBA0000005C2F20105B1F8F2602E44B1F8F04060
:10EBB0002544B0F8A2412544B54280F0E4806B883A
:10EBC0009342C0F0DB8040F0DE80B1F8947117F41E
:10EBD000007740F0D3806F78032F2CD1B1F8969155
:10EBE00019F4007922D1B1F8449019F010080ED12F
:10EBF00009F00F0909F1E00877F0F1FE95F80480BB
:10EC000077F0EDFE95F8058077F0E9FEB6E009F0C3
:10EC10000F0909F1E00878F0B0F995F8048078F070
:10EC2000ACF995F8058078F0A8F9A7E0B1F8443080
:10EC30007FF096FAA2E0042F2CD1B1F8969119F446
:10EC4000007922D1B1F8449019F010080ED109F0E2
:10EC50000F0909F1B00877F0C2FE95F8048077F04B
:10EC6000BEFE95F8058077F0BAFE87E009F00F093F
:10EC700009F1B00878F081F995F8048078F07DF911
:10EC800095F8058078F079F978E0B1F844307EF0B5
:10EC9000FCFC73E0052F20D1B1F8969119F40079AE
:10ECA0001AD1B1F8449019F010080AD109F00F09EF
:10ECB00009F1C00877F093FE95F8048077F08FFE95
:10ECC0005CE009F00F0909F1C00878F056F995F8F1
:10ECD000048078F052F951E050E0062F24D1B1F8C9
:10ECE000969119F400791AD1B1F8449019F01008EE
:10ECF0000AD109F00F0909F1D00877F070FE95F8F4
:10ED0000048077F06CFE39E009F00F0909F1D008B2
:10ED100078F033F995F8048078F02FF92EE0B1F807
:10ED200044307EF0CBFF29E0072F27D1B1F8969130
:10ED300019F4007922D1B1F8449019F010080ED1DD
:10ED400009F00F0909F1A00877F049FE95F8048051
:10ED500077F045FE95F8058077F041FE0EE009F06A
:10ED60000F0909F1A00878F008F995F8048078F007
:10ED700004F995F8058078F000F9FFE705F108053A
:10ED800004F1080418E7A0F8A241B0F8C42140F249
:10ED90000005C2F20105B1F8F4602E44B1F8F2406A
:10EDA0002544B0F8A4412544B54280F0E4806B8846
:10EDB0009342C0F0DB8040F0DE80B1F8947117F42C
:10EDC000806740F0D3806F78032F2CD1B1F89691F3
:10EDD00019F4806922D1B1F8469019F010080ED1CB
:10EDE00009F00F0909F1E00877F0F9FD95F80480C2
:10EDF00077F0F5FD95F8058077F0F1FDB6E009F0C4
:10EE00000F0909F1E00878F0B8F895F8048078F077
:10EE1000B4F895F8058078F0B0F8A7E0B1F846307E
:10EE20007FF09EF9A2E0042F2CD1B1F8969119F44D
:10EE3000806922D1B1F8469019F010080ED109F07E
:10EE40000F0909F1B00877F0CAFD95F8048077F052
:10EE5000C6FD95F8058077F0C2FD87E009F00F093F
:10EE600009F1B00878F089F895F8048078F085F811
:10EE700095F8058078F081F878E0B1F846307EF0BA
:10EE800004FC73E0052F20D1B1F8969119F4806944
:10EE90001AD1B1F8469019F010080AD109F00F09FB
:10EEA00009F1C00877F09BFD95F8048077F097FD95
:10EEB0005CE009F00F0909F1C00878F05EF895F8F8
:10EEC000048078F05AF851E050E0062F24D1B1F8D0
:10EED000969119F480691AD1B1F8469019F010088A
:10EEE0000AD109F00F0909F1D00877F078FD95F8FB
:10EEF000048077F074FD39E009F00F0909F1D008BA
:10EF000078F03BF895F8048078F037F82EE0B1F807
:10EF100046307EF0D3FE29E0072F27D1B1F8969135
:10EF200019F4806922D1B1F8469019F010080ED179
:10EF300009F00F0909F1A00877F051FD95F8048058
:10EF400077F04DFD95F8058077F049FD0EE009F06A
:10EF50000F0909F1A00878F010F895F8048078F00E
:10EF60000CF895F8058078F008F8FFE705F108053A
:10EF700004F1080418E7A0F8A441B0F8C62140F253
:10EF80000005C2F20105B1F8F6602E44B1F8F44074
:10EF90002544B0F8A6412544B54280F0E4806B8852
:10EFA0009342C0F0DB8040F0DE80B1F8947117F43A
:10EFB000006740F0D3806F78032F2CD1B1F8969181
:10EFC00019F4006922D1B1F8489019F010080ED157
:10EFD00009F00F0909F1E00877F001FD95F80480C8
:10EFE00077F0FDFC95F8058077F0F9FCB6E009F0C4
:10EFF0000F0909F1E00877F0C0FF95F8048077F079
:10F00000BCFF95F8058077F0B8FFA7E0B1F848306D
:10F010007FF0A6F8A2E0042F2CD1B1F8969119F454
:10F02000006922D1B1F8489019F010080ED109F00A
:10F030000F0909F1B00877F0D2FC95F8048077F059
:10F04000CEFC95F8058077F0CAFC87E009F00F093F
:10F0500009F1B00877F091FF95F8048077F08DFF03
:10F0600095F8058077F089FF78E0B1F848307EF0B8
:10F070000CFB73E0052F20D1B1F8969119F40069CB
:10F080001AD1B1F8489019F010080AD109F00F0907
:10F0900009F1C00877F0A3FC95F8048077F09FFC95
:10F0A0005CE009F00F0909F1C00877F066FF95F8F8
:10F0B000048077F062FF51E050E0062F24D1B1F8D0
:10F0C000969119F400691AD1B1F8489019F0100816
:10F0D0000AD109F00F0909F1D00877F080FC95F802
:10F0E000048077F07CFC39E009F00F0909F1D008C1
:10F0F00077F043FF95F8048077F03FFF2EE0B1F8FA
:10F1000048307EF0DBFD29E0072F27D1B1F896913A
:10F1100019F4006922D1B1F8489019F010080ED105
:10F1200009F00F0909F1A00877F059FC95F804805F
:10F1300077F055FC95F8058077F051FC0EE009F06A
:10F140000F0909F1A00877F018FF95F8048077F00F
:10F1500014FF95F8058077F010FFFFE705F108052B
:10F1600004F1080418E7A0F8A641B0F8C82140F25D
:10F170000005C2F20105B1F8F8602E44B1F8F6407E
:10F180002544B0F8A8412544B54280F0E4806B885E
:10F190009342C0F0DB8040F0DE80B1F8947117F448
:10F1A000805740F0D3806F78032F2CD1B1F896911F
:10F1B00019F4805922D1B1F84A9019F010080ED1F3
:10F1C00009F00F0909F1E00877F009FC95F80480CF
:10F1D00077F005FC95F8058077F001FCB6E009F0C2
:10F1E0000F0909F1E00877F0C8FE95F8048077F080
:10F1F000C4FE95F8058077F0C0FEA7E0B1F84A306C
:10F200007EF0AEFFA2E0042F2CD1B1F8969119F454
:10F21000805922D1B1F84A9019F010080ED109F0A6
:10F220000F0909F1B00877F0DAFB95F8048077F060
:10F23000D6FB95F8058077F0D2FB87E009F00F093F
:10F2400009F1B00877F099FE95F8048077F095FE03
:10F2500095F8058077F091FE78E0B1F84A307EF0BD
:10F2600014FA73E0052F20D1B1F8969119F4805962
:10F270001AD1B1F84A9019F010080AD109F00F0913
:10F2800009F1C00877F0ABFB95F8048077F0A7FB95
:10F290005CE009F00F0909F1C00877F06EFE95F8FF
:10F2A000048077F06AFE51E050E0062F24D1B1F8D7
